:020000040800F2
:1000000018250020D500000819980008A9700008DC
:1000100000000000000000000000000000000000E0
:100020000000000000000000000000007FC5000884
:100030000000000000000000C5A600081DEA00083E
:10004000E7000008E7000008B3AE0008E70000087A
:10005000E7000008692D0008792D0008892D0008A7
:10006000E7000008E7000008E7000008AD2C0008E2
:10007000E7000008E7000008E7000008E7000008C4
:10008000E7000008E7000008E700000800000000A3
:1000900005EB0008E7000008E7000008E70000089B
:1000A000E7000008E7000008E70000086DF400081A
:1000B000E70000084DAE000800000000E70000085F
:1000C0000348854600F09EFF004800476130010864
:1000D000182500200448804704480047FEE7FEE753
:1000E000FEE7FEE7FEE7FEE7B1EA0008C100000810
:1000F00030B50B46014600202022012409E00D46C0
:10010000D5409D4205D31D469540491B2546954047
:1001100040191546521E002DF1DC30BD70B500248B
:100120002546002801DA01244042002901DA012590
:100130004942FFF7DDFFAC4200D04042002C00D026
:10014000494270BDF0B51FB40646002082B0054696
:100150004024019100901BE0019922460F46304651
:1001600000F03EFD049A059B801A994110D3104679
:100170001946224600F024FD361A8F410197224687
:1001800001200021009F00F01BFD38184D41009018
:100190002046641E0028DFDC019B00982946324679
:1001A00007B0F0BDF0B51FB486B0002000900190FC
:1001B00002900698069980B204900798090C0204F0
:1001C0000014114307900027089D099806913E46A8
:1001D0003C4603900398A9B20204000C03900498D3
:1001E0002D0C154348430021224600F0E9FCC719B5
:1001F000714110340E46402CECDB3846029A00F078
:10020000DFFC009A019B80180090594102980191EF
:10021000103002904028CCDB00980BB0F0BD0346B4
:100220000B439B0703D009E008C9121F08C0042A2A
:10023000FAD203E00B780370401C491C521EF9D21D
:100240007047D2B201E00270401C491EFBD27047D9
:100250000022F6E710B513460A4604461946FFF792
:10026000F0FF204610BD10B5044605E00B78037082
:10027000401C002B00D0491C521EF7D2204610BD56
:10028000421C0178401C0029FBD1801A704710B530
:10029000002200E0521C835C8C5CA34201D1002B45
:1002A000F8D1D8B2E1B2401A10BD03460A78027004
:1002B000401C491C002AF9D11846704730B5054644
:1002C0000020034600E05B1C934205D2EC5CC85C56
:1002D000201A01D1002CF6D130BD0321001D401E93
:1002E000037812021A43491EF9D5104670470000E0
:1002F0000FB400B58DB009900B9010A900200091AB
:10030000C0430A9000200C900648069006480790CB
:100310006A4609A80F9900F09DFC0DB008BC04B016
:1003200018470000750C0008950C0008FFB5002761
:10033000FF4383B000205C6801909E681D46A96958
:100340007F1C049888470090296A88470028F6D1C6
:100350000098401C0CD0032040028443002E19DD7D
:10036000600614D500982B2809D02D280FD103E062
:100370000020C04307B0F0BD012080020443A969FA
:100380007F1C04988847761E0090002E02DD00989E
:10039000302803D00598002825D035E00120400200
:1003A0000443A969761E7F1C049888470090002E9C
:1003B00003DD782805D0582803D00598002810D0F0
:1003C00022E00598002801D010281DD1012040020C
:1003D0008443A969761E7F1C0498884700901020EA
:1003E00002E0082000E00A2005900DE0012149020A
:1003F0000C43059A0199761E514308180190A9698A
:100400007F1C049888470090002E05DD0599009810
:1004100000F00AFC0028E9DAE96904988847A00599
:1004200002D40120C043A5E7E00722D1600611D520
:100430006005019800D5404229680A1D2A600968B4
:10044000220501D5087014E0220701D5088010E0CC
:1004500008600EE02868011D29600068210502D5AA
:100460000199017005E02107019901D5018000E0A3
:10047000016038467EE770B506460FF0FFF8046865
:1004800005460A220021304600F016FC2C6070BDA3
:10049000F8B502464A40D40F42004B0052085B08B0
:1004A0009A4202D20246084611464A0023D0C30DA2
:1004B0004A00DDB2120EAD1A202D35DA49020126AE
:1004C000490AF6058A19002C00D0524220214F1B00
:1004D0001146B9402A411018C20D9A4221D0002C71
:1004E00017D0012D08DCDA05801AD20F8019D20747
:1004F000DBB200F021FCF8BDDA05801A01234000D0
:100500001B06C01880185A428018CA0F10434900B1
:1005100007E04908C2071143DA05801A801940082C
:10052000801800F001FCF8BD61000122511A001B87
:10053000F7E70122D2075140AAE70122D207504033
:10054000A6E7024670B54A40D30FDB0740002DD026
:100550004A002AD0010E140E000212020919400AA4
:10056000520A8418E50104465443000A120A2E0474
:100570005043A4194219200CC543AA18120C012596
:10058000AD03521C521912047F39240400D0521CAE
:10059000104301D44000491EC2B20C06C009201805
:1005A000401C4008802A02D003E0002070BD4008B3
:1005B0004000002900DA0020184370BD70B50246E3
:1005C0004A40D50F40004A00ED0740085208002875
:1005D00014D0002A12D0C40DD30D41020120C00551
:1005E0005202490A520AE41A091812187D3491423B
:1005F00001D3641C00E04900002C01DA002070BD2A
:100600000023914201D3891A03434008490000287E
:10061000F7D100290AD0914202D10121C90705E092
:10062000914201D2012101E00121C943E005C01836
:10063000401900F079FB70BD420005D04200120E57
:1006400052428A4201DB00207047C90508187047F2
:10065000F0B507460846584087B0C00F04904800E0
:100660000E46590040084908BC1A884105D2384650
:1006700031461E4617460B460246580040081043B6
:100680004CD0300D039040055900400D490D0590A8
:10069000401A0290402872DA18030121000B090564
:1006A0000843019004980092002805D00199524215
:1006B0000020884100920190029840210A1A019975
:1006C000009800F07DFA05460C466B4607CB00F01B
:1006D00098FAC0197141039A0E0D0023D71756409E
:1006E0001A467A40164344D0049A002A2DD0029A22
:1006F000012A039A15DC1205C01A9141012636051C
:10070000001C7141D20F059ED20700930192029600
:100710002A46234600F075FB07B0F0BD3846314647
:10072000FAE71605224A0F46B218C01AB74101214E
:100730000905001C4F4100187F41114618187941E6
:10074000E20F10436D19644113E0E2076D08154391
:100750006408C2071443039A01261205C01A914186
:100760003605001C7141CE07400830434908C018C7
:1007700051412A46234600F037FBCDE7FFE70498B6
:1007800001224000C117121A00238B410498314600
:10079000C417381AA141EEE730B40124E4076340DE
:1007A00030BC55E730B40124E407614030BC4FE76A
:1007B0000000E0FFF0B51FB488B00B990998002441
:1007C00048400999C00F490049080991C0070B9991
:1007D0000090490049080B9109990898A6460843DA
:1007E0001CD00B990A98084318D00998012440009E
:1007F000420D4800410D099824050003000B2043D9
:1008000009900B980003000B20430B9050181C49D3
:100810004018002201901446104605E000200146D1
:100820000DB0F0BD032801DA034600E003239C4627
:10083000C11A0AAE0AE05F0008ADED5B4F00F75B3E
:100840007D430027AA187C41491C5B1E6145F2DDEF
:10085000410004AB5A522104120C0A43240C401CE0
:100860000828DFDB01980290009970460191009002
:10087000059B049A0799069800F0C3FAD0E7000098
:100880000DFCFFFFF0B50C465C4085B0E40FE407BB
:1008900003944C0000266408590094464908024617
:1008A0000296224321D062460A431ED06200570DB1
:1008B0004A000E032303550D012402462C4924054A
:1008C000781B1B0B360B40182343264361460090D0
:1008D0001C46501AB44103D30098401C009002E01B
:1008E000921800985B41002803DA0020014605B009
:1008F000F0BD0020012109050746864611E0644647
:100900001D46141BB54106D36546521BB3417446C0
:1009100007430C43A646CD074008490828439218D0
:100920005B4105460D43EAD11046184313D060469B
:10093000194650407140084306D06046101AB34132
:1009400006D20122002306E000220123DB0702E099
:100950000122D2435310009874460105381C6141AE
:10096000029C039D0019694100F03EFABFE70000B8
:10097000FD03000070B54B005B0803430BD04B0038
:100980005C0D002633466542B341D417AD1AA3412E
:1009900002DB0020014670BD12053018514170BDC8
:1009A000C217C10F504010B54018CA079623002146
:1009B00000F0C2F910BD10B500229623114600F0D8
:1009C000BBF910BD0EB5C217C10F5040CA07401881
:1009D0000021054B0293019200910A460B4600F05C
:1009E00010FA03B000BD0000330400000EB5054945
:1009F0000291002100910A460B46019100F001FA94
:100A000003B000BD33040000C20F410040020123C7
:100A1000400ADB05D207090EC0187F2901DA002041
:100A20007047962903DC9623591AC84001E096398D
:100A30008840002AF4D04042704741004002012221
:100A4000400AD205090E80187F2901DA002070477C
:100A5000962903DC9622511AC8407047963988407F
:100A60007047000070B5CD0F4A0009030123090B40
:100A70001B0519430B4BED070024520D9A4201DA76
:100A8000002070BD074B34339A4203DC9A1A00F001
:100A9000A7F802E00449511888402C43F1D04042A5
:100AA00070BD0000FF030000CDFBFFFF4A000903FB
:100AB0000123090B1B051943094B10B5520D9A422E
:100AC00001DA002010BD064B34339A4203DC9A1A37
:100AD00000F086F810BD03495118884010BD000091
:100AE000FF030000CDFBFFFFC20FD207400040080C
:100AF0000BD0C10D0723DB01C91840020905400ACC
:100B00001143C20840071143704700200146704757
:100B100010B5002904DB0124E40740428C41214642
:100B2000002B04DB1C460123DB075242A3418B420E
:100B300000D1824210BD000010B5002904DB012461
:100B4000E40740428C412146002B04DB1C46012374
:100B5000DB075242A341994200D1904210BD0000F0
:100B6000CB0FDB07490010B5490802460A4307D0FE
:100B70000A0D07240903E401090B121B002A01DCFA
:100B8000002010BDC900440F0C43C100E018D2057D
:100B9000801800F0C9F810BD0122D207002800DB40
:100BA000101A002900DB511A814270470122D20736
:100BB000002800DB101A002900DB511A8842704718
:100BC00010B5202A04DB0146203A9140002010BDD8
:100BD000914020239C1A0346E3401943904010BDE6
:100BE00010B5202A04DB0846203AD040002110BD71
:100BF0000B46D340D0402024A21A91400843194606
:100C000010BD10B5202A06DBCB170846203A10414C
:100C1000C1170B4306E00B461341D0402024A21A13
:100C200091400843194610BD3A2800D2303820239D
:100C300002469A43412A01D310463738884201D3ED
:100C40000020C0437047000002681378511801600B
:100C50001846704710B5D1600449516104491162CA
:100C600000211161114600F0EDF910BD490C00089A
:100C7000311000084268002A08D001680B78491C2E
:100C8000002B03D0521E06C0184670470121C160D8
:100C9000881E70474268002A0BD0C3680168002B89
:100CA00007D183688B4204D0491E521C06C0002025
:100CB00070470020C0437047F7B5009C0F460026E0
:100CC0002578641C002D05D000F0AEF90068405D69
:100CD000C007F5D12B2D02D02D2D18D0641E39461A
:100CE0002046029A00F04AFB002F04D03968A14246
:100CF00001D1009939607105022400290BDA4042C4
:100D0000002803DD0EF0BAFC0460A007FEBD012040
:100D100080020643E3E70028F8DA0EF0AFFC046037
:100D20000048FEBDFFFFFF7F002904DA401C490098
:100D300001D140084000704770B40024050C05D173
:100D40001024000402D1002921D01124050E01D164
:100D500000020834050F01D10001241D850F01D1C7
:100D60008000A41C002801DB4000641C002908D07E
:100D700020252E1B0D46F540A14000D0012129431E
:100D8000084301061B1B000ADB1D02D5002070BCB6
:100D90007047DB05181880180029F8DA401C490054
:100DA000F5D170BC40084000704710B541000DD02F
:100DB0004100090E962909DC7E290ADC07DB410285
:100DC00005D0C00F7F21C007C905401810BD002005
:100DD00010BD9622541A20210A1B01469140E04082
:100DE000FFF7A2FFA04010BD10B5002B08DA0024C9
:100DF000401C614192185B411A4301D140084000F8
:100E000010BDF0B51FB482B005460C0003D00846F3
:100E10000EF0C0FB02E00EF0BDFB20300246009059
:100E200021462846FFF7CCFE049B059A04460F4650
:100E300018431143084314D0184610431BD00098A0
:100E400040210A1A18460599FFF7CAFE05460E46C4
:100E5000009A05990498FFF7B3FE084305D00120D6
:100E600004E02046394607B0F0BD0020C117054315
:100E70000E432C43374300990E986305401A7905B9
:100E8000E40A00220C43FD0A0A3002D50020014684
:100E9000E9E70105101969410C9C0D9D0019694194
:100EA000FFF7A2FFDFE7FEB500231A461B1A8A41AF
:100EB00003DB0020014603B0F0BD4A000D03012111
:100EC0002D0B0905520D0D43D10702D100186D41BC
:100ED000521E5110FF31FF310131002704463E46BA
:100EE0003846009701910246012100200905FFF7CD
:100EF00077FEC3197141F818324684468E464A413E
:100F000061462846611A904104D36046241A9541EF
:100F100076461F46241900986D41401C00903428E5
:100F2000E1DDF91930467041091BA84103D20022C6
:100F3000D243134601E00022134601980105381CF4
:100F40007141FFF751FFB6E7F8B505464800400884
:100F50000C46284304D06000184A400D904201DD41
:100F60002846F8BD15493539884210DC88420BDB2C
:100F7000290D200308432903014305D0E00F104940
:100F8000C00741180020F8BD00200146F8BD161A20
:100F90004020821B28462146FFF712FE074600919B
:100FA000284621463246FFF71BFE3A46009BFFF7D4
:100FB0001BFF3246FFF704FEF8BD000033040000BB
:100FC0000000F03F4A0009030123090B1B051943E8
:100FD0000A4B10B5520D9A4202DA0020014610BDAC
:100FE000064B34339A4203DC9A1AFFF7F9FD10BD21
:100FF000034BD218FFF7E4FD10BD0000FF03000013
:10100000CDFBFFFF064C0125064E05E0E36807CC4B
:101010002B430C3C98471034B442F7D3FFF754F8F5
:10102000786A0108986A0108004870475458010816
:1010300010B50446FFF7F8FF0068005DC007C00F59
:1010400010BD0000F3B58DB000200A9001200B9078
:10105000002608460C300C46099062690121099867
:101060009047051E2ED0252D2DD0216A88470028B7
:1010700018D06269012109989047216A88470028A1
:10108000F7D1411E62690998904700E0761CA1697A
:101090000D988847216A88470028F7D1E1690D98A3
:1010A0008847DAE7A1690D9888470746A84201D129
:1010B000761CD2E7E1690D9888477F1C02D10A9817
:1010C000002877D049E1002762693D4639460998F2
:1010D00090472A280CD1626901210998904701257F
:1010E00006E00A214F433F18303FEBD41020054360
:1010F0006269012109989047014630390A2903D2D3
:101100009B498F42DEDCECE7E90600D4994F6C285E
:101110000AD04C2810D0682824D06A282ED07428F1
:101120000CD07A280AD00DE0626901210998904715
:101130006C2823D004211CE0202005436269012192
:1011400009989047A760656065284FD026DC58282D
:1011500039D01ADC452849D012DC252834D0412862
:10116000B0D143E06269012109989047682802D014
:1011700008210D43E6E70120C002DEE70220DCE79C
:10118000462833D047282CD130E05B2870D0612826
:101190002CD063286CD0642823D161E06F284FD015
:1011A00009DC662822D0672820D0692826D06E283E
:1011B00017D12EE0CDE070284DD073286FD0752860
:1011C0004ED078280DD154E0A1690D988847054686
:1011D000252800D16CE7E1690D9888476D1C00D186
:1011E0006DE7BAE00A224CE00A2252E001202346D1
:1011F0006A46C0430D99C046C046A3E02846402138
:1012000008436060A807234601D5002239E0002288
:101210003FE0E80700D020E72068011D216000685A
:10122000290501D5067018E7290701D5068014E7BE
:10123000A90703D5F117066041600EE706600CE7C9
:101240002846402108436060A807234601D50822AC
:1012500017E008221DE0484928460840606016E073
:101260002846402108436060A8072346BCD5B9E75B
:1012700015E02846402108436060A80707D52346AB
:1012800010220120C0430D99C046C0465AE02346B3
:1012900010220120C0430D99FFF748F852E00021C9
:1012A0000C910B460091632802D05B2807D043E0E5
:1012B000E80601D40120A060012000903CE06269B2
:1012C0000121099890475E2805D101200C90014624
:1012D0006269099890472169002906D10B4601AA45
:1012E0008F00491CD3510829FADB002835D0216929
:1012F00000290ED1C117C90E09184A11930001AA7D
:101300009A1849094901411A01201368884003438A
:10131000136062690121099890475D28E5D10C9816
:10132000002808D0002001AB81005A58401CD2434D
:101330005A500828F8DB01AB01202246C0430D9922
:10134000C046C04600280ADA401C06D10B98002887
:1013500003D00020C0430FB0F0BD0A98FBE7E907B7
:1013600002D10A99491C0A91361800200B9074E6A4
:10137000CCCCCC0CFFFFFF7FF1F7FFFFF7B582B0BD
:10138000029C00272078641C15460197302802D063
:10139000002D15D015E020780127641C782804D092
:1013A000582802D0002D09D00BE0002D01D0102DBF
:1013B00007D1002710252078641C02E0082500E0F2
:1013C0000A250026009610E00099012769430818B5
:1013D000020C294680B2714300908E183804864270
:1013E00001D3012001902078641C2946FFF71CFCE2
:1013F0000028E9DA0398002805D0002F01D0641EE8
:1014000000E0029C04600198002806D00EF036F936
:1014100002210160C81E05B0F0BD009930040843E8
:10142000F9E770B58C180578401C6B075B0F01D18C
:101430000378401C2A1106D10278401C03E006788C
:101440000E70401C491C5B1EF9D12B0705D40023EC
:10145000521E0DD40B70491CFAE70378401CCB1ABE
:10146000921C03E01D780D70491C5B1C521EF9D5BF
:10147000A142D8D3002070BD38B5044606480549BE
:101480000068FEF735FE604300E0401E0090002833
:10149000FBD138BD40420F0080010020F8B5044662
:1014A000006881688907890F012902D10168C9078D
:1014B00022D18168114A10261140012500290ED140
:1014C0008168294381600120FFF7D6FF03F09CFA71
:1014D00007460CE003F098FAC01B0A2807D9A06D54
:1014E0003043A065E06D2843E0650120F8BD206829
:1014F0000068C043C007EDD10020F8BD1700008090
:10150000F0B589B00C46074610220021684611F05C
:1015100075FE6946224608460EF06FFE6846007862
:1015200087260106684600290FDA00214318425C2D
:101530005B785200DB091A434254491C0F29F5DB42
:10154000C17B0246490071400DE000214318425C16
:101550005B785200DB091A434254491C0F29F5DB22
:10156000C17B02464900D173E21DF932516910294D
:1015700012D0017809061BD500214518435C6D780F
:101580005B00ED092B434354491C0F29F5DBC17B5C
:1015900003464900714019E000216218FF32013210
:1015A0005378455C491C6B4053701029F5DB26E0ED
:1015B00000214518435C6D785B00ED092B434354D3
:1015C000491C0F29F5DBC17B03464900D973E11D96
:1015D00055698023FA316B54002500E05D5453694E
:1015E0005B1C5361102BF9D300216218FF320132CA
:1015F0005378455C491C6B4053701029F5DB002182
:1016000062181046FF32E0300132437C5278491CA8
:10161000534043741029F3DB21461022F13104A812
:1016200011F0D4FD2246394604A80EF0E6FD102242
:101630000021684611F0E2FD09B0F0BD10B5044686
:1016400010220021F13011F0D9FDFF2000211530CA
:101650000151F022204611F0D1FD10BD0B4610B50E
:101660000246102118460EF0F3FD10BDF0B50446F9
:10167000FF308BB00F4601300890E11D4069FA3110
:101680000091103915460791002843D010210E1AF9
:10169000AE4200D316460099B2B24018394611F056
:1016A00095FD0898089940698019486110283AD337
:1016B000B54238D0002162181046FF32E0300132C6
:1016C000437C5278491C534043741029F3DB07993B
:1016D000224608460EF091FDBF19AD1B1AE000200E
:1016E0002118E0314A7C3B5C401C5A404A74102867
:1016F000F6DB102202A8079911F068FD02A9224624
:1017000008460EF07AFD102202A9079811F05EFD3E
:10171000103D1037102DE2D8AAB23946009811F0CA
:1017200055FD089845610BB0F0BD0000FFB5FF49BD
:10173000A1B0CA7DC81DF9302D9E2E9D012A12D15F
:101740000022CA7503672A9941672B9981672199FD
:101750004166229981662399C1662C99C167014629
:1017600080310E604D60F24C1846216FFEF790FEFE
:101770000021C943FEF760FF0746616F2A98FEF714
:1017800087FE0021C943FEF757FF2A90A16F2B98CF
:10179000FEF77EFE0021C943FEF74EFF2B90616EDF
:1017A00000912198FEF774FE0021C943FEF744FF23
:1017B0000099FEF76DFE0021C943FEF73DFF009939
:1017C000FEF766FE0021C943FEF736FF2190E16F68
:1017D00000912C98FEF75CFE0021C943FEF72CFF18
:1017E0000099FEF755FE0021C943FEF725FF009939
:1017F000FEF74EFE0021C943FEF71EFF2C9027671F
:101800002A9860672B98A067219860662298A06646
:101810002398E0662C98E067204680300660803C84
:101820004560A16C03910846FEF78BFE1D90E16CAC
:1018300002910398FEF785FE0E90216D01910398A9
:10184000FEF77FFE0D90616D03980C46FEF779FE62
:101850000C9002990846FEF774FE0B9001990298CD
:10186000FEF76FFE0A9021460298FEF76AFE019984
:1018700009900846FEF765FE089021460198FEF79C
:1018800060FE214607900846FEF75BFE2B99069006
:101890000846FEF756FE2A9900900846FEF751FECC
:1018A000044639460846FEF74CFE2146FEF7F0FD99
:1018B0000099FEF7EDFD10F0AFFF044601463846F3
:1018C000FEF73FFE249021462A98FEF73AFE2A9022
:1018D00021462B98FEF735FE29462B900846FEF749
:1018E00030FE074631460846FEF72BFE2C9904468B
:1018F0000846FEF726FE2146FEF7CAFD3946FEF7EA
:10190000C7FD10F089FF044601462C98FEF719FE2A
:101910002C9021463046FEF714FE2D902146284695
:10192000FEF70FFE2E900D990998FEF7B1FD0446C3
:101930001F9001212E98FEF77FFE1C9021461B90E0
:10194000FEF7FFFDFFF7D0F819911A900C990A984D
:10195000FEF7EFFD04461E9001212D98FEF76CFE68
:10196000189021461790FEF7ECFDFFF7BDF80646EC
:1019700015910698FFF7B8F805460C4605910898AA
:10198000FFF7B2F800226B4B03910290FEF70AFFBB
:1019900023462A46FEF700FF04460F4601910090B9
:1019A00001212C98FEF748FE12901190FFF79CF849
:1019B00022463B46FEF7FEFE3246159BFEF748FEEA
:1019C000199B1A9AFEF744FEFFF7CAF813900E9976
:1019D0000798FEF7AEFD01461B98FEF7B2FDFFF734
:1019E00083F804460E46059F0B98FFF77DF800220A
:1019F000504BFEF7D7FE2A463B4605910490FEF772
:101A0000CBFE05460F461798FFF76EF82A463B4671
:101A1000FEF7D0FE07460D460C990A98FEF738FDF2
:101A200001461198FEF78DFDFFF75EF83A462B460A
:101A3000FEF70EFE22463346FEF70AFEFFF790F849
:101A40000646039B029A05990498FEF7A5FE0546F3
:101A50000C4602911C98FFF747F823462A46FEF7EA
:101A6000A9FE0C460A900E990798FEF711FD014653
:101A70000E901898FEF765FD07460D990998FEF738
:101A800058FD01460D901298FEF75BFD3946FEF7B2
:101A9000FFFCFFF729F823460A9AFEF7D9FDFFF766
:101AA0005FF8044631460846FEF74BFD139906469B
:101AB0000846FEF746FD3146FEF7EAFCFFF714F84C
:101AC00012F0CEFAFFF74CF8074601210D98FEF709
:101AD000B3FD099001210E98FEF7AEFD07900B991A
:101AE0001D98FEF726FD0899FEF723FD0699FEF7DF
:101AF000CFFC06460D98049001212046FEF79CFD80
:101B00000B900499FEF71DFDFEF7EEFF0490009880
:101B10000C46089001213846FEF78EFD0C90FEF72A
:101B2000E3FF019B089AFEF745FE05E094010020C3
:101B3000940200200000E03F2346049AFEF788FD4F
:101B4000FFF70EF807460E990B98FEF7FAFC0446CD
:101B50001E990C98FEF7F5FC2146FEF799FC0299B8
:101B6000044600950D460B98FEF7BEFF2B46009AE3
:101B7000FEF720FE054600911F990C98FEF7E1FC48
:101B8000FEF7B2FF2A46009BFEF762FDFEF7E8FF74
:101B9000054621462E98FEF7D4FC019029462D9843
:101BA000FEF7CFFC0199FEF7C4FC029007992B9831
:101BB000FEF7C7FC009031462A98FEF7C2FC009958
:101BC000FEF7B7FC0299FEF763FC049029462C98B7
:101BD000FEF7B7FC054639462E98FEF7B2FC2946BB
:101BE000FEF7A7FC054631462498FEF7AAFC0646F8
:101BF00009992B98FEF7A5FC3146FEF79AFC294679
:101C0000FEF746FC089039462D98FEF79AFC0546EB
:101C100021462C98FEF795FC2946FEF78AFC0446DF
:101C200009992A98FEF78DFC054607992498FEF736
:101C300088FC2946FEF77DFC2146FEF729FCFE4F75
:101C4000059039460498FEF77CFCFC4E3146FEF7C1
:101C500078FCFB4CA16DFEF71BFC0546A0653946E0
:101C60000898FEF76EFC3146FEF76BFCE16DFEF75F
:101C70000FFCE065009039460598FEF762FC31469E
:101C8000FEF75FFC216EFEF703FCEE4F0646206672
:101C900039460498FEF755FC2199FEF7F9FB2946D1
:101CA000FEF7F6FB054639460898FEF74AFC2299EE
:101CB000FEF7EEFB0099FEF7EBFB22903946059804
:101CC000FEF73FFC2399FEF7E3FB3146FEF7E0FB0E
:101CD0002390616D03910991FEF733FC216D074656
:101CE000029105912298FEF72CFC06460120E16C3A
:101CF000C007684001910891FEF723FC3146FEF7CA
:101D000018FC3946FEF715FC0021C943FEF794FC88
:101D1000E06607900C9009992298FEF712FC07469E
:101D200005992398FEF70DFCA16C06460091284604
:101D30000691FEF706FC3146FEF7AAFB3946FEF790
:101D4000F8FB0021C943FEF777FC206704900646A4
:101D500028460999FEF7F5FB0B9008992398FEF7A2
:101D6000F0FB074606992298FEF7EBFB3946FEF793
:101D7000E0FB0B99FEF78CFB0021C943FEF75CFCEE
:101D800060670A900E9028460599FEF7DAFB0B90E3
:101D900008992298FEF7D5FB074606992398FEF787
:101DA000D0FB3946FEF774FB0B99FEF7C2FB00210E
:101DB000C943FEF741FCA067A3490B90FEF7C1FBA6
:101DC0000999FEF765FB074617909F482399FEF790
:101DD000B0FB39461090FEF7B4FB09909A490E9873
:101DE000FEF7AFFB0599FEF753FB189007469648A0
:101DF0002299FEF79EFB39461590FEF7A2FB074697
:101E000091493046FEF79DFB0899FEF741FB0646D7
:101E10001A908D492846FEF790FB31461190FEF747
:101E200090FB064688490C98FEF78BFB0699FEF757
:101E30002FFB85491B90FEF784FB3146FEF728FBFC
:101E40003946FEF725FB0999FEF722FB0021C9431D
:101E5000FEF7F2FBE067199017991598FEF771FBF2
:101E600005907949189C2398FEF712FB0C902146A7
:101E70001490FEF766FB074673491A98FEF761FB5C
:101E80000646714928461B9CFEF702FB0D90214631
:101E90000890FEF756FB3146FEF7FAFA3946FEF790
:101EA000F7FA0599FEF7F4FA0021C943FEF7C4FBDF
:101EB000634C0746803420600F9017990898FEF70E
:101EC00040FB139060491898FEF73BFB09901A9964
:101ED0001098FEF736FB16905B491B9E2298FEF782
:101EE000D7FA059031461290FEF72BFB1699FEF7B4
:101EF000CFFA0999FEF7CCFA1399FEF7C9FA002137
:101F0000C943FEF799FB606006460E904E4917984C
:101F1000FEF717FB099018991198FEF712FB139022
:101F20001A991298FEF70DFB12901B991498FEF760
:101F300008FB1299FEF7ACFA1399FEF7A9FA099972
:101F4000FEF7A6FA0021C943FEF776FBA0603E49E2
:101F50000990FEF7F6FA0399FEF79AFA01461390F4
:101F60001098FEF7EEFA129037493046FEF7E9FA7C
:101F70000299FEF78DFA014614901598FEF7E1FAE2
:101F8000064631493846FEF7DCFA0199FEF780FA39
:101F9000014617901198FEF7D4FA07462A49199876
:101FA000FEF7CFFA0099FEF773FA27491690FEF76D
:101FB000C8FA3946FEF76CFA3146FEF769FA12990B
:101FC000FEF766FA0021C943FEF736FBE060189081
:101FD00013991598FEF7B5FA074614990C98FEF771
:101FE000B0FA069018491798FEF7ABFA064616990C
:101FF0000D98FEF7A6FA3146FEF74AFA0699FEF763
:1020000047FA3946FEF744FA0021C943FEF714FBAC
:1020100020610890069013990D98FEF792FA0D90A2
:1020200009491498FEF78DFA074617991098FEF79C
:1020300088FA0646169909E00AD7A33C52491D3C86
:10204000140200200000204252499D3B0598FEF7F3
:1020500078FA3146FEF71CFA3946FEF719FA0D995F
:10206000FEF716FA0021C943FEF7E6FA606107465B
:102070000D90FE491398FEF764FA10901499119888
:10208000FEF75FFA119017990598FEF75AFA06467F
:1020900016990C98FEF755FA3146FEF7F9F91199A1
:1020A000FEF7F6F91099FEF7F3F90021C943FEF7A0
:1020B000C3FAA061EE491090FEF743FA0399FEF7C8
:1020C000E7F906461790EA482399FEF732FA3146B7
:1020D0001C90FEF736FA0C90E5493846FEF731FAC7
:1020E0000299FEF7D5F906461690E1482299FEF7C7
:1020F00020FA31461290FEF724FA0746DC4906988A
:10210000FEF71FFA0199FEF7C3F906461590D84964
:102110002846FEF712FA31461B90FEF712FA0646E1
:10212000D3491898FEF70DFA0099FEF7B1F9D04996
:102130001490FEF706FA3146FEF7AAF93946FEF783
:10214000A7F90C99FEF7A4F90021C943FEF774FA28
:10215000E061059017991298FEF7F3F90690C449CB
:10216000169E2398FEF794F931461A90FEF7E9F986
:102170000C90BF491598FEF7E4F90746BC4928467C
:10218000149EFEF785F905463146FEF7DAF9394621
:10219000FEF77EF90C99FEF77BF90699FEF778F9C0
:1021A0000021C943FEF748FA206213902846179988
:1021B000FEF7C7F91290AE491698FEF7C2F9064627
:1021C00015991C98FEF7BDF90746A949149D229858
:1021D000FEF75EF929461D90FEF7B3F93946FEF782
:1021E00057F93146FEF754F91299FEF751F90021DB
:1021F000C943FEF721FA606206909D491798FEF7E1
:10220000A0F9074616991B98FEF79BF90546159904
:102210001D98FEF796F9064614991A98FEF791F95B
:102220003146FEF735F92946FEF732F93946FEF711
:102230002FF90021C943FEF7FFF9A0620C9001219C
:102240001898FEF7F9F9044601211998FEF7F4F9F8
:102250000799FEF71DF92146FEF71AF90599FEF7D1
:1022600017F9FEF741FC0022824BFEF7A3FA044661
:102270000E460098FEF738FC33462246FEF7E8F992
:10228000FEF76EFC7C490746886401210898FEF73A
:10229000D3F9064601210F98FEF7CEF9764C049942
:1022A000FEF7F6F83146FEF7F3F81399FEF7F0F86B
:1022B000FEF71AFC00226F4BFEF77CFA05460E462D
:1022C0000198FEF711FC2A463346FEF7C1F9FEF7E6
:1022D00047FC0646E06401210D98FEF7ADF905467E
:1022E00001210E98FEF7A8F90A99FEF7D1F82946C0
:1022F000FEF7CEF80699FEF7CBF8FEF7F5FB0022C5
:102300005C4BFEF757FA054601910298FEF7ECFB8D
:102310002A46019BFEF79CF9FEF722FC0546206544
:1023200001211098FEF788F9009001210998FEF725
:1023300083F90B99FEF7ACF80099FEF7A9F80C9910
:10234000FEF7A6F8FEF7D0FB00224A4BFEF732FA62
:10235000009001910398FEF7C7FB019B009AFEF7DE
:1023600077F9FEF7FDFB01466065FEF7EAF82946BE
:1023700001900846FEF7E5F8054631460846FEF7A7
:10238000E0F8064639460846FEF7DBF83146FEF728
:102390007FF82946FEF77CF80199FEF779F810F0EE
:1023A0003BFA07460146A06CFEF7CBF80646A06450
:1023B0003946E06CFEF7C5F8E06403903946206DBD
:1023C000FEF7BFF8054620653946606DFEF7B9F89F
:1023D0000746606501213046FEF72EF92946FEF7D3
:1023E000B0F803250646AD0729460398FEF7A9F87D
:1023F0003946FEF7A6F83146FEF74AF8FEF774FBB9
:102400000DF0A4FF1D4A1E4BFEF7D4F9FEF7A8FB02
:1024100030990860206D01210646FEF70DF931461E
:102420000490FEF78EF80646E06C29460746FEF754
:1024300088F83946FEF785F83146FEF77AF87F21AD
:10244000C905FEF725F8FEF74FFB0E4605460121AC
:10245000A06CFEF7F1F83946FEF773F807460498CA
:10246000616DFEF76EF839460CE0000052499D3B65
:1024700052491D3CE3365A3F1402002066666666E8
:1024800066A64CC0FEF704F8FEF72EFB2A4633463C
:102490000FF0D6FB264E254A3346FEF78BF9FEF7A2
:1024A0005FFB2F990860616D00910846FEF749F8BF
:1024B0000590216D04910846FEF743F8E16C07464C
:1024C00008460191FEF73DF8A16C054608460291C9
:1024D000FEF737F82946FDF7DBFF3946FEF729F806
:1024E0000599FEF726F8FEF7FFFA05460C46009917
:1024F0000298FEF726F8074604990198FEF721F89E
:102500003946FDF7C5FF0121FEF796F8FEF7ECFA14
:102510002A4623460FF094FB044A3346FEF74AF955
:10252000FEF71EFB3199086025B0F0BD6666666651
:1025300066A64C40F7B523498022097C214B511AED
:10254000CDB2D97B1B7C8026F31A0A46DEB2871EE9
:10255000491C0124C9B2761E3B000DF04AF8090659
:102560000C060C120C06062B3000164BAA4224D285
:10257000154CA05403E0134BB24215DB1DE0D97398
:102580000DE0104EAD1EAA4217DA0F4B9854019879
:102590005854491CC8B202991954401CF0730024C5
:1025A00008480121817308E0074CA0540198605449
:1025B000491CE4E7034BAA42F6D32046FEBD0220A5
:1025C000FEBD0000940400206A1A002010B586B0F9
:1025D00014216846FDF73CFE0D48C26A01210A43FA
:1025E000C262C06A052408400590042000900020C3
:1025F000029003200191240703906946204602F0CF
:1026000031F901220421204602F0F7F906B010BD8D
:102610000010024000B50B4887B0C26A01210A438E
:10262000C262C06A01910840059019200002009022
:1026300003200390029105206946000702F012F979
:1026400007B000BD0010024000B587B0FFF7BEFF25
:1026500000F0ACFE0A48C26A01210A43C262C06AA5
:10266000019108400590192000020090032003907A
:10267000029105206946000702F0F4F807B000BD9A
:102680000010024070B505260546360700220421D9
:10269000304602F0B2F9012004F026F9104C2080F7
:1026A00001220421304602F0A8F904F0DDF9208867
:1026B0000C49098848430C49FDF730FD608060886B
:1026C000392148432F21FDF713FDA080608839216F
:1026D00048432F21FDF70CFDFEF76DF9E86070BD52
:1026E0008801002048030020FF0F00000178044803
:1026F000024A4368D154012101707047E31500205C
:102700009C03002010B5034812F010FA0249002083
:10271000087010BDED2600089C03002010B512487B
:10272000017801290ED100210170104B42689C5C98
:10273000012C08D00D2C09D00A2C07D07F2A0DD0EF
:10274000521C426010BD4160082009E0002AF9D007
:1027500099544160054810F047FF10BD41600620C4
:102760000FF040FE10BD00009C030020E315002088
:10277000F8B506460F460068FEF7B6F90446002095
:102780000D46385EFEF71EF90022054BFEF712F8E3
:1027900022462B46FDF75CFFFEF7E2F93060F8BDFC
:1027A000008076403EB50D4C6946A27A0A70227FC1
:1027B0008A70C870E06B0CF03BFA0190606C02907C
:1027C000E07F69464870207E08F038FD218D606CFE
:1027D0004143081AA16E4018A0663EBD9404002033
:1027E000FFB5044689B00020039008900690218927
:1027F0001646002915D00190626904922069002ACA
:1028000004D000290FD00A4692B20392002900D0CA
:102810000E46E168884215D3039A61688018081A49
:1028200011E00220E7E722686568135C471CAF42AD
:1028300002D3451B6D1C00E03D46525D1202921C06
:102840009A18E1E700200199751807950C994D43F6
:10285000854201D2002102E00799FDF749FCC8B288
:102860000199884208D9217FCA0700D106980690AD
:10287000880701D5019800E00698002E6AD00499D7
:10288000491908186168884264D8002798E00398BD
:1028900008186168884200D3401A20612189002904
:1028A00011D121680E546168401C814200D8401A41
:1028B0002268310A11546168401C814200D8401AD4
:1028C0006169891C616161680D1AB54200D33546A2
:1028D000B5420DD0B54202D2217F002908D0002D8B
:1028E0006AD0217FCA0730D02189002913D019E08E
:1028F00039460A9A71438918226810182A46FDF74A
:102900008EFC60694019606107990895002089B2C2
:10291000751B039140E02368FF22811E5A542168F1
:10292000401E0A54606940196061002008902189A6
:10293000354600292AD1206805702168280A487088
:1029400061690220891C616120E089071ED5218907
:10295000002902D000200DB0F0BD2168821E8D54E8
:102960002268290A431ED15439460A9A71438918AC
:10297000226810182A46FDF752FC60694019606110
:102980000895A069751B401CA061D4E701996918DE
:1029900089B2039100212161002D0DD0089A0A9976
:1029A0003B46891822687343101859182A46FDF7C8
:1029B00036FC606940196061A069401C7F1CA06101
:1029C0000C982169874200D261E701980818616874
:1029D000884200D3401A21684018BCE710B5029C19
:1029E00001600021C1600161416142608161038138
:1029F0000477A00703D5002B01D0481E10BD00208E
:102A000010BD0000F0B503890022002B09D000237F
:102A100000240C804469002C58D00289002A02D07E
:102A20000DE00223F4E7C26804684668A55C571C01
:102A3000B74200D3921B521CA25C1202AA1894B295
:102A40000C80027FD50729D0920727D4204A9442D0
:102A500002D10289002A0AD0C468026994421DD9B1
:102A60000289002A1AD045682C1B944216D2446869
:102A7000C2684569A21AAA1A42610022C26002898C
:102A8000002A0AD10268012C157802D86442641C1D
:102A900000E00124125D1202AA180A80C568446889
:102AA000EA18A24200D3121B06680F8892194669E1
:102AB000FF18F61B466106D009886918C918A1429B
:102AC00000D3091BC1608169491E81611046F0BDB8
:102AD000FFFF0000F0B503890022002B0AD0002779
:102AE00000230B804369002B42D00389C268002B6E
:102AF00002D00DE00227F3E705684468531CAE5C82
:102B0000A342134600D31B1B5B1CEB5C1B02F31898
:102B10009CB20C80037FDD0723D09B0721D4154B8B
:102B20009C4202D10389002B0AD0C46803699C42ED
:102B300017D90389002B14D045682C1B9C4210D256
:102B400000221B041B0C0BD143680468012B02D824
:102B50005B425B1C00E00123E35C24781B021B1931
:102B60000B80D1194268914200D3891A00680A1873
:102B70001046F0BDFFFF0000FFB5002085B00090BB
:102B80000546064601900024770007980121C05BA6
:102B9000A14008422FD028190C2203905043089AD4
:102BA0001258002A27D0059A002A01D1490722D0BD
:102BB00008994118082002910856021100070117D0
:102BC000069840B208F061FD002814D00298407ABF
:102BD00001010E980818C068002804D00198401C14
:102BE000C0B2019007E0009A0F99039888540098AA
:102BF000401CC0B20090641CE4B2102CC5D3103548
:102C0000761CEDB2F6B2102DBDD310990198087064
:102C1000009809B0F0BD000030B50A4C03680A4DB9
:102C2000A34205D90B68AB4202DD13885B1C1380FD
:102C30000068A84205DD0868A04202D91088401E3D
:102C4000108030BD00002AC300002A4330B587B091
:102C500014216846FDF7FCFA032001900020029041
:102C600003204003104C0090E06A01210843E06219
:102C7000E06A0840059005206946000701F0F2FD72
:102C8000E06A40084000E062606B0125AD05284322
:102C9000606301F0BBFA01F0C9FA01F0BFFA606BA2
:102CA000A843606307B030BD0010024010B511F0BA
:102CB000DFFE10BD10B5046863608368102B0368E5
:102CC00003D099600068C26010BD9A600068C1605E
:102CD00010BD10B503F070FF10BD000010B507481F
:102CE00001224179008A090401430448143001603B
:102CF0000146034800F006F810BD0000A4030020C0
:102D000054000808F7B5174600260546EFF310846F
:102D100072B601F003FD0DE00198B100425829465A
:102D2000022001F0D1FC00280BD084F3108806A00B
:102D30000CF07EF8BE42EFDB01F0BCFC84F310889F
:102D4000FEBD2D1D761CF5E76572726F7220696EEF
:102D500020454550524F4D20577269746520657269
:102D6000726F720D0000000010B5012001F06EFDC1
:102D7000022001F06BFD10BD10B5042001F066FDCE
:102D8000082001F063FD10BDF8B5102001F05EFDD4
:102D9000202001F05BFD402001F058FD802001F073
:102DA00055FDFF20013001F051FD0120400201F0EE
:102DB0004DFD0120800201F049FD0120C00201F01B
:102DC00045FD1C4C60691C4EC0041C4F01250028A9
:102DD00018DA3078002810D01948006800280CD084
:102DE00018480078C00708D117480078012804D196
:102DF00016480068002800D17D7001200003606142
:102E000003F002FE0120400301F020FD6069400450
:102E10000AD53078002800D03D700D4805600120AB
:102E20008003606103F0F0FD0120C00301F00EFD9E
:102E3000F8BD000000040140A20100204C03002066
:102E400074030020D40400209E010020CC01002047
:102E50005402002070B5124886B0C16A0224214392
:102E6000C162C06A104E2040059060030D4D009075
:102E7000019502946946304601F0F4FCE0020090AE
:102E8000694601950294304601F0ECFC00220321D2
:102E9000072001F033FE072001F026FE06B070BDCA
:102EA000001002400000111000040050FEE7000076
:102EB00010B5084900224A6107494B684C15234365
:102EC0004B604B68082423434B60C009C00102607B
:102ED00010BD0000C81000200020024010B5214A9B
:102EE00000219069C305204804D541690223194394
:102EF0004161911593699B0505D5436901242343DD
:102F000043616302194393695B0505D5436908244E
:102F100023434361E301194393691B0505D54369C5
:102F20000424234343616302194393699B0405D539
:102F300043691024234343616302194393699B034C
:102F400004D5446920231C43446119439369DB037E
:102F500005D54369402423434361A00201439161A5
:102F600010BD000000200240C810002070B50546CA
:102F700001F04AFD0646184C0AE0681C08D0002DF6
:102F800004D001F041FD801BA84201D9032070BD8F
:102F9000A069C007F1D1A069800701D50220A06116
:102FA000A069C00511D4A06980050ED4A0694005B0
:102FB0000BD4A069000508D4A069800405D4A069D9
:102FC000800302D4A069C00303D5FFF787FF012067
:102FD00070BD002070BD00000020024010B5044606
:102FE00001F012FC0849002011C1012008600749C6
:102FF000054801F0A5FB002803D005A00BF018FF41
:10300000FBE701F0D9FB10BD4C05002000000020BB
:103010006572726F7220696E204572617365206FF0
:103020007065726174696F6E0A0D0000F8B516461E
:103030000F460446002501F0E7FB0DE0A8003A58D2
:103040002146022001F0C2FB002803D005A00BF0AE
:10305000EFFEFBE7241D6D1CB542EFDB01F0ACFB7E
:10306000F8BD00006572726F7220696E2057726938
:103070007465206F7065726174696F6E0A0D00006F
:1030800070B50D46044601F0BFFB21462A460220DA
:1030900001F09CFB002803D003A00BF0C9FEFBE766
:1030A00001F08AFB70BD00006572726F7220696E5C
:1030B000205772697465206F7065726174696F6EF4
:1030C0000A0D000001680248416040687047000036
:1030D00000000020FFB581B01D4614460E46019841
:1030E000FDF792FC3060FDF75BFC0199FDF725FAD6
:1030F000164F3946FDF725FAFDF786FC2060FDF7EF
:103100004FFC00903068FDF74BFC0199FDF715FA74
:103110003946FDF716FA0099FDF70BFA3946FDF727
:1031200010FA2860FDF7E0FC0022094BFDF73AFB9E
:10313000084A094BFDF7ECFC06D2002028606168C4
:10314000241D3C2900D1206005B0F0BD0000704274
:1031500000004E407B14AE47E17A843FF8B5002072
:10316000084D044607462602A95D012904D17019BD
:10317000401C00F0AFF9AF55641CE4B2062CF2D34A
:10318000F8BD0000580A002070B586B0FFF7E6FFD2
:103190004F48504C00682646403601286FD104AB9A
:1031A00003AA02A9206AFFF795FF25462035049857
:1031B000FDF79AFC0191009028794E2860D046A135
:1031C00047A0039B029A0BF033FE0028EFD1206A40
:1031D000FDF78AFC0B4629794E2953D03EA10246C1
:1031E00044A00BF025FE0028F1D104AB03AA02A9EC
:1031F000A06AFFF76FFF0498FDF776FC019100903D
:10320000287B452840D03EA13FA0039B029A0BF0AB
:103210000FFE0028EFD1A06AFDF766FC0246287B6E
:103220000B46452832D036A13CA00BF001FE002809
:10323000F1D1E06BFDF758FC3278009202460B4664
:1032400039A00BF0F5FD0028F3D1206BFDF74CFC05
:1032500002460B4639A00BF0EBFD0028F5D1606B60
:10326000FDF742FC02460B4639A00BF0E1FD0028B9
:10327000F5D1211D0EC910290ADA083109E01EE036
:1032800037A19DE736A1AAE737A1BDE736A1CBE775
:10329000103937A00BF0CCFD0028EAD139A06369C2
:1032A000A269E1690BF0C4FD0028F7D1094D603532
:1032B000EA78A97838A00BF0BBFD0028F8D1F078A7
:1032C000022801D0032801D10020A06306B070BD00
:1032D0008403002080070020536F7574680000008D
:1032E00025733A253364202532642725352E32662E
:1032F0002000000025733A20252E36660A0D0000B6
:10330000576573740000000025733A253364202547
:103310003264272530352E326600000025733A20AE
:10332000252E36660A0D2000416C7469747564653B
:103330003A252E3166256320000000005370656534
:10334000643A252E3166206B6D2F68200000000046
:10335000436F757273653A252E31662000000000B8
:103360004E6F7274680000004561737400000000C5
:1033700054696D653A2532643A253032643A253015
:1033800032642000446174653A3230253032642D55
:1033900025642D2564200000536174656C6C69748C
:1033A000653A2532642F2532640A0D0000B50B48BA
:1033B00087B0C26A02210A43C262C06A084005900F
:1033C0002020009001200190002002900320039013
:1033D0006946034801F046FA07B000BD00100240FC
:1033E0000004005070B50E4CA079002801D00020D8
:1033F00070BD0120A07100F039F80A4D00220821AB
:10340000284601F0FAFA00221021284601F0F5FAC8
:1034100001222021284601F0F0FAA07970BD0000B9
:10342000F40000200004005070B50E4886B0C26A57
:1034300002210A43C262C06A0324084005900820A2
:1034400000256A4631C2084E6946304601F00AFA44
:1034500010206A4631C26946304601F003FA06B0D0
:1034600070BD0000001002400004005070B5164806
:1034700086B0C26A02210A43C262C06A01240840BF
:1034800005900820114E032500900194694603958C
:103490000294304601F0E6F910200090019469464C
:1034A00003950294304601F0DDF92020009001944C
:1034B000694603950294304601F0D4F9044900208E
:1034C000887106B070BD000000100240000400507A
:1034D000F4000020F0B5014691B0401C029009783C
:1034E000242909D102AA2A2110F09EFD044602993E
:1034F0000EF05AFF012802D0002011B0F0BD204686
:1035000002AA2C21029410F08FFDFEA10390FCF77B
:10351000BEFE002805D1FD4901200870FC490020AD
:103520000870FCA10398FCF7B2FEFC4C2146103158
:103530000F1F0191083908911031264606911C365B
:10354000091F351D0591002829D0F5A10398FCF726
:103550009EFE00287ED0F4A10398FCF798FE264634
:103560003146603140360791002874D0F0A10398AD
:10357000FCF78DFE0028F8D0EFA10398FCF787FE3A
:10358000002869D0EEA10398FCF781FE00287CD0CA
:10359000EDA10398FCF77BFE0028F8D056E302AAC1
:1035A0002C21029810F040FD0390002812D0014613
:1035B0001422E748FCF782FE00280BD00097221D5A
:1035C000E4A1089B0398FCF793FE1422E0480399BA
:1035D000FCF749FE02AA2C21029810F025FD0028D4
:1035E00004D0007841287DD00020207002AA2C2130
:1035F000029810F019FD002837D009A900910CABF2
:103600000BAAD8A1FCF774FE0998FDF7C9F9FDF7DC
:103610006BFA0022D64BFDF735F90A9003910C980E
:10362000FDF7BEF9FDF760FA0022D24BFDF72AF94B
:10363000074607910B98FDF7B3F9FDF755FA3A469F
:10364000079BFDF705F8039B0A9AFDF701F8FDF7C4
:1036500087FA02E08CE02BE14DE22062FDF744FAAC
:1036600002460B46C4A00BF0E3FB02AA2C210298F1
:1036700010F0DAFC002804D00078532800D04E2047
:10368000287102AA2C21029800E09AE210F0CCFCEA
:10369000002835D010A900910FAB0EAABAA1FCF7F3
:1036A00027FE1098FDF77CF9FDF71EFA0022B04BBB
:1036B000FDF7E8F8009007910F98FDF771F9FDF715
:1036C00013FA0022AB4BFDF7DDF8074603910E9885
:1036D000FDF766F9FDF708FA3A46039BFCF7B8FFD9
:1036E000079B00E042E0009AFCF7B2FFFDF738FAD2
:1036F000A062FDF7F9F902460B469FA00BF098FB7C
:1037000002AA2C21029810F08FFC002804D0007827
:10371000572800D04520287302AA2C21029810F0C7
:1037200083FC00280AD00FF07FFEFDF7DDF9994AEF
:10373000994BFDF73FF8FDF713FA206302AA2C21FD
:10374000029810F071FC002802D00FF06DFE60634B
:1037500002AA2C21029810F067FC002805D00096E0
:103760008EA1069B059AFCF7C3FD6FE201203CE7A2
:1037700002AA2C21029810F057FC0390002812D0C6
:10378000014614227248FCF799FD00280BD00097DF
:10379000221D70A1089B0398FCF7AAFD14226C4817
:1037A0000399FCF760FD02AA2C21029810F03CFC62
:1037B000002804D00078412878D00020207002AA88
:1037C0002C21029810F030FC00282CD009A900917F
:1037D0000CAB0BAA63A1FCF78BFD0998FDF7E0F891
:1037E000FDF782F90022624BFDF74CF807910A9031
:1037F0000C98FDF7D5F8FDF777F900225D4BFDF742
:1038000041F8074603910B98FDF7CAF8FDF76CF9EC
:103810003A46039BFCF71CFF079B0A9AFCF718FF2C
:10382000FDF79EF9206202AA2C21029810F0FCFB01
:10383000002804D00078532800D04E20287102AA16
:103840002C21029810F0F0FB002800D158E710A9B5
:1038500000910FAB0EAA4CA1FCF74AFD1098FDF7A2
:103860009FF8FDF741F90022414BFDF70BF80A9054
:1038700007910F98FDF794F8FDF736F900223D4BBC
:10388000FDF700F8074603910E98FDF789F8FDF75C
:103890002BF93A46039BFCF7DBFE079B0A9AFCF7E1
:1038A000D7FEFDF75DF9A0622AE7FFE7012085E773
:1038B00002AA2C21029810F0B7FB0390002812D026
:1038C000014614222248FCF7F9FC00280BD000978F
:1038D000221D20A1089B0398FCF70AFD14221C4816
:1038E0000399FCF7C0FC02AA2C21029810F09CFB63
:1038F00000287DD00FA900910EAB0DAA19A1FCF7ED
:10390000F7FC51E0504D544B30303100A001002005
:10391000F4000020474E52524D4300008007002023
:103920004750524D430000004750474741000000B8
:10393000474E47474100000047504753560000009C
:103940004750475341000000474E47534100000095
:10395000440A00202532642532642532642E253441
:10396000640000002532642532642E253464000092
:10397000804F224100004E4025733A20252E3666A6
:10398000B6C80A0D000000002533642532642E25D8
:10399000346400006F1283C0CAA1FD3F2532642544
:1039A00032642532640000000F98FCF7F9FFFDF740
:1039B0009BF80022AC4BFCF765FF00910A900E9833
:1039C000FCF7EEFFFDF790F80022A84BFCF75AFF3A
:1039D000074601910D98FCF7E3FFFDF785F83A469D
:1039E000019BFCF735FE009B0A9AFCF731FE00E0D4
:1039F00002E0FDF7B5F8206202AA2C21029810F02F
:103A000013FB002804D00078532800D04E202871E2
:103A100002AA2C21029810F007FB00282CD00FA935
:103A200000910EAB0DAA9249FCF762FC0F98FCF7CF
:103A3000B7FFFDF759F800228B4BFCF723FF0391EA
:103A400008900E98FCF7ACFFFDF74EF80022874B6C
:103A5000FCF718FF074600910D98FCF7A1FFFDF752
:103A600043F83A46009BFCF7F3FD039B089AFCF7EA
:103A7000EFFDFDF775F8A06202AA2C21029810F064
:103A8000D3FA002804D00078572800D045202873A6
:103A900002AA2C21029810F0C7FA002802D00FF0D9
:103AA000C8FC707002AA2C21029810F0BDFA002800
:103AB00003D00FF0BEFC0799887002AA2C2102984F
:103AC00010F0B2FA002802D00FF0AEFCA06402AAF7
:103AD0002C21029810F0A8FA002802D00FF0A4FCC4
:103AE000E06302AA2C21029810F09EFA002801D06F
:103AF00000783070AAE002AA2C21029810F094FA03
:103B0000002803D00FF095FC5A49487002AA2C21D6
:103B1000029810F089FA002803D00FF08AFC55496A
:103B20008870544DA878012801D10020E87002AABD
:103B30002C21029810F078FA002803D00FF079FCBD
:103B40000799C870002602AA2C21029810F06CFA7E
:103B5000002805D00FF06DFCE978090109194866C5
:103B600002AA2C21029810F05FFA002805D00FF06D
:103B700060FCE97809010919886602AA2C210298DB
:103B800010F052FA002805D00FF053FCE978090133
:103B90000919C86602AA2C21029810F045FA0700FC
:103BA00005D00FF046FCE978090109190867E878A3
:103BB000401CE870002F49D0761CF6B2042EC2D308
:103BC00044E002AA2C21029810F02EFA002802D01C
:103BD0000FF02FFCB07002AA2C21029810F024FAEA
:103BE000002802D00FF025FCF070002502AA2C213D
:103BF000029810F019FA002804D00FF01AFC61198D
:103C0000403188756D1CEDB20C2DEFD302AA2C212A
:103C1000029810F009FA002804D00FF005FC1549AD
:103C20006064086102AA2C21029810F0FDF90028B6
:103C300002D00FF0F9FBA06402AA2C21029810F028
:103C4000F3F9002802D00FF0EFFBE0640A49206A84
:103C5000884201DD002020620849A06A884201DD17
:103C60000020A062012048E4804F224100004E4025
:103C700088390008F40000200000B44200003443FA
:103C800030B519498A68012A1DD00C4625790023D0
:103C9000164A2C02242817D04D79FE2D04D2A418E0
:103CA000641960706D1C4D71C868401CC860FF28A5
:103CB00009D10879000213548218487912185370F8
:103CC000401C4871CB6030BD012010556D1CECB21A
:103CD0000C71052C00D90B710C7924252402135585
:103CE000A41865704871DFE7F4000020580A00202E
:103CF0000649800009580648091803D0C14203D07C
:103D00000020704701207047022070473C53010893
:103D1000702FFCFF10B5094A0021CB00D458844213
:103D200007D89B189B68834203D9C8008018007984
:103D300010BD491CC9B21529EFD3FEE7204C01087C
:103D400030B593B038216846FCF782FA012500248B
:103D5000059508200A940090684601F0D3F90028E0
:103D600001D0FFF7A3F81B491B4812C004601B4990
:103D700084604160083802F085F9002801D0FFF71F
:103D800095F81421144802F0A0F80C2010900E941D
:103D900000220EA90F9511940F4802F0CDF80028CB
:103DA00001D0FFF783F800210B4802F099F90028B1
:103DB00001D0FFF77BF80A4CA0680228FCD1002153
:103DC000054802F0B1F9044802F046F9606813B002
:103DD00030BD00000008014068050020FFFF000022
:103DE00008000020F8B5054604464035287D002629
:103DF000012808D001202875206881688907890F6B
:103E000001290ED101E00220F8BD0168C90708D0E0
:103E1000A06D20210843A0650126002028753046AA
:103E2000F8BDA16DFF220132914302221143A16529
:103E3000C1688907890F0091C16889088900C1603C
:103E40002068816892071143816000F0DDFD07461C
:103E50000EE000F0D9FDC01B0A2809D9A06D02218F
:103E6000884310210843A065002028750120F8BD73
:103E7000206880680028ECDB2068C168009A114344
:103E8000C160A06D80088000401CA065C5E70000EF
:103E9000F8B506460D464036317D01290DD0012189
:103EA000317501688A68520709D5816D2022114356
:103EB0008165002030750120F8BD0220F8BD174B48
:103EC0006A68D80547109A42154C8A6A2B6812D046
:103ED0005B035B0B1A438A622968490305D5A16815
:103EE0000143A1600A20FDF7C7FA2868800312D5B4
:103EF000A06838430EE05B035B0B9A438A62296833
:103F0000490302D5A1688143A1602868800302D5D6
:103F1000A068B843A06000203075F8BD0110000013
:103F2000002701400068006C7047000070B5040075
:103F300006D0A06D264600254036002802D006E0B7
:103F4000012070BDE5653575204600F0D1F8A06D03
:103F5000C00603D421688868400705D5A06D1021EC
:103F60000843A0653575EBE7A06DFF220132904351
:103F700002221043A06588688207920F5A48012ADE
:103F800002D10A68D2072BD1032362689B079A42A9
:103F900005D05B429A4202D05B009A4209D10A697D
:103FA000920092080A6121680A6963681A430A61EB
:103FB0000CE00A69920092080A6181680F2292045B
:103FC0009143816081686268114381602168CA6899
:103FD00018239A43CA602168CA68A3681A43CA6052
:103FE000816801225206914381608168228F5206C6
:103FF0001143816020688168C90004D4816801226E
:104000001207114381602068C168384A1140C160BD
:104010002169E068022923D000210843216A226B2C
:104020004903520011430843616B0843A1698903A6
:104030000843E169C90308432168CA681043C8609E
:10404000A06A0146FF39C23905D0E16A08432168F8
:10405000CA681043C860606A0121012802D00BE0E1
:104060000421DAE7206A002823D0A06D2022104323
:10407000A065E06D0843E065206C012820681FD032
:104080000169C90703D00169490849000161206835
:104090004169C908C900416120684169E26B114367
:1040A0004161E565A06D80088000401CA06500208E
:1040B00070BD2068C26801231B041A43C260DBE79D
:1040C0000269FF239B009A43026120680269636CC6
:1040D000E66C1A43A36C33431A43026120680269F9
:1040E0000A430261D3E70000002701401902FEFFE6
:1040F0007047F8B504464069254640350E46082805
:104100000BD02068C068C00709D0A06D20210843EB
:10411000A065002028750120F8BD082700E00C27C5
:1041200000F072FC009011E0701C0FD0002E05D042
:1041300000F06AFC0099401AB04207D9A06D042132
:104140000843A065002028750320F8BD206800689A
:104150003842E9D0A06D012149020843A0652068DA
:10416000C16809058A0F0C21002A1AD1226A002A87
:1041700017D10268120714D5826853070122002B59
:1041800008DB43688B434360A06D130298431043E0
:10419000A06506E0A06D20231843A065E06D1043E4
:1041A000E065A069002801D1206801600020F8BD09
:1041B00070B50446216800208968490721D4254646
:1041C0004035297D01291CD001212975E16901298A
:1041D00004D02046FDF762F9002811D1A16D0A4AEA
:1041E0001140FF2201321143A1650021E1652975CB
:1041F00022681C21116021688A6804231A438A609E
:1042000070BD022070BD0000FEF1FFFF0248416852
:104210004908490041607047005801400248416820
:1042200004229143416070470058014002484168B0
:1042300002229143416070470058014070B500244C
:10424000024620325179022903D00421C16301249E
:104250003CE001680B680E25AB430B6001680B68FE
:104260005B085B000B601A4B0168994201D1012188
:1042700021E0174B1433994201D110211BE0144B5C
:104280002833994201D1891515E0114B3C339942ED
:1042900001D189140FE00E4B5033994202D1012114
:1042A000090408E00A4B6433994202D1012109054F
:1042B00001E001210906064B083B596001215171BB
:1042C00000211171816B002900D08847204670BD04
:1042D00008000240F8B504469D4801689C4A9C4E7F
:1042E0009B4F0832206813041C363037904201D1AE
:1042F00008221EE0B04201D180221AE0B84202D169
:104300000122D20215E0924A4432904202D10122A7
:10431000D2030EE08E4A5832904201D11A4608E08C
:104320008B4A6C32904202D10122D20501E0012277
:10433000D20625461140203500293BD001680907E7
:1043400038D501680822914301608149206808310D
:10435000884201D108201EE0B04201D180201AE03D
:10436000B84202D10120C00215E0794944318842A7
:1043700002D10120C0030EE075495831884201D1B5
:10438000184608E072496C31884202D10120C0050C
:1043900001E00120C0066E494860E06B012108433E
:1043A000E0630420687100202871616B002901D04E
:1043B0002046884766480168654A20680832131518
:1043C000904201D104221EE0B04201D140221AE005
:1043D000B84201D11A4616E05D4A4432904202D1F9
:1043E000012292030FE05A4A5832904202D1012230
:1043F000920408E0564A6C32904202D101229205A2
:1044000001E001229206114238D00168490735D5F2
:104410000168890603D4026804218A4302604C497A
:1044200020680831884201D104201EE0B04201D149
:1044300040201AE0B84201D1184616E04449443100
:10444000884202D1012080030FE04149583188425F
:1044500002D10120800408E03D496C31884202D13C
:104460000120800501E001208006394948600520CF
:104470006871216B002901D02046884734480168C3
:10448000334A206808325315904201D102221EE0BF
:10449000B04201D120221AE0B84201D11A4616E0FA
:1044A0002B4A4432904202D1012252030FE0284AA3
:1044B0005832904202D10122520408E0244A6C3260
:1044C000904202D10122520501E00122520611421E
:1044D0003CD00168890739D50168890603D4016891
:1044E0000222914301601A4920680831884201D1B3
:1044F00002201EE0B04201D120201AE0B84201D1D2
:10450000184616E012494431884202D10120400386
:104510000FE00F495831884202D10120400408E0E1
:104520000B496C31884202D10120400501E0012095
:10453000400607494860E06BE06301206871002095
:104540002871E16A002901D020468847F8BD0000A3
:104550000000024070B5002805D003462033597989
:10456000002902D003E0012070BD00211971022151
:104570005971046822683749C5680A4081684669EC
:10458000294305693543294385692943C569294379
:10459000056A2943114321602F492F4C0268783165
:1045A000A24206D18A6A120912018A628A6A4068A6
:1045B00049E0294C1434A24207D18A6AF024A2436C
:1045C0008A628A6A406800013DE0234C2834A24296
:1045D00008D18A6A0F242402A2438A628A6A406848
:1045E000000230E01C4C3C34A24208D18A6A0F24FD
:1045F0002403A2438A628A6A4068000323E0164CBF
:104600005034A24208D18A6A0F242404A2438A6249
:104610008A6A8088000416E00F4C6434A24208D1F4
:104620008A6A0F242405A2438A628A6A8088000568
:1046300009E08A4209D18A6A0F242406A2438A62C9
:104640008A6A0079000602438A62012058710020BC
:1046500070BD00000FC0FFFF08000240F8B504461F
:1046600020300579012D1ED00125057102264671E5
:1046700020680768AF4307602046FEF71BFB2068F1
:104680000168314301602068016804221143016020
:1046900020680168082211430160206801682943ED
:1046A00001600020F8BD0220F8BD01B50098FEF7BA
:1046B00010FB08BD034841680122114341600020FE
:1046C0007047000000200240F8B5124D0746287CD4
:1046D00014460E46012807D0012028740E48FEF724
:1046E00045FC002802D00CE00220F8BD00216961E1
:1046F000022F09D0012F09D0002F09D00648FEF75C
:1047000035FC00212974F8BD3460FAE73480F8E7FD
:104710003470F6E7C810002050C300000548416817
:10472000C90705D00449C1600449C1600020704731
:104730000120704700200240EFCDAB890504030241
:10474000F8B51A4E0546307C0F46012807D00120E7
:1047500030741748FEF70AFC010002D021E0022065
:10476000F8BD0020C04338606C6814E02046FEF7B6
:104770009FFB0F48FEF7FAFB01460E4842680823EC
:104780009A434260426843159A434260002901D02F
:104790003C6006E08034A8686A68C0018018A042C6
:1047A000E4D8002030740846F8BD0000C81000208E
:1047B00050C3000000200240034841680222114318
:1047C000416000207047000000200240F8B50C4C0A
:1047D0001646207C0F46012808D001202074094885
:1047E000FEF7C4FB0025002802D006E00220F8BD39
:1047F00065613E600348FEF7B9FB2574F8BD000013
:10480000C810002050C300000948416889070CD532
:104810004168C90703D00749C1600749C16007491A
:1048200001610749016100207047012070470000C5
:1048300000200240EFCDAB8905040302BFAE9D8C82
:104840001615141310B502F0DFF810BD10B50449A9
:104850004A69024202D04861FFF7F4FF10BD000030
:1048600000040140F8B500230124A7E027469F403B
:104870003A4070D04D68022D01D0122D14D1DD08C0
:10488000AD002D1800952D6A5E07AC46F50E0F267B
:10489000AE46AE406546B543AC460E697546AE4081
:1048A00065462E43009D2E624D68012D05D0022DD8
:1048B00003D0112D01D0122D16D185680326AC46E8
:1048C0005D00AE46AE406546B543AC46CE68754623
:1048D000AE4065462E43866046680D79BE43ED06C0
:1048E000ED0F9D403543456006685F000325BD40E0
:1048F000AE46AE430D79B446AE07B60FBE40654630
:104900002E430660C6687546AE438D68BD4035438C
:10491000C5604D68ED0050D52B4D6E6B26436E6320
:104920009E082A4DB6007519AC46AD689E07360F35
:104930000F27B740BD4305273F07B84201D10027E5
:104940001AE0234FB84201D1012715E0214FB842A8
:1049500002D1022710E030E01F4FB84201D10327F7
:104960000AE01E4FB84201D1042705E01C4FB842AF
:1049700001D1052700E00627B7402F436546AF6009
:10498000184D2E684F689643FF0300D516432E60DE
:104990006E684F689643BF0300D516436E60AE68DD
:1049A0004F689643FF0200D51643AE60EE684F682D
:1049B0009643BF0200D51643EE605B1C0A6815469D
:1049C000DD4000D052E7F8BD001002400000014079
:1049D0000004005000080050000C0050001000506F
:1049E000001C0050000401400069084000D0012074
:1049F000704742694A4042617047002A01D0816194
:104A000070478162704700000148006870470000ED
:104A10008401002070B504000FD02168134808609D
:104A200021681348086003CC41602068083C216875
:104A30008860FFF7E9FF054608E0012070BDFFF739
:104A4000E3FF401B302801D9032070BD2068C068F7
:104A50000028F4D120680269E1688A4201D001612E
:104A600001E004490160002070BD0000CCCC0000D2
:104A700055550000AAAA0000006802490160002004
:104A800070470000AAAA000002480168491C0160A2
:104A9000704700008401002010B50648016802221A
:104AA00011430160032000F007F800F007F8002030
:104AB00010BD0000002002400020704710B50848DB
:104AC000816B02041143816300F02CF800F022F89E
:104AD0000448016808221143016000F013F810BD7A
:104AE0000010024000200240C106C90E012088408B
:104AF000014908607047000000E100E010B504F0D3
:104B00008DFE10BD02480168021511430160704717
:104B1000007000400248016842151143016070476F
:104B20000070004002480168102291430160704704
:104B300000700040094B1A689208920002431A6004
:104B40000748026904239A430261012903D040BF48
:104B500020BF20BF704730BF70470000007000408A
:104B600000ED00E00A4B1A689208920002431A60B6
:104B700008480369042213430361012906D040BF9A
:104B800020BF20BF016991430161704730BFF9E741
:104B90000070004000ED00E0F8B5664907460125C9
:104BA0000020ED03624B634A4031102F6FD011DCBF
:104BB000012F77D0022F6CD0042F6BD0082F24D177
:104BC000C9680324240321407BD0BD026C10A94294
:104BD0007CD0A0E00326584C3604202F0BD0402F69
:104BE00035D0FF3F012F10D1C968314069D07C0416
:104BF000A1426BD096E00B690969012731403F045F
:104C0000B94203D1990559E02846F8BD01256D0444
:104C1000A94203D19907F8D54848F8BDB142FCD163
:104C200011688903F9D511680320000501400120AE
:104C30000005091A09D0091A05D0814201D140485E
:104C4000F8BD2046F8BD3F48F8BD3F48F8BDC968EB
:104C50000125AD06294006D0A942F7D19168890700
:104C6000F4D53A48F8BD11688901FBD5D068D16800
:104C70008002374D000F2D5C0802810FD068491C5F
:104C8000C0030AD41068C00605D5204606E045E0FA
:104C900008E023E030E0184600E02E486843FBF7C8
:104CA00027FAF8BDCC68A407A40F0CD0022C0DD0B5
:104CB000012C10D0032CF4D1096989050029A3DB4C
:104CC000F8BD16E002E000F0D1F9F9E711684907F4
:104CD000F6D51846F4E700F0D9F9F1E7CC680C26D0
:104CE000344006D0082CF1D0042CF4D00C2CE3D0A6
:104CF000E6E700F0ABF9E3E7CC680326B602344000
:104D0000F7D00127FF02BC42E0D07A109442E2D0F3
:104D1000B442D1D0D4E7A142DDD0D1E7916B4902B2
:104D2000E7D4CDE7012212049142D4D0C8E70000B5
:104D30000024F4000010024000093D0088900000AB
:104D400020A1070040420F0080841E00006CDC029E
:104D5000484D010800127A00F8B5044600785E4D0F
:104D6000800672D55C4E0027403EB06BC00004D474
:104D7000B06BA9050843B063012758480168C9050D
:104D800011D40168821511430160FFF73DFE0090C8
:104D900005E0FFF739FE0099401A642837D84F48DC
:104DA0000068C005F5D532680321090560680A402E
:104DB0000140914208D08103890F032904D1316851
:104DC000890301D50120F8BD2A69032109040A409D
:104DD00022D0084090421FD0207880061CD5286938
:104DE0002A6988430121C9040A432A612A698A433E
:104DF0002A612861C0050FD5FFF706FE009008E084
:104E0000FFF702FE0099411A3548814201D903207B
:104E1000F8BD28698005F3D561688803800F0328F1
:104E200005D132680005824301400A433260286997
:104E3000032261681204114008432861002F04D046
:104E4000B06B012109078843B0632078C00705D003
:104E5000E868A168800880000843E860207880073F
:104E600005D5E8680C218843E1680843E8602078AC
:104E7000400706D5E8680321890288432169084371
:104E8000E8602078000706D5E86803210903884315
:104E900061690843E8602088C00506D5E8680321F9
:104EA00009048843A1690843E8602078400606D5D4
:104EB000E868012189068843216A0843E860207870
:104EC000000606D5E868032189048843E1690843A0
:104ED000E8600020F8BD0000401002400070004073
:104EE00088130000F8B5054653480E460068C00711
:104EF000C00FB0420AD25048016849084900314306
:104F000001600068C007C00FB0426FD128784B4CD9
:104F1000800705D5E068F0218843A9680843E06070
:104F20002878C00752D06868022817D0032818D004
:104F30002168012818D08905002957DAE168890815
:104F400089000143E160FFF75FFD696807460229B8
:104F500012D003291CD0012926D033E0216889030F
:104F6000EAE721688901E7E74907E5E7FFF74CFD34
:104F7000C11B3348814223D8E0680007800F022814
:104F8000F4D123E0FFF740FDC11B2D48814217D823
:104F9000E0680007800F0328F4D117E0FFF734FD25
:104FA000C11B274881420BD8E0680007800F012809
:104FB000F4D10BE0FFF728FDC11B2148814201D944
:104FC0000320F8BDE0680007800FF3D11A4801689C
:104FD000C907C90FB1420BD90168490849003143DB
:104FE00001600068C007C00FB04201D00120F8BDC9
:104FF0002878400706D5E068072109028843E96858
:105000000843E0602878000707D5E0680721C90257
:1050100088432969C9000843E06000F037F8E16877
:10502000084A0906090F515CC84007490860032077
:10503000FFF742FD0020F8BD0020024000100240B2
:1050400088130000384D01088001002004480549FC
:105050000068C968044A4905490F515CC840704757
:105060008001002000100240514D0108044805490C
:105070000068C968044A8904490F515CC8407047F8
:105080008001002000100240514D010810B5184A5F
:10509000D1680C20084004280BD0082810D00C2818
:1050A00010D050680004410F0120C003491C884003
:1050B00010BD1068C00601D50E4810BD0E4810BDC9
:1050C0000E4810BD88020E4B000F185C0902D36811
:1050D000890F491CDB0301D5084A05E01268D20696
:1050E00001D5044A00E0044A5043FBF701F810BD23
:1050F0000010024000093D000024F40000127A0074
:10510000484D0108F8B504460078FF4DC0074CD063
:10511000E8680007800F022807D0E8680007800FC2
:10512000032809D1E868C00306D5286880033CD568
:105130006068002875D038E001206268000482426F
:1051400003D129680143296011E0052301211B04D3
:1051500089049A422A6802D10A432A60F1E782430D
:105160002A602A68024000922868884328606068A4
:1051700000280DD0FFF748FC0646E44F04E0FFF797
:1051800043FC801BB8427DD828688003F7D50CE02B
:10519000FFF73AFC0646DD4F04E0FFF735FC801BC5
:1051A000B842F0D828688003F7D42078800741D52A
:1051B000E8681F270007800F3F02012807D0E86832
:1051C0000007800F032809D1E868C00306D42868C7
:1051D000400717D5E068012823D113E0E0680028D4
:1051E00017D029680922914301432960FFF70CFC7D
:1051F000064604E0FFF708FC801B0228C3D8286895
:105200004007F7D568682169B84309020843686018
:1052100010E02868400840002860FFF7F5FB0646CC
:1052200005E090E0FFF7F0FB801B0228ABD8286870
:105230004007F7D42078C00676D5E868B44E00075A
:10524000800F0BD0E06900285DD02868FF21013174
:1052500008432860FFF7D8FB074644E0286880052C
:1052600002D5E06900286ED0606A696831408842E2
:1052700012D905F0B3FD0028AED16868616AB04369
:10528000084300E0E4E068606868218C0002000ADE
:105290000906084368600FE06968B143014369602B
:1052A0006868218C0002000A090608436860606A89
:1052B00005F094FD00288FD1606A410B0120C003E6
:1052C000491C8840E968934A0906090F515CC840A7
:1052D000914908600320FFF7EFFB25E0FFF794FBFF
:1052E000C01B02288AD828688005F7D56868616ADB
:1052F000B043084368606868218C0002000A090610
:105300000843686010E02968FF200130814329606C
:10531000FFF77AFB064604E0FFF776FB801B0228C6
:1053200084D828688005F7D420787C4E000723D5E0
:1053300060690028306910D0012108433061FFF70F
:1053400063FB074605E009E1FFF75EFBC01B02288F
:105350007ED830698007F7D50EE040084000306104
:10536000FFF752FB074604E0FFF74EFBC01B022885
:105370006ED830698007F7D42078400761D5A86BD4
:105380000027C00005D4A86B012109070843A863C2
:10539000012763480168C90511D4016882151143CA
:1053A0000160FFF731FB009005E0FFF72DFB00994E
:1053B000401A64284CD85A480068C005F5D5FF202B
:1053C000A2680130824203D131690143316111E0A9
:1053D00001218902002A07D005231B029A4203D12A
:1053E00032690A433261EFE73269824332613069E0
:1053F00088433061A06800280ED0FFF705FB0090BD
:1054000006E0FFF701FB0099411A404881421FD88E
:1054100030698005F5D50DE0FFF7F6FA009006E05B
:10542000FFF7F2FA0099411A3848814210D83069E2
:105430008005F5D4002F04D0A96B0120000781431B
:10544000A9632078800630D53649A0694A1400E067
:105450007DE0002816D0AB6801200343AB606B6B86
:1054600003436B63086A10430862FFF7CDFA0646F0
:1054700004E0FFF7C9FA801B022868D8A8688007F3
:10548000F7D512E0A86840084000A860086A904379
:105490000862FFF7B9FA064604E0FFF7B5FA801B89
:1054A000022854D8A8688007F7D4A06A002853D0EF
:1054B000E9680907890F032950D00126360602281A
:1054C000286805D0B0432860FFF79EFA044640E004
:1054D000B0432860FFF798FA074604E0FFF794FA14
:1054E000C01B022833D828688001F7D4216BE06AFA
:1054F000EA680843616BFD231B049A431143084388
:10550000E860286830430FE0001002408813000074
:1055100000E00000384D01088001002040100240EA
:1055200000700040000001402860FFF76DFA04465B
:1055300004E0FFF769FA001B022808D828688001F8
:10554000F7D509E0FFF760FA001B022801D9032014
:10555000F8BD28688001F5D40020F8BD0120F8BD11
:1055600030B5014620310A78012A15D001220A708F
:1055700002234B700468CA23636204685323636286
:1055800003689C6820252C439C600068FF234362CD
:105590004A700020087030BD022030BD10B509F0FF
:1055A00069FB10BDF8B5054604462035287801286A
:1055B0001DD001202870022068702268CA20506225
:1055C000226853205062FF2001300026FF278142CD
:1055D0001CD121688A6882438A6020688168012220
:1055E000120391438160FFF70FFA009009E0022057
:1055F000F8BDFFF709FA0099411A7D20C0008142E9
:105600001BD82068C068C007F3D020E020688168FC
:105610000122520291438160206881681201914306
:105620008160FFF7F1F900900DE0FFF7EDF90099C7
:10563000411A7D20C000814205D9206847620320BD
:1056400068702E70F8BD2068C0688007EDD52068AE
:105650004762012068702E700020F8BD10B5006808
:105660000B464068C021C94301400002000ECC0433
:10567000D870E40E5C708C06A40E0904490F9C706F
:105680001970002A0AD105F0E5FBD870587805F0AA
:10569000E1FB5870987805F0DDFB9870002010BD94
:1056A00030B50B460168896A596001680969490487
:1056B000490C9960006804680F482146014088023F
:1056C0004D04800E18706D0E49065D70490E99707C
:1056D0006102490E40242140D970002A0AD105F008
:1056E000B9FB1870587805F0B5FB5870987805F03C
:1056F000B1FB9870002030BD7F7F7F0070B5040043
:1057000005D0254620356878002802D006E0012023
:1057100070BD00202870204600F042F8022068701A
:105720002168CA204862216853204862204605F05B
:10573000A4FBFF210028206803D041620420687088
:10574000E5E78268154B1A408260226890686368BA
:10575000A669184323693343184390602268E068C0
:1057600010612068026923891B041A4302612068C2
:10577000C26880239A43C2602068C26C920892007B
:10578000C264E269606902432068C36C1A43C26460
:105790002068416201206870002070BDBFFF8FFF4C
:1057A00000B597B00420009000200A90FF2001303F
:1057B00002906846FFF7A6FC002801D0FDF776FBB3
:1057C00020200E90C0020F900EA8FFF7C5FA002807
:1057D00001D0FDF76BFB08480169012292041143D7
:1057E0000161002211460220FFF788F90220FFF72D
:1057F0007BF917B000BD000040100240FEB5064620
:105800000446203630780B46012842D00120307003
:105810000220707020681D46002720358068002A0D
:1058200039D0400655D5187805F014FB287805F0D6
:1058300011FB19789878090408435978DA78090235
:10584000120411430843297809060843D96908431B
:1058500059690843054699695868084300902168CA
:10586000CA204862216853204862FF205A6A0130EA
:10587000802182424AD122689368834393602268E0
:10588000D0680840FF388238D060FFF7BDF801903B
:1058900029E00220FEBD400600D4DF70187805F034
:1058A000E1FA0204587805F0DDFA00020243987824
:1058B00005F0D8FA0243D87800040243287805F0AE
:1058C000D1FA00060243D8690243586902431546DB
:1058D000C1E7DF70AAE7FFF797F80199411A7D2029
:1058E000C00081422AD82068C068C007F3D0206871
:1058F000C56121680098486420688168FF220132F0
:105900001143816020688168120130E0206882685C
:1059100001235B029A4382602068C2680A401D49E5
:105920005118C160FFF770F801900EE0FFF76CF8B6
:105930000199411A7D20C000814206D92168FF20CB
:105940004862032070703770FEBD2068C068800711
:10595000ECD5206805622168009888642068816819
:1059600001225202114381602068816812011143B3
:10597000816009480268012149040A430260826883
:105980000A4382602168FF204862012070703770EE
:105990000020FEBD7FFDFFFF00040140F8B5054675
:1059A0000446203528780B46012815D001202870A0
:1059B000022068705878002A10D005F04BFA9878C9
:1059C00005F048FAD8789E7800040643587819788C
:1059D00000024903084316E00220F8BDC10603D5C2
:1059E000EF2108400A305870D87805F03BFA0604D9
:1059F000587805F037FA00020643987805F032FA35
:105A000006431878400306432168CA20486221688B
:105A100053204862204605F030FA0027002811D1B3
:105A200010480640206846602068C1688022914383
:105A3000C1602068806880060CD4204600F08CF895
:105A4000002807D02168FF204862042068702F706A
:105A50000120F8BD2168FF204862012068702F7086
:105A60000020F8BD3FFFFF00F8B50646044620368B
:105A700030780D4601280ED0012030700220707061
:105A8000206800278068002A07D040061AD52878A9
:105A900005F0E0F917E00220F8BD400600D4EF70F1
:105AA000287805F0DFF90204687805F0DBF90002D8
:105AB0000243A87805F0D6F90243E87800040243CF
:105AC00000920BE0EF702978A87809040843697800
:105AD000EA78090212041143084300902168CA20A1
:105AE0004862216853204862204605F0C6F9002824
:105AF0001FD1184900980840216808602068816813
:105B000001229204914381602969E8680843216871
:105B10008A68104388602068C16880229143C16010
:105B20002068806880060CD4204600F015F8002814
:105B300007D02168FF204862042070703770012070
:105B4000F8BD2168FF204862012070703770002086
:105B5000F8BD00007F7F7F0070B504460068C16813
:105B6000A0229143C160FEF74FFF7D260546F60057
:105B700006E0FEF749FF401BB04201D9032070BD8B
:105B80002068C0688006F4D5002070BD70B50400A0
:105B900006D025464035687C0026002802D005E066
:105BA000012070BD2E74204600F032F80220687487
:105BB00020680168402291430160A1686068226901
:105BC0000843E16811430843616901220843A16960
:105BD000520211400843E1690843216A0843A16A5F
:105BE000084321680860A0690421000C0840616A2C
:105BF0000843216848602168E06A08612068C1693B
:105C000092009143C161666501206874002070BDF7
:105C10007047F8B504460027684607802646403698
:105C2000707C012802D0707C22287ED100290CD003
:105C3000002A0AD0002B08D0307C012875D0012022
:105C40003074707C012802D003E00120F8BD3220BE
:105C500070746765A263A387E3872163A386E386E5
:105C6000A764E7640125A06A6D03A84207D12068F4
:105C70000168A94301602068016829430160206828
:105C80000168490603D401684022114301600121E3
:105C9000FF20E268C90205308A42616866D10029A6
:105CA00004D081420CD1E08E012809D1206B2168FB
:105CB0000088C860206B801C2063E08E401EE08658
:105CC000E08E002843D1A06AA84246D1206801682E
:105CD00001221203114301603FE02068C068A16BFC
:105CE0000880A06B801CA063B0E000220221204647
:105CF000069B06F0EBFB00287DD1206B2168008815
:105D0000C860206B801C2063E08E401EE086E08E21
:105D1000002808D1A06AA84205D1206801680122A4
:105D2000120311430160002200E0CCE00121204673
:105D3000069B06F0CBFB00287FD12068C068A16BD2
:105D40000880A06B801CA063E08F401EE087E08E7F
:105D50000028CAD1606800287BD10022012120469A
:105D6000069B06F0B3FB002867D1B6E7002904D0F4
:105D700081420BD1E08E012808D1206B411C2163A8
:105D800021680078C860E08E401EE086E08E002822
:105D900045D1A06AA84205D12068016801221203FA
:105DA00011430160002201212046069B06F08EFB74
:105DB000002842D12068C068A16B087046E000222C
:105DC00002212046069B06F081FB002835D1206B7E
:105DD000411C216321680078C860E08E401EE08687
:105DE000E08E00280AD1A06AA84207D12068026884
:105DF0000121090300E020E00A43026000220121A2
:105E00002046069B06F062FB002816D12068C26877
:105E1000A06B411CA1630270E08F401EE087E08E02
:105E20000028CCD16068002813D10022012120462F
:105E3000069B06F04BFB002802D00320F8BD08E0CB
:105E40002068C168A06B421CA2630170E08F401EF5
:105E5000E087A06AA8420FD1002201212046069BBC
:105E600006F034FB002802D0606D02210EE02068AD
:105E7000C068694608800888012280212046069B68
:105E800006F024FB002804D0606D202108436065E3
:105E9000D3E701207074A06AA84211D120688168FC
:105EA000C943C9060CD4616D0222114361650168C2
:105EB000A943016020680168294301603774C4E682
:105EC00037740020BAE70220B8E702462032137D7B
:105ED000012B07D00123137500680165537500205D
:105EE000107570470220704710B500210F4800F070
:105EF000DBF90F4CA268214653005B18521CA260CC
:105F00001880A06802280FD34A8808880021C94356
:105F1000081A401C101881B206480068FAF7E8F821
:105F200060606068C000606010BD0000680500200F
:105F30000800002080010020F8B5064604462036FF
:105F4000307D0D4601283DD001203075022070754E
:105F5000002A39D0042A46D0082A57D02B68297B3A
:105F600020689E468C466B68016A012212039143A9
:105F70000162C169026A03273F02B9431B020B4356
:105F80000F2109038B4361460907090C19430523B7
:105F90005B039A4373460A273B401B031343C161CB
:105FA00003622068C169032292029143C1612068A3
:105FB000C169AA6812021143C161012070750020F5
:105FC0003075F8BD0220F8BDEB6806CD083D2068AD
:105FD00008F0E0FD206882690C218A438261206814
:105FE0008169AA680FE0EB6806CD083D206808F0DB
:105FF000FFFD20688269032189028A43826120684B
:106000008169AA68120211438161D6E788CD287997
:1060100021688446086AFF22013290430862C869F9
:106020000A6A800880003843F027B84367463F0774
:106030003F0E07430520400282430A200340180216
:106040001043CF6108622068C1690C229143C1618D
:106050002068C1692A68AEE710B5022104462034E1
:10606000617501680A6A064B1A4203D10A68520830
:1060700052000A6000F020F800206075207510BD05
:106080001111000070B5040005D025462035687D4B
:10609000002802D006E0012070BD002028752046AF
:1060A00000F00CF802206875211D206808F036FD0C
:1060B00001206875002070BD7047000010B50748CA
:1060C000416B042211434163002204211420FEF796
:1060D00015FD1420FEF708FD10BD00000010024061
:1060E00010B502680446002906D0042907D0082903
:1060F00014D00C2907D114E0D068022301E0D06845
:1061000004231843D0600122206808F037FD20687E
:106110000168012211430160002010BDD0680823EE
:10612000EFE7D0681023ECE710B5026804460029B9
:1061300006D0042907D0082918D00C2907D118E067
:10614000D068022301E0D06804239843D060002285
:10615000206808F013FD2068016A074A114203D144
:106160000168490849000160002010BDD06808237B
:10617000EBE7D0681023E8E71111000070B5044682
:10618000006801690025C9438907002915DBC1683A
:10619000C943890711D4E91E0161012020752068D7
:1061A00080698007204602D0FFF79EFE04E000F0E1
:1061B00078F8204600F076F8257520680169C94313
:1061C000490717D4C168C943490713D40421C943F7
:1061D000016102202075206880698005800F2046BB
:1061E00002D0FFF781FE04E000F05BF8204600F0EB
:1061F00059F8257520680169C943090716D4C16893
:10620000C943090712D40821C9430161042020753C
:106210002068C0698007204602D0FFF765FE04E0D1
:1062200000F03FF8204600F03DF825752068016930
:10623000C943C90617D4C168C943C90613D410217C
:10624000C9430161082020752068C0698005800F5E
:10625000204602D0FFF748FE04E000F022F8204676
:1062600000F020F8257520680169C943C90708D1E5
:10627000C168C943C90704D1891E0161204600F0E5
:1062800012F820680169C943490609D4C168C943A5
:10629000490605D44021C9430161204600F027F892
:1062A00070BD70477047704710B5034620331C7DA2
:1062B0000022012C0AD001241C75002908D00429D1
:1062C00009D008290AD00C290DD10AE0022010BDFE
:1062D0000068426B07E00068826B04E00068C26BF4
:1062E00001E00068026C00201875104610BD704770
:1062F000014660310A7A012A0DD001220A72242255
:106300004A720068026802231A4302602020487221
:10631000002008727047022070470000FEB5054655
:1063200004466035287A00269446012811D00123BE
:106330002B7224206872206802689A4302602768E2
:10634000B8680322120590430843B860002902D0C0
:1063500015E00220FEBD60460091019021686A466A
:10636000928848681027B843104348602068416805
:106370006A4609029279090A1206114341602068AF
:10638000016819430160FEF73FFB0949009103468C
:10639000012100228905204609F037F8002801D0A4
:1063A000032601E020206872002028723046FEBDDE
:1063B000FFFFFF0170477047F8B502680446D069D7
:1063C00011680607360F07D1830605D58B0603D55E
:1063D000204608F08FFEF8BD95682023002E65D07A
:1063E000EE07F60FFF2721370F4037435ED0C70770
:1063F00006D0CF0504D501271762E26E3A43E26664
:10640000820708D5EA0706D0276802223A62E26EC0
:1064100004273A43E266420708D5EA0706D0256812
:1064200004222A62E26E02252A43E266020709D5A7
:106430000A461A40324305D0236808221A62E36EE6
:106440001343E366E26E002AC5D0800604D58806B1
:1064500002D5204608F04EFEE06E000703D4206807
:10646000806840061CD5204608F02CFE2068816814
:10647000490611D5826840218A438260606E0028F7
:106480000AD01D498163606EFDF7D8FE0028A2D0B6
:10649000606E816B8847F8BD2046FFF78CFFF8BD22
:1064A0002046FFF788FF0020E066F8BD2646C702B9
:1064B0006036002F0ADA6D0208D50120000510624F
:1064C0007372B3722046FFF775FFF8BD050605D558
:1064D0000D0603D5204608F065FFF8BD4006FCD543
:1064E0004806FAD52046146840218C431460737224
:1064F00000F0C2F9F8BD00002DF0000870B50400EE
:1065000005D025466035687A002802D006E00120D3
:1065100070BD00202872204600F026F82420687202
:1065200020680168490849000160606A002802D0BB
:10653000204608F0E5FC204608F01CFE0128E7D0C4
:10654000206841680922D202914341602068816835
:106550002A22914381602068016801221143016071
:10656000204608F033FD70BD70B50546006830491F
:10657000304C8AB0884246D1E06A01263043E0625E
:10658000E06A30400990E06A3043E062E06A3040FF
:106590000990A06BB1040843A06324216846F9F771
:1065A00057FE04200090400204906846FEF7D4FB9A
:1065B000206B30432063206B304009900EF086FA48
:1065C0001E4C1D48206000211020E160A060616128
:1065D000A161E16180202162206105206060204688
:1065E000FDF7B8FF2C66012211460B20A562FEF7CD
:1065F00085FA0B20FEF778FA012211461D20FEF7DE
:106600007DFA1D200FE00E4988420ED1606B0121FA
:106610008903084360630EF013F9002202211B2056
:10662000FEF76CFA1B20FEF75FFA0AB070BD00009F
:10663000004800400010024080000240F413002097
:1066400000380140F0B5034660339C7A202C44D1D9
:1066500000290BD0002A09D0012584682D03AC4203
:1066600006D10669002E03D1CE0701D00120F0BD6E
:106670001E7A012E31D001261E724165014640313D
:106680000A834A83FF27AC4204D10269002A12D14F
:10669000134A0EE07F22002C08D001252D07AC42C2
:1066A0000AD10469002C04D03F2202E00469002CC6
:1066B00001D08A8300E08F830021C16622229A7272
:1066C000197201688A6832438A6000680168FF2293
:1066D0002132114301600020F0BD0220F0BD000016
:1066E000FF01000010B504460068094988420DD139
:1066F00008488168002904D0E06E002801D10548CF
:106700008847012203492046FFF79CFF10BD000087
:106710000048004050030020FFB50646044660369E
:10672000707A83B00D46202858D1002D0CD00598E2
:10673000002809D00120A1680003814207D1206907
:10674000002804D1E80702D0012007B0F0BD307A5C
:10675000012843D0012030720020E06621207072B1
:10676000FEF752F901902746403705983882059880
:10677000788218E0788A401E78820698009000227D
:1067800080212046019B08F040FE002818D10120FE
:10679000A1680003814202D12069002812D021683B
:1067A000287888626D1C788A0028E3D106980090CA
:1067B000002240212046019B08F027FE002808D037
:1067C0000320C2E728882168C005C00D8862AD1C7F
:1067D000E9E72020707200203072B6E70220B4E7AB
:1067E000F8B5054604466035687A20283BD1002973
:1067F0000BD0002A09D00123A0681B03984206D1C0
:106800002069002803D1C80701D00120F8BD287AEB
:10681000012828D00120287220464030E1640282FD
:1068200042820026E66621206872216E0F48C86207
:10683000216E0F480863216E0E484863206E134690
:1068400086632768E16C3A462832206EFDF706FF22
:106850002168402008622E722068816880221143DE
:1068600081600020F8BD0220F8BD00008BF0000818
:10687000BBF0000841F0000802484068002800D042
:1068800000477047500300207047000010B51248C1
:10689000017800291ED10122027011480F490160C0
:1068A00000210164C161D30781614360826381601B
:1068B000C160016207234162C3630261C1620422B5
:1068C000426101630748416B42151143416304482B
:1068D000FDF72CFB10BD00004A03002000240140FE
:1068E00094130020001002407CB51E49064609782A
:1068F0000020002934D01C484168C9430907FBD453
:106900001A4C606B65152843606300211848FDF739
:1069100069FA184800901848019069461448FDF734
:10692000B7FAA0140190694600961148FDF7B0FA35
:106930000F48FDF73DFC0021C9430D48FDF7D9FB89
:106940000B48FDF7EFFA0A4980B20A6893680226FD
:1069500033439360096803220A60616BA943616352
:106960007CBD00004A03002000700040001002407F
:1069700094130020FFFF07000110000001460020D3
:106980000A0A00D00820084A114201D0042210430C
:10699000064A114201D002221043054A114201D099
:1069A0000121084370470000F0F00000CCCC00004B
:1069B000AAAA000038B50B231B07C518114B0FD02E
:1069C0001C152D1B18D02D1B19D0A542DD6A05D131
:1069D00008242543DD62DB6A234007E08024F8E7D2
:1069E000DC6A01252C43DC62DB6A2B4000931160DA
:1069F0001146FDF737FF38BDDD6A0224E9E7DD6A9D
:106A00000424E6E70010024010B5FFF7B7FF81004D
:106A100002484058002800D0804710BDE0100020F8
:106A200070B51C4615460E460846FFF7A7FF0A49F3
:106A3000002C0DD080000C50304602F063FE04465E
:106A400000222946FEF75AF82046FEF74DF870BDA1
:106A5000002280000A5070BDE010002010B5D2B2B4
:106A6000FDF7CBFF10BD000070B500241148FFF703
:106A70003BFF114D01000CD01048114A008B5043D0
:106A8000F9F736FB80B20E492880884203D9FE24EC
:106A90000DE0002028800B48864208D34042301881
:106AA000FE214843FF21F531F9F722FBC4B220460D
:106AB00070BD000000000244480300206000F81F81
:106AC000B80B0000C409000003494A690869496A13
:106AD00050404840704700004000F81F70B5114812
:106AE000FFF702FF104C01001AD0208B0F4A5043D1
:106AF000F9F7FEFA05460E48FFF7F6FE68430B4924
:106B0000F9F7F6FA618B0522401A12035043E28B23
:106B1000511AF9F703FB0F214902401880B270BDEA
:106B20000025E8E7000002446000F81FB80B0000F1
:106B3000000004480F494B6A0A69D218120EC2714C
:106B40004B6A0A69D218120C82710A8A8B8CD2188D
:106B5000120A42710A7C8B8CD21802714A69120E99
:106B6000C2704A69120C82708A8A120A4270097DC8
:106B7000017070474000F81F10B50D4C6078002878
:106B800014D1FFF783FE0B480068804700F0E2F95C
:106B900000F096F808F03AF904F090F90DF030FEA4
:106BA000FBF752FDFBF736FD0120607010BD0000C1
:106BB0004A030020D04C010870B5410EC0017D226F
:106BC0000023F9F7BFFA054600F072F8044600E02A
:106BD00000BF00F06DF8001BA842F9D370BD0000A3
:106BE00070B505460C4600222048FEF759FD0022EC
:106BF00029461E486668FEF731FD002221461B48E3
:106C0000FEF74EFD6068B042F1D1E878184A0146BF
:106C10005043C01C8308880726D0164968783D2257
:106C20000646504302463C3A7000801EC140880729
:106C3000D10F8918800F4910081AC018A978401E72
:106C400008180D493C2248436178E12351432278DA
:106C50001B015A438918A27810180818074A61685E
:106C60008002511A401870BD0549D7E72011002055
:106C7000B5050000A0AA990080510100FF030000A3
:106C800050554400032070470148006870470000D9
:106C90006C11002000B587B0694605A8FFF7A0FF7A
:106CA0000249096807B0401A00BD00006C110020BD
:106CB00000B587B0694605A8FFF792FF07B000BD91
:106CC00010B5084C207800280AD100F04BF8FF21BD
:106CD00001310548FEF766FC00F074F801202070D1
:106CE00010BD00008E0100202011002010B50C4CBA
:106CF0000021042001F0A8FC21688868C0040ED59A
:106D0000C868C0050BD5C86880221040FF3882389B
:106D1000C8600449900248612046FEF73FFC10BD60
:106D2000201100200004014070B50446FFF7B2FFB7
:106D3000211A0B4D0220285EC01C814201D900217E
:106D400000E00121042001F07FFC01F055FC012846
:106D500002D10220285E241A204600F03FF870BDC0
:106D60008E01002010B51449144886B0002412C0CA
:106D70001F21016084600461114944614160083849
:106D8000FEF7BCFC6946CC7501204875887508750E
:106D9000002205A90948FEF701FE0094019404941D
:106DA0000022694605480394FEF75EFE0348FEF79D
:106DB000D7FB06B010BD00000028004020110020C5
:106DC000FF03000010B5044C2046211D1830FFF7CA
:106DD00007FF206010BD00006C110020F0B587B0E7
:106DE000044614223F4901A8F9F719FA3D485038E2
:106DF000406E009000F07EF83B4802993B4A401AF2
:106E0000A105890D081887B2A10A68468078534207
:106E100002E08918401C80B29942FAD26A4615797C
:106E2000E122120102E0891A6D1CADB29142FAD240
:106E30006A46547902E0641CA4B23C393C29FAD277
:106E4000927951188EB20121890203E07A1A761CD8
:106E500097B2B6B28F42F9D203E03C3E641CB6B2A0
:106E6000A4B23C2EF9D203E03C3C6D1CA4B2ADB2FE
:106E70003C2CF9D203E0183D401CADB280B2182D75
:106E8000F9D26946C978890769464A7827D01849EE
:106E9000491E515C814202D2F9F72AF9084612498B
:106EA000CA1B10492C394A60052252068A618E702D
:106EB0004C700A460D70203210706846C079C87058
:106EC0000020C861FF2248610132C8604A6208613F
:106ED000024608462438FEF791FC07B0F0BD04498D
:106EE0000C31D5E770110020FF03000080AEFEFFDB
:106EF000594D010810B506480168C8688022104045
:106F0000FF388238C86051000148FEF74BFB10BDC6
:106F10002011002010B57D2108F053FB4906C0095F
:106F2000084310BD10B5410EC0017D220023F9F7C2
:106F300009F910BD01B582B00020C04300900123C3
:106F400001AA02A90248FEF764FE684680880EBDC9
:106F50008811002010B51C481A4901601C4A1B4BBF
:106F60000021126803E05208491C072901D29A4205
:106F7000F9D84A078B07D20FDB0F52011B011A43C6
:106F8000C90700D008210A43C26100218160016164
:106F90004161FF22C16005328162426001220162CB
:106FA0005202826141620B48416B8214114341637A
:106FB0000548FEF7EBFD002801D0FBF777FF00F056
:106FC00045F810BD003001408811002080969800DF
:106FD000800100200010024070B586B01421684680
:106FE000F9F736F905260125022436076A4680217D
:106FF000304601950294FFF7DDFC002280213046E7
:10700000FFF72CFD6A46402130460294FFF7D2FC80
:10701000002240213046FFF721FD6A4620213046FC
:107020000294FFF7C7FC002220213046FFF716FD2F
:10703000A4036A46214630460295FFF7BBFC0122B5
:1070400021463046FFF70AFD06B070BD30B585B069
:1070500014216846F9F7FCF8022001900290032001
:10706000039000200524240704906A46202120462E
:10707000FFF7A0FC6A4640212046FFF79BFC6A46CA
:1070800080212046FFF796FC01210191CD0302915A
:107090006A4629462046FFF78DFC012229462046F4
:1070A000FFF7DCFC05B030BD00BFFDE770B5012483
:1070B000052564022D07002221462846FDF79DFC88
:1070C00005F0E8F9002261002846FDF796FC00F083
:1070D0000DF8012221462846FDF78FFC00F006F846
:1070E000002221462846FDF788FC70BD08B5072020
:1070F0000090401E0090FCD108BD000008B50B4870
:10710000C16A01221143C162C06A1121104000907E
:1071100007484160002181600321C160490201608C
:10712000014605200007FDF79DFB08BD0010024049
:107130004407002070B50124052564022D070022B4
:1071400021462846FDF759FC05F0A4F901229102D9
:107150002846FDF752FCFFF7C9FF012221462846C9
:10716000FDF74BFCFFF7C2FF002221462846FDF742
:1071700044FC70BDF1B505F071F9002401267602DA
:10718000052725463F076006040E00223146384693
:10719000FDF733FCFFF7AAFF012231463846FDF721
:1071A0002CFC012189023846FDF71EFC002801D085
:1071B000641CE4B2FFF79AFF6D1CEDB2082DE2D318
:1071C0000098002803D0FFF771FF2046F8BDFFF7B5
:1071D000B1FFFAE7F8B5054605F05CF90126052789
:1071E00076023F07002231463846FDF706FC0024B0
:1071F000280601D5012200E000220121890238463B
:10720000FDF7FBFBFFF772FF012231463846FDF721
:10721000F4FBFFF76BFF002231463846FDF7EDFB2C
:10722000012291023846FDF7E8FB6806050EFFF7DC
:107230005DFF641CE4B2082CDAD3F8BD70B505F02C
:1072400029F90122052594022D0721462846FDF73C
:10725000D4FB0122560231462846FDF7CEFBFFF74C
:1072600045FF002221462846FDF7C7FBFFF73EFFFA
:10727000002231462846FDF7C0FBFFF737FF70BDFF
:1072800070B505F007F90124052564022D070022D9
:1072900021462846FDF7B1FB66000022314628460C
:1072A000FDF7ABFBFFF722FF012221462846FDF741
:1072B000A4FB012231462846FDF79FFBFFF716FF8E
:1072C00070BDF8B5002405F0C9F801220525960225
:1072D0002D0731462846FDF790FBFFF707FF0122F7
:1072E000570239462846FDF788FBFFF7FFFE07E007
:1072F000641CE4B2FA2C03D9FFF7C2FF0120F8BDE9
:1073000031462846FDF770FB0028F1D100223946AE
:107310002846FDF772FBFFF7E9FE0020F8BD0000EC
:1073200010B50448FDF7A8FB002801D0FBF7BEFD0F
:1073300010BD0000580500200149052088717047E4
:10734000A403002010B507A1095C07A007F070FD99
:107350000C480021017102214171002100F0E0FC84
:1073600010BD000041424300737769746368207464
:107370006F20636C61737320256320646F6E650AF0
:107380000D0000001C030020014900200872704716
:10739000A40300200149012008727047A4030020C3
:1073A000F8B52D480125057003F088FD2BA007F0E6
:1073B0003FFD0028FAD1FBF747F901220526140307
:1073C000360721463046FDF718FB012217023946E1
:1073D0003046FDF712FB7D20C000FBF77AFC00224F
:1073E00021463046FDF709FB002239463046FDF7BD
:1073F00004FB1D4C002060710BF01AFB012801D129
:107400000CF016FA194807F0D1FC002000F054F9EE
:10741000FFF74EFC206515481549283807F014FC85
:107420001248FF21F531283807F076FC03F032F8D6
:107430000E481049143007F007FC0C480E49143070
:1074400007F06AFC0DF01CF80BF0EAFD7F200B49F9
:10745000C0058863A573F8BDA40300204A4F494EB8
:1074600045440D0A00000000940100201C13002078
:1074700095A4000881440108409C0000800700207A
:1074800070B5354CE161606203F018FD33A007F080
:10749000CFFC37A007F0CCFC3BA007F0C9FC41A013
:1074A00007F0C6FC0CF0E8FB0BF0F6F921460120D2
:1074B00030310870414840490160414941604149CB
:1074C0008160606A214600682031086005223B48DF
:1074D00001F00CF9394D02200C352870E069007874
:1074E0002871284601F0BAFB07202870E0698078EF
:1074F0002871284601F0B2FB002028702871284628
:1075000001F0ACFBE0694178204670302E4C0175EB
:107510002046FBF7D7FD002809D02046FBF7D2FD17
:1075200012280ED003F0CAFC00F06EF870BD0BF00C
:10753000B1F811212046FBF7A3FD24A007F078FC49
:1075400070BD0BF0A7F82046FBF748FD112120463F
:10755000FBF796FD02F0A0F9A40300200A0D4C47AA
:10756000542D3932204465766963650A0D000000A8
:10757000496D6167652056657273696F6E3A207652
:10758000312E362E350A0D004C6F526157616E2038
:10759000537461636B3A2044522D4C57532D303055
:1075A000350A0D004672657175656E63792042611A
:1075B0006E643A2000000000359700087417002020
:1075C00039970008D5970008808F0108506C6561D5
:1075D0007365207365742074686520706172616DD5
:1075E0006574657273206F722072657365742044D0
:1075F000657669636520746F206170706C792063B3
:1076000068616E67650A0D0070B5234D002029780A
:107610002E46303E86B0012928D0204C032121700F
:107620006060204601F01AFB04202070E86860606A
:10763000204601F013FB05202070284628306060AA
:10764000204601F00BFB0620207028463830606091
:10765000204601F003FB012020702071204601F03C
:10766000FDFA706A4069804706B070BD69460870CF
:10767000094801AD801C01900E3002900830039043
:10768000F069C07808741ECD04481C381EC06846D6
:1076900001F028FCE8E70000D40300208017002058
:1076A0000EB501216846017001F05CFA6846007968
:1076B000012800D000200EBDFEB506460024684615
:1076C0002746047001F04EFA68460079B04223D094
:1076D0003100124E124D02D002291DD10DE00028BA
:1076E0001AD16846077101F0B9FA002803D1706A0F
:1076F000816900200FE02C460EE0002800D02C46C7
:10770000022069460871684601F0A8FA0028F2D103
:10771000706A8169022088472046FEBDA4030020CC
:10772000FFFFFFFFFEB505460279016840790CF0C6
:1077300035FC2868FE4A0178D41F01260027F93C51
:10774000A5297DD014DC21297BD00CDC04292FD085
:1077500004DC012916D0022932D14BE005293ED0A4
:107760002029F9D18FE122296CD02329F4D15DE2BF
:10777000A8390B0007F03DFF0AC8F1939DA3A9BBF0
:10778000C2F0EF2429790429E6D1417883780904ED
:107790001B02C07819430143D162062902D2E54891
:1077A000E06241E27D20C00066704143E1623BE25D
:1077B00029790229D0D14078FF2802D0FE2802D0B2
:1077C00037E2E67030E2DC48FBF708FC1221DA48C9
:1077D000FBF756FCD8488030FBF700FCF1E729792D
:1077E0000229EDD14078012801D00028E8D10BF022
:1077F00031F99BE129790229E2D140780128DFD1D2
:10780000FFF756FA2065CD493C200870CC49087036
:10781000A763CC482764006801280BD1FAF714FF4E
:107820000122052011020007FDF7E7F87D20C000C6
:10783000FBF74FFAFF21002201310520000702E08B
:1078400007E02DE134E1FDF7D8F8BFA007F0F0FA2A
:10785000EFE12979C04A022902D0042906D01BE0B1
:107860004178BEA0116007F0E3FA0EE041780329E9
:107870000BD1116028688278BB4802602868C37801
:10788000BA480360BAA007F0D3FA28684078002805
:1078900002D0FFF70DFA2065BC480670F0E02979A8
:1078A0000329FBD1817842780802104340BAB849D5
:1078B000B1E029790229F1D14078B649ABE02979C4
:1078C0000229EBD14078B449A5E029790329E5D113
:1078D000817842780802104340BAF9F787F800220D
:1078E000AE4BF8F7CFFFF9F73BF9AD4993E02979B3
:1078F0000229D3D1417893480160C1E02979022956
:10790000CCD14078A74986E029790A29C6D14078A8
:10791000012823D001210520277400220903000734
:10792000FDF76BF828680079012834D0FF21052085
:107930006774002201310007FDF75FF82868C079FD
:10794000012845D00121052067740022C9020007E3
:10795000FDF753F894E060E058E075E0FAF75AFE5E
:107960000122052011030007FDF747F82674296856
:10797000C87889780002084340BAE0660028D1D070
:10798000FBF7A7F901210520002209030007FDF7F5
:1079900034F82774C6E7FAF73DFE012205201102EC
:1079A0000007FDF72AF86674286881794079090292
:1079B000014348BA20670028C0D0FBF78AF9FF21AD
:1079C0000520002201310007FDF717F86774B5E7BD
:1079D000FAF720FE01220520D1020007FDF70DF87D
:1079E000A6742968487A097A0002084340BA606799
:1079F000216F002944D0FBF76CF9012105200022FA
:107A0000C9020007FCF7F9FFA77439E029790229B8
:107A100036D140786449086032E0417883780904BF
:107A20001B02C07819430143D162062905D25FA029
:107A300007F0FEF96648206322E07D20C000414344
:107A4000667064A0216319E0297904291AD141786C
:107A5000837809041B02C07819430143FF20693071
:107A6000D162814205D260A007F0E2F96748606305
:107A700006E07D20C000414365A0616307F0D8F9AE
:107A800006F0F4FDD5E02979022917D140780028C5
:107A900001D0012812D10AF0D1FF06F0E7FD90E6EF
:107AA000297902290AD14078042807D8A0713DE03D
:107AB00029790220022902D004290ED0B9E02968D0
:107AC0004978012933D16946087028684078002830
:107AD00000D001200871084626E02968497800296D
:107AE00025D16946087028684078002800D0012018
:107AF0000871084601F0B2F828688078FF2808D09D
:107B0000152168460170286881786846017101F086
:107B1000A5F82868C078FF2808D0162168460170AB
:107B20002868C1786846017101F098F87AE080E031
:107B30009402002070170000808F01089A04002032
:107B40009B040020700300204578697420416C611B
:107B5000726D0D0A00000000740300204D443A20AD
:107B6000253032780A0D00007C03002080030020BD
:107B7000536574204D443A20253032782C2530321C
:107B8000782C253032780A0D0000000063030020B5
:107B900068030020620300206103002000002440ED
:107BA000BC030020780300206C03002041434520E3
:107BB00073657474696E67206D75737420626520D7
:107BC0006D6F7265207468616E203130530A0D004C
:107BD00010270000536574204143453A2025642056
:107BE0006D730A0D000000004B41542073657474DE
:107BF000696E67206D757374206265206D6F7265A4
:107C0000207468616E20366D0A0D0000407E05000C
:107C1000536574204B41543A202564206D730A0D3E
:107C20000000000006F022FD267002E029790229FA
:107C300003D06078012806D017E00121415608469C
:107C40000AF07EFE72E706F011FD2049204806F09A
:107C5000FBFF1F48A16A07F05FF81D4807F06EF8A8
:107C60001B48283007F06AF867701AA007F0E0F8A0
:107C70000028FAD118A007F0DBF80028FAD12879FB
:107C800008281BD82078002818D0697916A007F09A
:107C9000CFF80028F9D1002607E02868815D13A0FD
:107CA00007F0C6F80028F8D1761C2879B042F4DC39
:107CB0000CA007F0BDF80028FAD105E029790DA045
:107CC00007F0B6F80028F9D12770FEBD59A40008C6
:107CD000E01200200D0A0000526563656976652098
:107CE000646174610A0D000025643A002530327821
:107CF000200000004275666653697A653A25642C57
:107D000052756E2041542B52454356423D3F2074DC
:107D10006F207365652064657461696C0D0A0000ED
:107D200070B586B00E4604460AF09CF90025ED4376
:107D3000002822D1207904A901F0E8F902460021A7
:107D40001548002A04D06A461170029191811FE003
:107D5000002E15D0012269460A7062790A712279D3
:107D60008A812168029108226946CA73007D88735E
:107D7000684600F061FE002800D0284606B070BDBD
:107D80006A4611706179117121799181216802919E
:107D9000007D9073ECE7000014040020F8B51D4C42
:107DA000064601212068C905884201DA3046F8BD3F
:107DB000A168E069F8F7C5FB05466168A069F8F7B6
:107DC000C0FB3146F8F7B9FB2946F8F7B2FB054688
:107DD00007F04CFC002804D1284607F03EFC0028A0
:107DE00000D035466169E069F8F7ABFB0090A06907
:107DF00021690746F8F7A5FB06462846E168F8F72B
:107E0000A0FB3146F8F744FB0099F8F741FBE76126
:107E1000A561F8BD34000020F8B51D4C06460121CF
:107E2000206AC905884201DA3046F8BDA16AE06BD4
:107E3000F8F787FB0546616AA06BF8F782FB3146CD
:107E4000F8F77BFB2946F8F774FB054607F00EFCB4
:107E5000002804D1284607F000FC002800D0354651
:107E6000616BE06BF8F76DFB0090A06B216B074630
:107E7000F8F767FB06462846E16AF8F762FB3146E9
:107E8000F8F706FB0099F8F703FBE763A563F8BD75
:107E900034000020F8B51D4C06460121206CC905B0
:107EA000884201DA3046F8BDA16CE06DF8F749FB75
:107EB0000546616CA06DF8F744FB3146F8F73DFBD1
:107EC0002946F8F736FB054607F0D0FB002804D119
:107ED000284607F0C2FB002800D03546616DE06DF2
:107EE000F8F72FFB0090A06D216D0746F8F729FBEE
:107EF00006462846E16CF8F724FB3146F8F7C8FA45
:107F00000099F8F7C5FAE765A565F8BD34000020CB
:107F1000F8B51D4C06460121206EC905884201DADC
:107F20003046F8BDA16EE06FF8F70BFB0546616EB9
:107F3000A06FF8F706FB3146F8F7FFFA2946F8F785
:107F4000F8FA054607F092FB002804D1284607F00E
:107F500084FB002800D03546616FE06FF8F7F1FA36
:107F60000090A06F216F0746F8F7EBFA0646284607
:107F7000E16EF8F7E6FA3146F8F78AFA0099F8F771
:107F800087FAE767A567F8BD34000020F8B51D4CF7
:107F9000064601212068C905884201DA3046F8BD4D
:107FA000A168E069F8F7CDFA05466168A069F8F7BD
:107FB000C8FA3146F8F7C1FA2946F8F7BAFA054681
:107FC00007F054FB002804D1284607F046FB0028A0
:107FD00000D035466169E069F8F7B3FA0090A0690E
:107FE00021690746F8F7ADFA06462846E168F8F732
:107FF000A8FA3146F8F74CFA0099F8F749FAE76120
:10800000A561F8BDB4000020F8B51D4C064601215D
:10801000206AC905884201DA3046F8BDA16AE06BE2
:10802000F8F78FFA0546616AA06BF8F78AFA3146CD
:10803000F8F783FA2946F8F77CFA054607F016FBAD
:10804000002804D1284607F008FB002800D0354658
:10805000616BE06BF8F775FA0090A06B216B074637
:10806000F8F76FFA06462846E16AF8F76AFA3146E9
:10807000F8F70EFA0099F8F70BFAE763A563F8BD75
:10808000B4000020FEB50D46F8F798FAF8F72CFD7D
:1080900002460B4628482949F8F7F4FBF8F760FD3B
:1080A0000CF036F901460090F8F74BFA04460190BF
:1080B00023480AF027FA0121F8F7BEFA0099F8F7E9
:1080C00040FA7F27FF053946F8F7E2F92146F8F72D
:1080D000DFF906461B4C0120C0052560854229DBDF
:1080E00031460198F8F76AFA05460121E060F8F791
:1080F000A3FA6561206139460198F8F71AFA01215F
:10810000F8F79AFA3146F8F759FA60600C48019D81
:108110000AF0F8F90121F8F78FFA0099F8F711FA47
:108120003946F8F70AFA2946F8F7B2F93146F8F76E
:1081300045FAA060FEBD00004AD8124DFB2109405F
:10814000DA0F493F34000020FEB50D46F8F736FA45
:10815000F8F7CAFC02460B4628482949F8F792FB73
:10816000F8F7FEFC0CF0D4F801460090F8F7E9F9B6
:108170000446019023480AF0C5F90121F8F75CFA9A
:108180000099F8F7DEF97F27FF053946F8F780F9FF
:108190002146F8F77DF906461B4C0120C0052562F3
:1081A000854229DB31460198F8F708FA0546012196
:1081B000E062F8F741FA6563206339460198F8F701
:1081C000B8F90121F8F738FA3146F8F7F7F96062A3
:1081D0000C48019D0AF096F90121F8F72DFA009953
:1081E000F8F7AFF93946F8F7A8F92946F8F750F942
:1081F0003146F8F7E3F9A062FEBD00004AD8124DFF
:10820000FB210940DA0F493F34000020FEB50D463E
:10821000F8F7D4F9F8F768FC02460B4628482949D4
:10822000F8F730FBF8F79CFC0CF072F80146009070
:10823000F8F787F90446019023480AF063F9012111
:10824000F8F7FAF90099F8F77CF97F27FF05394626
:10825000F8F71EF92146F8F71BF906461B4C0120DA
:10826000C0052564854229DB31460198F8F7A6F957
:1082700005460121E064F8F7DFF9656520653946B8
:108280000198F8F756F90121F8F7D6F93146F8F7D1
:1082900095F960640C48019D0AF034F90121F8F762
:1082A000CBF90099F8F74DF93946F8F746F9294620
:1082B000F8F7EEF83146F8F781F9A064FEBD00004A
:1082C0004AD8124DFB210940DA0F493F3400002003
:1082D000FEB50D46F8F772F9F8F706FC02460B46B4
:1082E00028482949F8F7CEFAF8F73AFC0CF010F8CC
:1082F00001460090F8F725F90446019023480AF05A
:1083000001F90121F8F798F90099F8F71AF97F2790
:10831000FF053946F8F7BCF82146F8F7B9F80646E4
:108320001B4C0120C0052566854229DB314601989A
:10833000F8F744F905460121E066F8F77DF965672D
:10834000206739460198F8F7F4F80121F8F774F935
:108350003146F8F733F960660C48019D0AF0D2F80F
:108360000121F8F769F90099F8F7EBF83946F8F7C1
:10837000E4F82946F8F78CF83146F8F71FF9A066BB
:10838000FEBD00004AD8124DFB210940DA0F493FDB
:1083900034000020FEB50D46F8F710F9F8F7A4FBFD
:1083A00002460B4628482949F8F76CFAF8F7D8FB3B
:1083B0000BF0AEFF01460090F8F7C3F804460190B9
:1083C00023480AF09FF80121F8F736F90099F8F7E9
:1083D000B8F87F27FF053946F8F75AF82146F8F72D
:1083E00057F806461B4C0120C0052560854229DB55
:1083F00031460198F8F7E2F805460121E060F8F708
:108400001BF96561206139460198F8F792F801215E
:10841000F8F712F93146F8F7D1F860600C48019D81
:108420000AF070F80121F8F707F90099F8F789F8D0
:108430003946F8F782F82946F8F72AF83146F8F76E
:10844000BDF8A060FEBD00004AD8124DFB210940D6
:10845000DA0F493FB4000020FEB50D46F8F7AEF83C
:10846000F8F742FB02460B4628482949F8F70AFA72
:10847000F8F776FB0BF04CFF01460090F8F761F837
:108480000446019023480AF03DF80121F8F7D4F89A
:108490000099F8F756F87F27FF053946F7F7F8FFF8
:1084A0002146F7F7F5FF06461B4C0120C005256263
:1084B000854229DB31460198F8F780F8054601210D
:1084C000E062F8F7B9F86563206339460198F8F778
:1084D00030F80121F8F7B0F83146F8F76FF860622C
:1084E0000C48019D0AF00EF80121F8F7A5F8009953
:1084F000F8F727F83946F8F720F82946F7F7C8FFC4
:108500003146F8F75BF8A062FEBD00004AD8124D74
:10851000FB210940DA0F493FB400002010B50B4899
:108520000168002904D000F014F800F03AF810BDFA
:108530004068002804D000F013F800F033F810BDB4
:1085400000F006F800F02CF810BD00003405002003
:10855000704710B501210020FCF7ECFA10BD0000B7
:1085600010B5EFF3108472B6FEF736FD0A48406886
:1085700080470AF08DFA012801D0FAF755FF074825
:10858000016804221143016084F310880121084628
:10859000FCF7E8FA10BD0000D04C01080070004064
:1085A0007047704710B5EFF3108472B61048016839
:1085B00001221143016001684907FCD501680122CD
:1085C00012061143016001688901FCD5C1680322CC
:1085D0001143C160C1680907890F0329FAD1FEF769
:1085E00035FD04480068804784F3108810BD000002
:1085F00000100240D04C0108EFF3108172B607481A
:108600000268002A01D0002005E04068002801D05F
:10861000012000E0022081F310887047340500201B
:1086200010B5EFF3108272B6064B00295C6803D0D8
:10863000012903D1044300E084435C6082F3108885
:1086400010BD00003405002010B5EFF3108272B6A3
:10865000064B00291C6803D0012903D1044300E024
:1086600084431C6082F3108810BD00003405002094
:10867000F8B5174605460A461948069C089E07990C
:10868000447183711C0AC4711C0C04721B0E43726A
:1086900081720B0AC3720B0C0373090E4173D4B2BF
:1086A000C4731048F8F7CAFF39460E48F8F7D6FFEA
:1086B00010220B490B48F8F7D9FF224629460948F2
:1086C000F8F7D4FF0749C81FFD38F8F719FF064C23
:1086D000601CF7F702FE2178000208433060F8BD05
:1086E00010050020D01D0020CC1C0020F8B50E463F
:1086F000050017467ED028680028FBD0686800284F
:10870000F8D0A8680028F5D0104603F09BFD00289B
:1087100071D0784C00212667E56622462776223202
:1087200011706176921E2164117001265670E176F7
:108730006166A1660F216A4611703846694603F0EA
:1087400070FD002800D0012020770A2168460170C2
:108750006946207E03F065FD674D06212870684656
:1087600001706946207E03F05CFD68701021684648
:1087700001706946207E03F054FDE86011216846CF
:1087800001706946207E03F04CFD28611221684685
:1087900001706946207E03F044FD6861132168463C
:1087A00001706946207E03F03CFDA86114216846F3
:1087B00001706946207E03F034FDE86117216846A8
:1087C00001706946207E03F02CFD2F46203778701B
:1087D0001821684601706946207E03F022FD686218
:1087E0001921684601706946207E03F01AFD38722F
:1087F0001E2101E079E07AE0684601706946207E3A
:1088000003F00FFD38731F21684601706946207E12
:1088100003F007FD78732021684601706946207EC9
:1088200003F0FFFC28632121684601706946207E21
:1088300003F0F7FC68630021207E03F0FCFC3E702F
:108840000A2068600620287228460A2138384160CC
:1088500006210172E968C1602969016169694161A4
:10886000A9698161E969C1612030067003F05CFD8E
:1088700028462249383006F0E7F97D212846C9000C
:10888000383006F049FA28461D49683006F0DCF910
:1088900028461C497C3006F0D7F928461A49903002
:1088A00006F0D2F928461949CC3006F0CDF906F089
:1088B000B9F9E063284616494C30016015498160DA
:1088C00015490161154941601549164DC160A968F6
:1088D0008847E86980470BF0E7FBA676296E3046AB
:1088E0008847686B80470020F8BD0320F8BD0A2048
:1088F000F8BD000094040020A41B0020419900084A
:10890000E5A30008F1A200086DA30008B5980008CF
:10891000C9A10008DD9B000801A10008B5A200085C
:1089200061A10008D04C0108F8B504461D46174661
:108930000E460D48F8F782FE39460B48F8F78EFED2
:10894000F2B221460848F8F791FE0749C81FFD38E2
:10895000F8F7D6FD054C601CF7F7BFFC2178000244
:1089600008432860F8BD0000D01D0020CC1C00206A
:10897000FFB585B00F46044607ADF02200211D4823
:108980000E9E0AF03BFC1B4A1021204607F060FCBB
:108990001022002168460AF031FC0121684601706E
:1089A000062239466C46401C0AF010FC0222294679
:1089B000E01D0AF00BFC0F4A6846089907F01DFC01
:1089C0001022002168460AF019FC02216846017055
:1089D00006223946601C0AF0F9FB02222946E01DF6
:1089E0000AF0F4FB034A3146684607F006FC09B07A
:1089F000F0BD0000DC1C0020F8B517460E46054609
:108A00001C46F02200210B480AF0F8FB094A10210D
:108A1000384607F01DFC074A2146284607F0EDFBC3
:108A2000102E06D321462846024A1031103007F096
:108A3000E4FBF8BDDC1C0020F0B5044687B0022042
:108A40000490002006460190002C79D04248016C29
:108A5000CA0701D1C80602D5012007B0F0BD002029
:108A600069460872014614223C480AF0C7FB3B489D
:108A700001214170384801752178002904D001296D
:108A80000AD0032926D118E00126C6746A46117A55
:108A9000C906C90E403107E0E17BC1746A46117A0C
:108AA0000126C906C90E8031117221790191A16890
:108AB00000910E25A78965570CE00126C6746A4609
:108AC000117AE02211436A461172616800910A2509
:108AD00027896557022269460A75214906910A7B52
:108AE00069468A751C4805A9007E03F09AFBA842D6
:108AF00000D3054668B2002E1FD0174DE97A002931
:108B000010D16946087306980522007B887303A973
:108B1000287E03F0FEFB002812D011496846007B36
:108B2000203948703B4602A8009A019905F070FC74
:108B30000490002806D00020287304988DE7FFE7F2
:108B400003208AE70548217801700348012222307A
:108B5000017811430170F0E7940400209C1C002070
:108B60008C1B0020F8B500250446002818D0394990
:108B7000277837480E463836027E3B0006F039FD2E
:108B80001E121417191B1E2023252729303B39429A
:108B900046484A4C4E50525654585A5C5E60626485
:108BA0000320F8BD407E00E0807A20714DE0C07A5D
:108BB000FBE7C06D00E0006E606046E02648FBE722
:108BC00025481030F8E7807EEFE7C07EEDE71D20F6
:108BD00012E020492039486C896CA160606034E063
:108BE0001C49203908467C30C96F40686160A0602C
:108BF0002BE01B2000E01A2069460870104603F0A5
:108C000010FBD9E7134820300078CEE7C868D3E7D7
:108C10000869D1E74869CFE78869CDE7C869CBE73C
:108C20007078C2E74878C0E73078BEE70878BCE7DC
:108C3000006BC1E7406BBFE7C06ABDE74868BBE7B0
:108C4000087AB2E7486BB7E702252846F8BD00006E
:108C5000940400206C1B00204C180020F0B5002468
:108C600089B00746002806D09A4D286CC00704D06A
:108C7000012009B0F0BD0320FBE7984E3A7830465A
:108C800020300290407B039092489349007E13006D
:108C900006F0AFFC1E102124272A2D333C41F0445E
:108CA000839A96A6ADB0B3B6B9BCCCF1D9EEEDF0CF
:108CB000ECEBEAF038796876002804D0012804D07B
:108CC000022802D102E0486B804701E100202873AE
:108CD00001F04CFBFCE03879A872F9E03879E872D1
:108CE000F6E07868E865F3E078682866F0E079688F
:108CF000002974D010227A4805E0796800296ED0E6
:108D00007748102210300AF061FAE1E03879A8764D
:108D1000096E8847DCE03879E876D9E0397A6A4626
:108D2000117103995171072201A903F0F2FA002889
:108D30007BD06A49BA68203978688A644864687E5A
:108D4000022827D1A87A002824D0644F0298F0374F
:108D5000009708214156327A7368287E02F09DFC04
:108D6000687F3870706A786002983A46407B387441
:108D7000E87E78740120F874B8742C323946287E65
:108D800003F08FFA002806D0B87CF16803F05AFB94
:108D9000F87CA8759CE00C249AE0397A6A46117137
:108DA00003995171072201A903F0B3FA002859D0A1
:108DB0004A48BB6820387A688021C2670B5087E038
:108DC00079680691012102E07968069100216A46DE
:108DD000117706A902F039FA002843D078E041E083
:108DE0003879411E0E293DD80299087070E07868E4
:108DF000F0606DE0786830616AE07868706167E023
:108E00007868B06164E07868F06161E039796A4659
:108E10001171062201A903F07CFA002822D06846CD
:108E200001792E483830417052E039E039796A468C
:108E30001171052201A903F06CFA002830D06846B0
:108E40000079707044E039796A4611710A2201A9EB
:108E500003F05FFA002805D0684601791F483830D2
:108E6000017035E0032433E02EE027E020E01CE031
:108E700018E000E02BE039796A461171092201A956
:108E800003F047FA002802D06846007906E06946F8
:108E900004200856014628390A2901D8307017E005
:108EA0000B2415E07868286312E0786868630FE0A7
:108EB0000A48796838304160716009E007483979BB
:108EC00038300172317203E07868706300E0022488
:108ED0002046CEE694040020D04C01086C1B0020F4
:108EE0004C180020F0B50446022085B00090002CFC
:108EF00041D04E48006CC00718D10C2200214C48CC
:108F00000AF07CF94A4E01207070484D20780827FD
:108F10002235002806D001286AD0022874D0032800
:108F20005DD179E04148006CC00602D5012005B052
:108F3000F0BD40480178002906D0002101703B486F
:108F40000221007E03F077F96068002813D0A06842
:108F5000002810D0E06800280DD0207C00280AD01E
:108F6000694608733148222203A9007E03F0D1F933
:108F7000002802D00AE00320D9E7232069460874BC
:108F80002A4804A9007E03F04CF920742878694629
:108F90003843287020783070244E60683065A068AF
:108FA0007065E068B065207C344620346070002035
:108FB0002070087103F0B8F920786946401C0881D8
:108FC00002A9307E02F01DF91B49002348701A46A1
:108FD000194601A805F01CFA0090002806D0134994
:108FE000002008732878F7210840287000989EE731
:108FF00028780022384328702078307011460220EB
:10900000F9F798FAE8E7FFE73070287838432870D6
:10901000A08805F0E3FADFE730702878384328703D
:10902000227BA088A16805F003FBD5E7940400200B
:10903000B01C0020430300206C1B0020FEB508AFCD
:1090400070CF6F4670C700F001F8FEBDFFB50D464A
:10905000002681B01F460124F022314629480AF03B
:10906000CDF8284A1021039807F0F2F826480A990B
:1090700041718771390AC171390C0172390E41721F
:109080000B9981720B991F4F090AC1720B99090C38
:1090900001730B99090E4173203F18E01A48194AD1
:1090A000C473641C1146A4B2203907F0A6F800204E
:1090B0003118019A3B5C525C401C5A400C9B80B2B8
:1090C0005A541028F4D3103D1036ADB2F6B2102D1C
:1090D000E4D2002D13D00B4A0B481146C47320393B
:1090E00007F08BF8002008E0019A3118525C3B5CD5
:1090F0005A400C9B401C5A5480B2A842F4D305B08D
:10910000F0BD0000DC1C002020050020F3B52B483A
:1091100087B00E46427869460A710078284C087676
:10912000E07B217C4018C5B2002E32D00021684679
:109130000172E17A4172A06B2049039038394A7874
:10914000684602741D4F09784174183F397B817459
:1091500020463830009006AB01AA02A9207E02F01A
:1091600041F8397B68468175017941750D2101759A
:10917000E07E002802D00E206946087505A9207EF1
:1091800003F04FF8C0B27070A84205D3401B307096
:1091900006E0032009B0F0BD30700025E5732574AA
:1091A0006846042141562A46079806F067F90028C8
:1091B00001D00020EEE70820ECE70000A41B00200F
:1091C0009404002038B504466846054D04700F220B
:1091D0006946287E03F09DF8002800D02C7738BD22
:1091E0009404002070B50124240321461348FBF7A2
:1091F000FBFB012821D112A005F01AFE0028FAD1AC
:1092000012490120087112480068012815D1F9F7A8
:109210001BFA05252D07012221462846FBF7EDFB09
:10922000FF26F5363046F9F754FD00222146284640
:10923000FBF7E3FB3046F9F74CFD70BD000400502E
:10924000496E204D6F74696F6E0A0D00A4030020F3
:1092500078030020FFB581B001AB07CB00F054F8D4
:1092600007004BD1274C6069F7F73EFC0E46019989
:109270000546C85FF7F7A6FB0B22D243F7F77AFB48
:109280002A463346F7F788FAF7F76AFCFEF786FDB9
:109290002062A069F7F728FC0E4602990546C85FD0
:1092A000F7F790FB0B22D243F7F764FB2A463346CD
:1092B000F7F772FAF7F754FCFEF7AEFD6062E0696B
:1092C000F7F712FC0E4603990546C85FF7F77AFBDD
:1092D0000B22D243F7F74EFB2A463346F7F75CFAE8
:1092E000F7F73EFCFEF7D6FDA0620498216A016004
:1092F0000A98616A01600B98A16A0160384605B05E
:10930000F0BD0000200100207CB515460C46064645
:109310006B4606223B21682000F05CF900280ED144
:109320006946098849BA31806946498849BA218025
:109330006946898849BA29802188494221807CBDB3
:10934000FFB581B01D460646039A029900F034F835
:10935000040029D1305EF7F735FB154E154F324624
:109360003B46F7F727FAF7F7FBFBFEF7D1FD28603E
:109370000299085FF7F726FB32463B46F7F71AFAE1
:10938000F7F7EEFBFEF702FE0A9908600399085F03
:10939000F7F718FB32463B46F7F70CFAF7F7E0FB16
:1093A000FEF732FE0B990860204605B0F0BD0000C4
:1093B000218F2F030A74513F7CB514460D46064693
:1093C0006B4606224321682000F004F900280BD1E7
:1093D0006946098849BA31806946498849BA29806D
:1093E0006946898849BA21807CBD000010B50022F9
:1093F0006B21682000F064F900223721682000F01A
:109400005FF900226B21682000F05AF907226C21D5
:10941000682000F055F909221D21682000F050F95C
:1094200040223821682000F04BF9C02269216820D1
:1094300000F046F917480068012804D0022809D036
:1094400003280ED01FE00C221F21682000F038F9FD
:10945000022214E09F221F21682000F031F9072228
:109460000DE001F02BFD0C480C4C02780C482270EA
:10947000007860701F21682000F022F962781E21B8
:10948000682000F01DF920226B21682000F018F9F7
:1094900010BD0000740300207C0300202001002088
:1094A0008003002070B580226B21682000F008F94D
:1094B0006420F9F70EFC00226B21682000F000F90F
:1094C000032000F0C1F8022000F0B6F8C82000F038
:1094D000DFF800223821682000F0F2F800226A212B
:1094E000682000F0EDF800222321682000F0E8F861
:1094F00000223721682000F0E3F87521682000F091
:1095000049F8712801D0732815D101226B216820F8
:1095100000F0D6F83220F9F7DCFB00226C2168203D
:1095200000F0CEF8C82000F0B3F800210C2000F0C5
:1095300031F8482801D0012070BD01220B210C20F8
:1095400000F0BEF83220F9F7C4FB11220A210C20EA
:1095500000F0B6F80D4C0E4D21462846FEF792FD60
:1095600021462846FEF7F0FD21462846FEF74EFE2E
:1095700021462846FEF7ACFE21462846FEF70AFFA4
:1095800021462846FEF768FF002070BD0000F0412C
:109590000000484370B50D460446FDF74FFE6400D9
:1095A000E0B2FDF717FEFDF78CFE2846FDF712FE30
:1095B000FDF787FEFDF742FE641CE0B2FDF70AFEF0
:1095C000FDF77FFE0020FDF7D5FD0446FDF758FEB0
:1095D000204670BDF8B51D4614460F460646FDF7F9
:1095E0002DFE7600F0B2FDF7F5FDFDF76AFE0028CE
:1095F00003D0FDF745FE0120F8BD3846FDF7EAFD32
:10960000FDF75FFEFDF71AFE761CF0B2FDF7E2FDF6
:10961000FDF757FE08E0012C0CD00120FDF7AAFD54
:10962000641E2870E4B26D1C002CF4D1FDF728FEF6
:109630000020F8BD0020F1E7C00610B5020E1C2185
:10964000682000F03DF810BDC000C01C10B5C2B2CB
:109650001B21682000F034F810BD10B5BC2801D3E0
:10966000012210E0622801D302220CE02A2801D353
:10967000032208E0142801D3042204E00A2801D3BD
:10968000052200E006221A21682000F019F810BD1A
:1096900010B504467D20C000844201D9044602E092
:1096A000042C00D204242146F6F722FD401EC2B24B
:1096B0001921682000F004F86008FFF7CEFF10BD04
:1096C00070B515460E460446FDF7B8FD6006000E5F
:1096D000FDF780FDFDF7F5FD00280BD13046FDF7C5
:1096E00079FDFDF7EEFD2846FDF774FDFDF7E9FD78
:1096F000002803D0FDF7C4FD012070BDFDF7C0FDBB
:10970000002070BDFF220132811A90420CD009DC8A
:1097100008280DD008DC012808D0022806D004282B
:1097200002D105E00F221202072070470520704782
:1097300006207047704700007CB504461F49002092
:109740001F4D08701F4E287030706078002817D1A8
:1097500008F088FC002801D008F072FC607B01282A
:109760000ED1E278E02A07D0237801211648002B99
:1097700007D0012B0AD00FE01449204608F078FCEE
:109780007CBD0078012807D1297005E00078022807
:1097900001D0042800D1317068464271217B0171EB
:1097A000A06800900A48E1890181217C81727038AB
:1097B000406A0169684688477CBD00004303002079
:1097C00041030020420300209A010020641700207A
:1097D0001404002010B50446007800280CD001289D
:1097E00009D16078002806D108F03CFC002802D09E
:1097F000204608F02DFC10BD6078002803D00449F5
:109800000120087010BD0348406A4069804710BDC0
:1098100040030020A4030020704700008307FF22BC
:10982000DB0E9A408907090E994000280BDA0007E1
:10983000000F0838830808489B001818C369934331
:109840000B43C3617047830804489B001B181868CA
:10985000904308431860704700ED00E000E400E02A
:10986000BFF34F8F04490348C860BFF34F8F00BF59
:10987000FDE700000400FA0500ED00E0BFF34F8FA4
:1098800004490348C860BFF34F8F00BFFDE70000E5
:109890000400FA0500ED00E0BFF34F8F04490348D0
:1098A000C860BFF34F8F00BFFDE700000400FA055A
:1098B00000ED00E010B50B4805F078FA0A48017B8E
:1098C000002905D001214175016C042291430164F6
:1098D000407E022805D1044810222230017811432D
:1098E000017010BD701C00209404002010B504A06D
:1098F00005F09EFA0028FAD108F0AAFC10BD00007D
:109900004F6E20436572746966207478206E6578A6
:1099100074207061636B65740D00000010B505491B
:10992000054805F0F9F9044805F008FA0349012053
:10993000087110BD5046000008130020940100205B
:10994000F8B50027944805F031FA944D944C2878E6
:10995000C1067DD5216C4A0604D5402291434908B1
:10996000490021648C490207D4310026002A01DB1A
:10997000C20711D0884AC0325378022B02D04B78EC
:10998000022B09D1236C5B085B002364E673237D03
:109990005371167101279660227B3A437E4F503FE8
:1099A000002A3CD1020702D4C10703D137E00A786C
:1099B000002A06D03978627C914213D9810717D4E6
:1099C00028E0764A921E13788B724978002903D0DA
:1099D00051788B4219D21DE03C202663A071E671BC
:1099E000667412E0800703D4E673A06B401CA0638A
:1099F0006674207A002808D1206B401C2063A0796F
:109A0000401CA071E079401CE071206C40084000CF
:109A1000206404E0EF210840287000F0E3FC28787F
:109A200080071FD55C4AC0321079012803D0207D01
:109A3000E17C884216D966752673207A00280AD1FF
:109A4000206B401C2063A079401CA071E07900E0ED
:109A50003FE0401CE071207D5071206C40084000C8
:109A6000206455E0607D002852D0206CC0064FD4A1
:109A70006675207DE17C884231D208282FD8401CB1
:109A80002075C0070DD0242168460170397B424FF4
:109A90008170703F797841706946207E02F0C1FB89
:109AA000787004F007F9002814D03B480921C03031
:109AB0004170E673216C49084900216426730671E0
:109AC000217D41713449703949788170207A0028AC
:109AD00015D01DE02878EF210840287018E00121FA
:109AE000207E02F0A8FB206C4008400020642A4839
:109AF000E6732673C0300671217D4171E6E7206B65
:109B0000401C2063A079401CA071E079401CE071EA
:109B1000206C810702D502218843206400280ED0E2
:109B20007D21C9001C4805F0F7F81B4805F006F92F
:109B3000287880072ED5607E02281DD01EE0287868
:109B4000C00708D0E06E01681348C0308847287805
:109B50004008400028702878000708D5E06E81682A
:109B60000D48D43088472878F72108402870287895
:109B7000EF2108402870DBE700F0F8FB2878400769
:109B800004D4E06E41680448A83088472878F92159
:109B900008402870F8BD0000DC1B0020B60400203F
:109BA0009404002010B5044805F000F90348002192
:109BB0008175417510BD00008013002094010020C4
:109BC00010B5054805F0F2F801210520002209032F
:109BD0000007FAF712FF10BD6C130020FFB5044612
:109BE000002097B00E4601461190089005460A9055
:109BF000FD480E9010300B90002010901390FB4801
:109C000001711838C2811A9A0274F94A927D42741D
:109C1000C1708170417181600173417381744161D0
:109C20000170F448406B8047F048683805F0BEF892
:109C30002078694608704109701E0190301FEE4F70
:109C400014911290012919D003297DD005297BD0C8
:109C500007297AD038460124F830447000F074FEA9
:109C6000E348C470E248E14A017B1479437E027DF7
:109C7000C07C00296AD0002C69D124E2DC4DA87A8E
:109C8000002808D0D94801241838447000F05CFE40
:109C9000EC701BB0F0BD0198D84B81B2601CAA6D6E
:109CA000FEF7AAFE68460178D44808AB401E017052
:109CB0001298AA6D81B2D148401EFEF735FECF48FA
:109CC000401E80192038417F027F09021143827FA4
:109CD000C07F12040A4300060899104388424FD1FE
:109CE000C148C64C10300090641EBF4BEA8C611C0A
:109CF000A86DFEF73DFE6079217900020843A17945
:109D000009040143E965207AE17900020843617A98
:109D100009040143A07A000608432866E07A410658
:109D2000490F00077970000F3872E875207BB44C3A
:109D30000007000F206101D1012020617D21C900B1
:109D400048434118616103E01FE0A4E1B8E1BCE1D0
:109D50002061E964A864A948113E0C30049068466B
:109D6000067504A9287E01F055FAA0490020143197
:109D700048700120A872A04818304078607071E7E0
:109D80009A480721143041706CE7797B68468173EB
:109D90009648974F18380179684641730D21017331
:109DA000F87E002802D00E206946087303A9387E89
:109DB00002F037FA014630460D3800B2002800DACA
:109DC0000020884207D9894801241838447000F0DF
:109DD000BBFDFC705DE7A178607809020143E07883
:109DE000834A000408432179090601430691126E53
:109DF0000520914219D07E4FFD6A0BE02A688A4205
:109E000007D101211091291D0E9110310B916F6A1C
:109E10000DE0AD6A002DF1D174480B211838417066
:109E200000F092FD0120F87033E771494F6B215C1F
:109E30006A461170401C0D91235C401C205C02029C
:109E40000807000F08300990A0191A432038017F35
:109E50000A9B1943437F1B020B43817FC07F090488
:109E60001943000608430A90D01B80B20122D20396
:109E700008A90F90904212D23F180120009012982A
:109E80000291019781B22046069B0E9AFEF7F0FBE5
:109E900008990A9888421AD10120139017E000B25D
:109EA000012238181204801815900190129801228E
:109EB0000291009281B22046069B0E9AFEF7D8FBD3
:109EC00008990A98884202D10120159F1390152005
:109ED00069460873464803A9007E02F0A2F90F996B
:109EE000884205D841480A2118384170476120E06E
:109EF0001398002877D03D4B0021183B5970109AD9
:109F00009A700D9A3948D206D20F5A719960197316
:109F10005F61374A4170916311741099002910D024
:109F200002221A706A6ABA4209D1002A07D00820B0
:109F3000587000F009FD2E490120C870A9E66F6233
:109F40001FE0149905290FD0294D00226A731A7059
:109F50006A6BBA4213D1002A11D00820587000F061
:109F6000F3FC0120E87094E6214901224A731A703B
:109F7000496BB94203D1002901D0012111911C493B
:109F80004F63017801293DD0194A0021D173099905
:109F9000711A091F002964DD099D09996D1C721B46
:109FA000121F615CD2B20F921E46D970002937D0C1
:109FB0000D98000707D01A980821C3B2681EC2B2D4
:109FC000204600F0DFFC0D480121401E0197009162
:109FD00002906019069B0B9A0F99FFF72FF81198C2
:109FE000002837D047E052E04C1800209C1C00208D
:109FF00094040020D04C01088C1B00206C19002018
:10A000006C1B00200D998906C1D53A490022CA73FC
:10A010000D9A9206D20F02719A7401220A70B6E765
:10A020000D99090705D00121119100210171997441
:10A0300021E0314801210197009102906019069BAF
:10A040000E9A0F99FEF7FAFF1A980021C3B22A4818
:10A050000F9A0EE02848B0600F983073012070739B
:10A0600009E00D98000706D01A980821C3B22046CF
:10A07000099A00F087FC1F49022222310878104318
:10A08000FB221040119A920010430870EAE51B4829
:10A090000C2141704DE7611C3246174809F096F8D3
:10A0A0001648032101700021417013498160019914
:10A0B0000173104802222230017811430170D1E56A
:10A0C000022B02D005E0824203D90C48143804F078
:10A0D0006DFE0848102222300178114301700748B4
:10A0E0000121A83804F018FE0448A83804F026FE20
:10A0F000CFE50000940400206B190020841C002090
:10A1000070B5144C607E022803D01348406B804722
:10A1100001E000F02BF911480E4DA27D01462235D9
:10A1200010261431237B002A05D00622002B00D0F4
:10A1300042704A700AE00522002B00D042704A703B
:10A14000606E04F075FDA16F884202D32878304319
:10A15000287070BD94040020D04C01089C1C002085
:10A1600070B5164C607E022803D01548406B8047BE
:10A1700001E000F0FBF81348104DA27D01462235A6
:10A1800010261431237B002A08D00422002B00D093
:10A1900042704A70607E02280BD170BD0322002BF2
:10A1A00000D042704A70606E04F042FDA16F884298
:10A1B000F3D328783043287070BD00009404002049
:10A1C000D04C01089C1C0020FEB504F02BFD364C41
:10A1D0000646607E022803D03448406B804701E089
:10A1E00000F0C4F8304D607A2235002700282AD0CC
:10A1F0002F48616F04F090FD2D4804F09FFD607EB4
:10A2000002280ED02A48A16F143004F085FD28489A
:10A21000143004F093FD607E022802D0207B0028D9
:10A2200020D016206946087202A9207E01F0F9FFAD
:10A23000A16F41181E48503004F06EFD1C4850308C
:10A2400004F07CFD0EE01A4804217C304770143085
:10A2500041702878002801D101202870C0B2102157
:10A26000084328702878000704D5114890300078FA
:10A27000002815D0E777607FA07769460870A07A3C
:10A2800048700196207E02F020F86666207B002848
:10A2900005D107487C304770607C401C6074FEBD6F
:10A2A0000120E077E7E7000094040020D04C01088B
:10A2B000201C002010B50B48407E022803D00A481D
:10A2C000406B804701E000F051F8084902204870D7
:10A2D0001431487003481022223001781143017074
:10A2E00010BD000094040020D04C01089C1C0020EC
:10A2F00070B5194804F05AFD184D0021164CA97587
:10A30000687F283420702046BC384278E270407B59
:10A310002074E87E6074A1741148E17401781148DA
:10A32000002905D00078A060687E022803D005E0EF
:10A33000217A0170F8E70C48806B8047064A287E36
:10A3400068321146403901F0ACFF0348B438C168A7
:10A35000A07C02F077F870BD201C0020940400203F
:10A360005E0300205D030020D04C010870B5194841
:10A3700004F01CFD174D184C2835607F2E462870C0
:10A38000F03E706A68602846D038407B2874E07ED2
:10A39000687401201149E8740A781149002A16D01E
:10A3A0000978A960617E022900D00020094AA874BA
:10A3B000543211462C39207E01F073FF002805D05D
:10A3C000A87CF16802F03EF8E87CA07570BD2A7A9E
:10A3D0000A70E7E7341C002094040020600300208A
:10A3E0005F0300201FB51A4804F0E0FC194C10214F
:10A3F000206C88432064204622300078000723D553
:10A400001348A430007800281ED101F08DFF2046AB
:10A41000203000786946401C888103A9207E00F026
:10A42000F0FE0B49A0394870002069460871E17AB6
:10A430000246C9010A4369460A7203460246009071
:10A4400002A901A800F040F903F034FC1FBD000090
:10A450000C1C00209404002010B57F210A48C90577
:10A46000816300210162816208F012FB022801D0A1
:10A4700008F0D6FD0548816A054804F04DFC044803
:10A4800004F05CFC10BD0000800700209401002057
:10A49000E012002010B5144CA078002818D0012834
:10A4A00015D11249124804F0CFFB1148A16A04F0FB
:10A4B00033FCFFF7D1FF08F0B3FD7F210D48C9053C
:10A4C0008163002101628162A078401CA07010BDF0
:10A4D0000748FF21F531143004F01EFC0448143005
:10A4E00004F02CFCF0E700009401002059A40008BF
:10A4F000E01200208007002009480178094801295E
:10A5000007D0022907D0032908D0042905D106A1C4
:10A5100002E00BA100E010A14161704714A1FBE72C
:10A5200061030020F400002024504D544B33353398
:10A530002C312C312C312C302C302A32410D0A0098
:10A5400024504D544B3335332C312C312C302C309E
:10A550002C302A32420D0A0024504D544B333533EF
:10A560002C312C302C302C302C312A32420D0A0068
:10A5700024504D544B3335332C312C302C312C306E
:10A580002C302A32420D0A000B4801780B48012971
:10A5900009D0022909D003290AD004290AD00529A3
:10A5A00005D107A102E00AA100E00DA18161704779
:10A5B0000FA1FBE712A1F9E762030020F4000020DD
:10A5C00024504D544B3838362C342A32430D0A006F
:10A5D00024504D544B3838362C302A32380D0A006E
:10A5E00024504D544B3838362C312A32390D0A005C
:10A5F00024504D544B3838362C322A32410D0A0043
:10A6000024504D544B3838362C332A32420D0A0030
:10A6100010B5F8F72BFF012220210F48FAF7EDF9CA
:10A620000E480078012816D80D480E4900780978A0
:10A63000084310D00C4C207800280CD109F072FC93
:10A640000A480178491CC9B201701E2903D10121B1
:10A6500021700021017010BD00040050A9030020EA
:10A660006103002062030020A0010020F40000200C
:10A67000F0B5064600242046002E01D0002A1ED147
:10A680000020F0BD355DAF1E3B0004F0B2FF09169F
:10A6900014160612140E16061600641C1554E4B2A5
:10A6A000401CC0B2335D135400E01554401CC0B2CE
:10A6B00003E0A41C00E0641CE4B2641CE4B28C421D
:10A6C000E0D3F0BD70470000F0B50C4687B084467B
:10A6D000002198480C9D069181841E1E1746017327
:10A6E00000D10025EAB242716146934D0978297084
:10A6F0000121009161460978490908D002293FD01B
:10A7000004293BD007297DD0022007B0F0BD009975
:10A7100004468184681C0822616D08F062FDA08CEB
:10A720000822083080B2A0842818216D08F059FD55
:10A73000A08C0830A0848148C06980470146E0842D
:10A74000A08C06AB2954401C80B2090A2954401C35
:10A75000A084C1B27848A26DFEF7E6F8A08C0699F5
:10A760002954401C80B20A0A2A54401C80B20A0CA8
:10A770002A54401C80B2090E2954D7E001210173EC
:10A78000817A002969D0012269460A7321786948D3
:10A79000CA0969464A736A4A806B04905078087502
:10A7A0001078487510462030007B88756148134644
:10A7B00038300090383803A9007E521C00F012FD9A
:10A7C00081012078BF22104008435A492070497BFC
:10A7D000002905D0574A00215173202108432070D9
:10A7E0005448016E54480A0A417082700A0CC270C3
:10A7F000090E0171217841714E49098E8171090A52
:10A80000C17100E088E04B49FF30C97BFF30401840
:10A81000484908250A7C4A49823908F0D7FC45484E
:10A82000C17B007C0818C1B24248002EC1731FD002
:10A830004279002A1CD0827B002A22D00F291DD801
:10A8400020783D4A030940181B010007000F03430D
:10A850002370537100203B4C07E0072055E7235C31
:10A8600053556D1C401CEDB280B28842F7D308E00E
:10A870003048002905D0827B002A02D0314E417138
:10A8800000272C4C00202F4AA07380322D48FFF760
:10A89000EFFE2074002801D00120A073002E14D0F8
:10A8A0006179002911D0244847556D1CEDB2002F65
:10A8B00027D0236B002240190092019302901E4A78
:10A8C000236E103A3046FEF7C1FB607906AB2918BB
:10A8D000A18400206E46226B0DC6174A1648203A06
:10A8E000236EFDF7C5FE144AA18C06985054030A46
:10A8F00052185370030C000E9370D070091DA18480
:10A9000016E00022E273236B401900920A4A019379
:10A910000290203A236ED5E7002B09D00446002A86
:10A9200006D0681C314608F051FC6079401CA084B8
:10A930000020EAE6940400206C180020D04C0108A6
:10A940006C1B00206A1A002010B50C484022016CD4
:10A9500011430164007B002801D0FEF7ABFF0749DB
:10A96000122222310878104308700121044804F0B3
:10A97000D3F9034804F0E2F910BD0000940400206C
:10A98000DC1B0020FFB505468DB000200A90E04892
:10A9900016460C46099092E1285D641C801EE4B2C4
:10A9A000030004F026FE090614B7C5FEFDFCFBFA01
:10A9B000F900D84901200870D74900204870285D67
:10A9C0000872641CE0B22A5C4A72401CA0E00020BD
:10A9D000694608730877087208A908700A98002861
:10A9E000D9D101200A902819401E311B04906846D5
:10A9F000491CCA4F0175F97A8175099807AB017B2B
:10AA000068464175C24920394A78C275097801768D
:10AA1000099803AA01786846417608A902A801911D
:10AA2000009004A9387E01F013FC0B90C04340074E
:10AA30005AD1B84901200870B5486946097B2038C9
:10AA400041706946097F017069460998097A017069
:10AA5000B3A004F0EDF90028FAD1B248007800283C
:10AA600038D0B1A004F0E4F90028FAD138790128EF
:10AA700001D100203871787800280ED068460C216A
:10AA80004156ADA004F0D4F90028F7D1A4A004F0F9
:10AA9000CFF90028FAD1787026E068460C2141569B
:10AAA000B4A004F0C5F90028F7D168461C2141562E
:10AAB000B7A004F0BDF90028F7D16846017ABAA022
:10AAC00004F0B6F90028F8D195A004F0B1F90028F7
:10AAD000FAD109E0BAA004F0ABF90028FAD190A0AD
:10AAE00004F0A6F90028FAD1002706E0002203208E
:10AAF0000B99F7F71FFD7F1CFFB208A8052100780E
:10AB0000F5F7F6FAB842F1D808A800782018401EE8
:10AB1000C4B2D4E07F4901200870295D7F4A641CDB
:10AB20009174884010850022E4B211460420C4E0EC
:10AB3000285D4006410F68464170285D641C01078E
:10AB4000090F68460170E0B2295C401CC0B2019157
:10AB50002A5C401C12021143C0B201912A5C401CC5
:10AB600012041143C4B208466421484301906B4863
:10AB70006946007E01F0A0FB0146C843400715D19D
:10AB8000644A012010706846027809980272604891
:10AB9000019A2038426205E094E095E05DE043E0F0
:10ABA00017E006E0684642780998427000220520C6
:10ABB00083E05849012008705848FE21006F0028A2
:10ABC00004D00068002801D0804701460620109A72
:10ABD00073E0504901200870285D69460874641CC0
:10ABE000E0B20391295C401CC0B200912A5C401C79
:10ABF00012021143C0B200912A5C401C120411439E
:10AC000064225143009100210191C0B22A5C401C92
:10AC10006946C4B20A72414803A9007E01F029FBCB
:10AC200000220146072048E03A4901200870285DCB
:10AC3000641C0007000FE4B2002800D101207D2130
:10AC4000C900484332497D222039D200086180186A
:10AC500000224861114608202FE0285D00216A4645
:10AC6000641C11705170E4B2810601D5012151704C
:10AC7000C10601D5012111700007000F907027480F
:10AC80001146007E01F03CFB401C18D021490120F8
:10AC900008706846017809980173684641780998F8
:10ACA0004173684680784C49085CF5F784FE184982
:10ACB00000222039086311460920F7F73BFCB44213
:10ACC00000D269E611B0F0BD124901200870285D7C
:10ACD00069460870641CE0B2295C401CC0B2019156
:10ACE0002A5C401C12021143C0B201912A5C401C34
:10ACF00012041143C4B20846642148430190074836
:10AD00006946007E00F0D6FC002201460A20D4E706
:10AD10008C1B002044030020B01C00209404002061
:10AD20000D0A00005C030020414452204D657373FE
:10AD30006167653A0D0A00005458204461746172DD
:10AD400061746520746F6F20736D616C6C20666F29
:10AD5000722074686973207061796C6F616420730C
:10AD6000697A652C206368616E676520746F2025A1
:10AD7000640D0A0054582044617461726174652046
:10AD80006368616E676520746F2025640D0A00009A
:10AD90005478506F776572206368616E67652074C0
:10ADA0006F2025640D0A00004E62526570206368B2
:10ADB000616E676520746F2025640D0A0000000035
:10ADC00052656365697665643A20414452204D6559
:10ADD00073736167650D0A00B053010870B51749B8
:10ADE0000023CA681206120F18D18A6B154CD500C1
:10ADF000134A02D51268224009E08E6B01252D0707
:10AE00002E438E6312688E6B2240AE438E63A24245
:10AE100004D103218903884200D101230A48016833
:10AE200049084900194301600068C007C00F9842F3
:10AE300001D0012070BD002070BD00000010024054
:10AE400000700040001800000020024010B509F01A
:10AE500017FE10BD01090A2200075143000F4018D8
:10AE6000C0B27047002102E00A38C0B2491C0A286B
:10AE7000FAD20907090E0843704770B50446006806
:10AE8000C168490613D40021C943C160F9F7BCFD6C
:10AE90007D260546F60006E0F9F7B6FD401BB042F8
:10AEA00001D9032070BD2068C0684006F4D5002099
:10AEB00070BD10B5FBF71AFF10BD0000F0B5B1B0C2
:10AEC000AD4D002420AE2846F8F7FCF8A100641C24
:10AED0002D1D7050112CF6DB0025A84C0095019516
:10AEE000A11C0820219B209A08F087FE2298E06090
:10AEF0002699259801910090214618311020249B15
:10AF0000239A08F07AFE29982A9901910090214607
:10AF100028311020289B279A08F06FFE2E992D9833
:10AF2000019100902146383110202C9B2B9A08F07B
:10AF300064FE21460095019510310820309B2F9A20
:10AF400008F05BFE8E4F00263846F8F7BBF8B200DB
:10AF500005A9761C3F1D88501B2EF5DB0220694693
:10AF600008720598000E01D0012100E0002168461A
:10AF7000017302A8FDF772FE16216846017205985A
:10AF800001146846017302A8FDF768FE05987B4E20
:10AF900000124036307505980127C0B201287DD0D7
:10AFA00065706078012800D00020FEF70BF90720BB
:10AFB000694608720698000E00D00120087302A8A6
:10AFC000FDF74CFE06980002000E012867D02570A0
:10AFD000684605720698010A6846017302A8FDF7E3
:10AFE0003DFE0698C0B201287ED035730A27684618
:10AFF00007720798039002A8FDF730FE5F4D303DC1
:10B000002878002871D020780028FBD06846077285
:10B010005C4801786846017402A8FDF71FFE297894
:10B02000102000297ED0217800297BD06946087243
:10B0300055480068039002A8FDF710FE29781120FA
:10B04000002970D0217800296DD0694608724F48D8
:10B050000068039002A8FDF701FE12216846017204
:10B060000B98039002A8FDF7F9FD132168460172C1
:10B070000C98039002A8FDF7F1FD032168460172C8
:10B080000D98039002A8FDF7E9FD41490E9808606C
:10B090000F984049000A08700F9801E058E059E005
:10B0A000F072364810990838016011993A4A090C33
:10B0B00011801199394A090A117011990171139C73
:10B0C0003B4E240E6C72139C3548240CAC72139CBE
:10B0D0003480384E149C3460374E159C34603149AE
:10B0E000314A324B354E01E036E037E0169C346091
:10B0F000334E179C3460334E189C3460324E199C8A
:10B100003460324E1A9C3460314E1B9C3460314E98
:10B110001C9C34601D9C240E04701D98000C08704B
:10B120001D9801E020E023E0000A10701D981870BF
:10B130001E98F5F740FC2849F5F740FAA8611E98DB
:10B140002649000A087026491F98087031B0F0BDE2
:10B15000677026E727703BE7377347E769460F724A
:10B1600008980874E87257E769460872099861E719
:10B17000694608720A986CE700910108D403002020
:10B1800000900108AB040020DC040020E004002053
:10B19000C001002064030020460300209A01002023
:10B1A0005D0300205E0300205F0300206003002099
:10B1B000940300206C03002068030020700300202B
:10B1C00074030020780300207C030020800300200B
:10B1D000C4010020C80100200000C8426203002012
:10B1E0006103002070B51C46049B15460E460528D9
:10B1F00001D0002070BD22462946304600F064FA96
:10B2000070BD10B5052801D0002010BD084600F023
:10B2100097FA10BD10B5052802D1084600F0A7FA2C
:10B2200010BD70B514460D46052801D0D0B270BDD2
:10B230001A462146284600F0D4FA70BD10B50528FC
:10B2400002D1084600F0D4FA10BD10B5052801D08F
:10B25000002010BD084600F0E7FA10BD30B50246E8
:10B260000168C07A0C2358430930095C50680B010F
:10B27000C45A00250C33C550507A002809D0907A62
:10B28000012805D1106901466143081A5168C85068
:10B2900030BDD06800F024F9844200D92046917A6C
:10B2A000002902D1117A002903D011694843401ABC
:10B2B000ECE75068C55030BD10B50B0914099C422D
:10B2C00001D3914201D3002010BD5A000C07835ACC
:10B2D000240F0121A1408B438352012010BD30B5C2
:10B2E00000280AD0002908D0002304E05C000D5B90
:10B2F0005B1C0553DBB29342F8D330BDFFB50E465D
:10B300001946099A029800F0C0F9002824D00024B8
:10B3100025461DE000236F00F15B012098400142AB
:10B320000ED0E0180C2148430A994018007A010613
:10B330000A0F0107090F029800F0A7F901280BD0A6
:10B340005B1CDBB2102BE7D310346D1CE4B2EDB202
:10B3500000988442DED3002004B0F0BDFEB505465F
:10B3600014460E465800F5F741FB009060000F466A
:10B370000838F5F727FB2A463346F5F71BFA3B4614
:10B38000009AF5F765F92A463346F5F77BFA06F099
:10B39000F3FDF5F78BFBA04200D904460998046041
:10B3A0000898F5F723FB009001912046F5F71EFB66
:10B3B0002A463346F5F7FEF90022D243F5F7DAFACA
:10B3C0000C460746022228463146F5F7D3FA3A469C
:10B3D0002346F5F7E1F9019B009AF5F7DDF906F050
:10B3E000CBFDF5F73FFB0A990860FEBD10B5F5F7F8
:10B3F000FDFA02460B4600200149F5F743FA10BD5D
:10B400000000204070B506460846F5F7EFFA0546FD
:10B4100001200C46B040F5F7D5FA2A462346F5F749
:10B4200031FA0022014BF5F7C5F970BD00408F409D
:10B4300070B50C460146283915460B0004F0D9F8C2
:10B440000B07090B0D0F11131517191B1D000A20EF
:10B4500070BD0B2070BD0C2070BD0D2070BD0E2086
:10B4600070BD0F2070BD102070BD112070BD122066
:10B4700070BD132070BD142070BD4000F5F79BFA1D
:10B480002146F5F75AF82946F5F753F8F5F72CFB5E
:10B4900007F04CF9F5F7E6FA40B270BDF0B5844616
:10B4A000964600206246002A01D0012215E00020C5
:10B4B000F0BD4C0063461F5B102600242346154652
:10B4C0009D40BD4301D1641CE4B25B1CDBB2B342BE
:10B4D000F5D32018491CC0B2C9B27145E9D3F0BDFB
:10B4E0000249884200D302496420704780EE36004A
:10B4F000803F5C02FFB504460678022083B02056E8
:10B5000002900325042761786557E75700290BD17E
:10B510000F2801D10F2D02D000260727E75705205D
:10B520002056062502906557002E25D01120205662
:10B530006169019100901023E356207AE168029A34
:10B54000FFF7DCFE002801D1FD200640182219215A
:10B55000A2566156284600F098F8002807D1192015
:10B560002056A84201DD054601E0FB200640072EDB
:10B5700002D1002F00D1A7570499029808700598AE
:10B58000057006980770304607B0F0BD03780022BA
:10B59000032B14D1427813071B0F12068B70120F66
:10B5A0004A7082788A80C3781B021A438A800079A5
:10B5B0004206520F0007CA70000F0870052210469D
:10B5C000704700288A6000D14A607047FFB50024A8
:10B5D000E44381B01F46002552E0019800280FD0B7
:10B5E0000298002844D0039829010E18B06803F08F
:10B5F0001FFB0146F06881422BD30020F0603DE044
:10B600000398290108180090406803F011FB0646D2
:10B610000298002803D00098806803F009FB864256
:10B6200002D90098406804E00298002803D00098EE
:10B63000806803F0FDFA0099C968814202D80020B1
:10B6400000991AE0002919D0081AA04216D204461F
:10B6500014E0002812D0B06803F0EAFAF168081A82
:10B66000A0420BD2B06803F0E3FAF1680C1A05E0CF
:10B67000002403992A0120465118C8606D1CEDB2C0
:10B68000BD42AAD3204605B0F0BD884203DB9042FC
:10B6900001DC012070470020704770B51C46049BF8
:10B6A00015460E46052804D122462946304600F0AC
:10B6B00057F970BD10B5052801D0002010BD08460F
:10B6C00000F080F910BD0000FFB504460F460820C9
:10B6D000092681B02056A657616819606178002557
:10B6E000012925D100280BD06168402901D301250B
:10B6F000002660291CD3C906C90E012903D017E012
:10B700000021196014E0242269460A704870A07A6A
:10B710008870684600F074F940B2002808D121789A
:10B720000025012904D1054907230A881A430A8004
:10B73000387003980670284605B0F0BD300400202C
:10B74000014609880020032901D8052070470629F1
:10B7500001D804207047092901D8032070470C291B
:10B7600001D8022070470F29FCD801207047F0B59E
:10B7700087B00746502069460872387910282ED1C4
:10B7800000240325264601E0082D19D23868611CE3
:10B79000005D00903A68515C0902084300903A68E5
:10B7A000A11C515C019609040843642148430090A0
:10B7B0000AD068460390057403A800F04BF808E02F
:10B7C00068460096067201966846057505A800F061
:10B7D000AFF8E41C6D1CEDB2E4B2102DD4D307B069
:10B7E000F0BD881A40B2002800DA0020C0B27047CD
:10B7F00000B585B00A4900910A490191427869462D
:10B800000A7202784A7282788A72C278CA72416871
:10B810000391806804906846FFF720FD05B000BDE5
:10B820008C1700203404002010B50179002903D0C2
:10B83000012905D0002010BD01680122044803E061
:10B84000016803480122801CFFF749FD012010BD5B
:10B8500030040020F8B505460020694608702E79AE
:10B8600004460746102E01D30320F8BD286807229E
:10B87000007A002100070017FFF707FF002800D11A
:10B880000124286808214156072208110021FFF7EA
:10B89000FCFE002800D10124296808200856010771
:10B8A00009170211914200DD0124032E12D2002952
:10B8B00000DD0124001107220521FFF7E6FE002824
:10B8C00000D101242868184902680C2070430858E8
:10B8D00082420AD128686946006803F0F3FD002817
:10B8E00003D03C4203D00620F8BD0127F9E7002C25
:10B8F00001D00520F8BD002F01D00420F8BD0C2098
:10B900003146414308482B6808180ECB0EC06946E3
:10B9100009780C384172054801220188B240114370
:10B9200001800020F8BD00008C17002030040020AA
:10B9300010B50178032901D2002010BD0C22064B5E
:10B940004A430020D21810605060906010220348D3
:10B95000FFF7B2FC10BD00008C170020300400205F
:10B96000FFB583B01C461646072800DB0720607031
:10B97000F8F7BEF9A07001202056104A072819D008
:10B980008100134618335958105CFFF73BFD0546FC
:10B990000B480F46406E804721460C310834029117
:10B9A00000903346019428463946049AFFF7D6FCA6
:10B9B00007B0F0BD105CFFF719FDE8E7245301085C
:10B9C000D04C010838B505460020694608700324AC
:10B9D000686803F077FD002800D1022429780C2044
:10B9E000414306484258002A01D1FD221440032C4D
:10B9F00002D108186A684260204638BD8C170020C2
:10BA000070B5024615787D21C90000204C002B003E
:10BA100003F0EFFD251C1C1C1C1C1C1C1C1C1C1CEE
:10BA20001C1C1D2127292B2D2F3133361C3B3D4259
:10BA30004447491C1C4B4E5050141C00012010560A
:10BA40000021002801D0401EC1B248B270BD0120C3
:10BA50001056194903E00120174910560831085CB7
:10BA600070BD012070BD154870BD084670BD2046F0
:10BA700070BD134870BD134870BD0120800370BDB8
:10BA8000114808F0AFF8001970BD104870BD10499A
:10BA900009780029FAD0E8E70E4870BD0D48801CEF
:10BAA00070BD102070BD0C4870BD8320C00570BDF6
:10BAB0000A4870BD122070BD2C530108B80B00005D
:10BAC000881300007017000018FCFFFF08E6D3334E
:10BAD000AF030020300400208C1700209A99094001
:10BAE00070B5044606F0CAFD19491A4A1A4B002CD3
:10BAF00012D0012C0FD1981E04881B8868311C437A
:10BB000004800BC90BC2124874300BC80BC2104B17
:10BB100080330BCB0BC270BD00280BD00C6E496E6E
:10BB2000916011C201200C4918800122881EFFF784
:10BB3000D6FB70BD0846383031C831C208464430A3
:10BB400031C831C2503113C913C20720EBE70000DE
:10BB5000245301088C17002032040020FFB507256C
:10BB60008FB0044600266846374606803BE02068D2
:10BB700002A98019FFF70AFD002837D03018C6B295
:10BB8000694688890880C97A0725084304D0481E79
:10BB9000042801D9072901D3062524E0002006291D
:10BBA0000DD06B4601221B8882401A4217D00C220E
:10BBB00003465343374AD258002A0ED00FE00C22D6
:10BBC000344B42439A58002A09D06B4601221B8805
:10BBD00082401A436B461A8001E06D086D00401CDC
:10BBE000C0B21028DBD32079B042C0D80221684609
:10BBF00001716179817101A8FFF702FF0146684672
:10BC00000574A2794274427A8274827AC274027A8A
:10BC10000275E2794275227A8275627AC2751022C3
:10BC20000276079008A80170072141701948099011
:10BC300008A8017202AB47729A1C511E04A8FFF7B4
:10BC400059FC072803D114496A4612880A806A46BB
:10BC500009215156002903D0012901D0022908D118
:10BC60000E490978332904D3032151720C4A01216A
:10BC7000117069464A7A10990A7069468A7A119950
:10BC80000A7069460A7A12990A7018990E7013B0F0
:10BC9000F0BD00008C170020300400209F01002020
:10BCA000950400203EB5016803240A68002A0DD0DF
:10BCB00000910079694608716846FFF7CBFD0028BE
:10BCC00012D004280BD005280DD10AE0007969466E
:10BCD000087202A8FFF72CFE002804D004E002241A
:10BCE00002E0012400E0002420463EBDFFB589B0FB
:10BCF000044600256846057316461F4604950595BB
:10BD000006950122294625480795FFF7C7FB00281D
:10BD100004D122480722018811430180606802F0A3
:10BD200087FF2168884220D33D601C4AA17A607A4F
:10BD30000623121DFFF74AFC0746184803AA04A968
:10BD4000001D6B4607C3217A607A154B134AF6F73C
:10BD500013FF002812D0411E002007F043FF04A962
:10BD6000095C0A98017035600DE06946087B401C4B
:10BD70000873606802F05CFF21680F1A6846007B58
:10BD8000002803D0376001200DB0F0BD0348072222
:10BD900001881143018000203560F5E73004002060
:10BDA0008C170020F3B501254A4F044645574668D5
:10BDB000F8688DB08047002802D000200FB0F0BD99
:10BDC000E07C002809D121780C20414342484658A4
:10BDD00008184068002800D00646404840570A909E
:10BDE0003C484169304688473D4900200A88012A7D
:10BDF00002D10C220A9208800121072D36D001229F
:10BE00000B92A27C07AB069007C32189059089B2EB
:10BE10000291082100900390049001912D48012384
:10BE2000076AA17818460A9AB847607C012837D07B
:10BE30002A480830405D0D30C1B22648C26D0B98CB
:10BE400090472848007800282DD002F0EBFE0446E9
:10BE5000214625A002F0ECFF0028F9D12A46314600
:10BE600023A002F0E5FF0028F8D12FE000220B927A
:10BE7000A27C06900790099208902289059192B2BF
:10BE800002920521214A009201917D210A9AC9005E
:10BE90004A431049039004900F6A00231C49C3E7EA
:10BEA0000E481030C6E71B493046F4F721F986B238
:10BEB00008467D21C900F4F71BF984B22B462246BF
:10BEC000314615A002F0B4FF0028F7D10E98057096
:10BED000012073E7D04C01088C170020245301087F
:10BEE0002C0400205C0300205B256C755D000000C5
:10BEF0005258206F6E206672657120256420487A42
:10BF00002061742044522025640D0A0085450100FB
:10BF100050C3000040420F005258206F6E206672DE
:10BF200065712025642E2564204D487A2061742097
:10BF300044522025640D0A0070B50F490546896AF0
:10BF4000072440688847002800D10624002028568E
:10BF500007220021FFF799FB002801D1FD200440B2
:10BF60000120285605220021FFF78FFB002801D170
:10BF7000FB200440204670BDD04C010810B501786C
:10BF80000C235943054B4268C918497A044B0901EF
:10BF9000C9184078FFF715FB10BD00008C17002072
:10BFA0003404002070B502220446825601780C2029
:10BFB0000B4B4143C818407A0A4D00014519022035
:10BFC0002856824200DD10465D58A2686168FFF77E
:10BFD0002FFA01460448A289436C2846984770BD51
:10BFE0008C17002034040020D04C0108F7B5012143
:10BFF000044641565C480C23475620785B4E584314
:10C000008019407A5A4B0001C31802220220A2561E
:10C0100018568EB0824200DD10460A900846F7F7A7
:10C0200067FE0C90A26861680A98FFF701FA0D900C
:10C0300020780C2148434F493058496988474E4879
:10C040000088012802D114200C270D90627801206D
:10C050004A490025072A2DD001220891099208217A
:10C0600005950695079501AB23C3424900970490B7
:10C070004F6A00220C9B0D99B84741480078002870
:10C080003AD002F0CFFD074639463EA002F0D0FE7E
:10C090000028F9D1384F3888012821D020780C2188
:10C0A000484301223158A25638A002F0C1FE0028B0
:10C0B000F4D13DE0002208910992052104907D20F1
:10C0C0000795C000029147430595069503952948B9
:10C0D00001950097476A344A28460C9B0D99CBE797
:10C0E00020780C2148433158002228A002F0A0FEFD
:10C0F0000028F5D13D801BE020780C2148433058C2
:10C100002A49F3F7F5FF80B2019008467D21C90066
:10C11000F3F7EEFF184E87B23088012819D00123BB
:10C12000E3563A4622A0019902F082FE0028F6D199
:10C13000104D217BEA6D09989047EA6A217B0998A6
:10C140009047109908600F990A980870012011B063
:10C15000F0BD00233A4616A0019902F069FE0028BE
:10C16000F7D13580E4E70000245301088C17002044
:10C1700034040020D04C01082C040020B80B00002F
:10C180005C0300205B256C755D0000005458206F37
:10C190006E206672657120256420487A20617420C3
:10C1A00044522025640D0A00A861000040420F009F
:10C1B0005458206F6E20667265712025642E2564A8
:10C1C000204D487A2061742044522025640D0A00D5
:10C1D0000020C043704710B509290ED006DC0529A0
:10C1E0000BD006290DD0072919D106E00A2904D061
:10C1F0000F290FD0222912D10EE00023C3560722A7
:10C2000002E00023C356052200211846FFF73DFA3D
:10C21000002800D0012010BD00781228FAD200209A
:10C2200010BD10B50022052801D0104610BD0846EB
:10C23000FFF7E6FB10BD10B5052802D10846FFF751
:10C240004FFC10BD052801D0002070470120704729
:10C25000F8B51C460E46069B07991546052801D0E1
:10C260000020F8BD0091224629463046FFF776FCB3
:10C27000F8BD10B5052801D0002010BD0846FFF715
:10C2800011FD10BD70B51C46049B15460E460528D1
:10C2900001D0002070BD224629463046FFF726FD1A
:10C2A00070BD10B50B46052801D0002010BD114609
:10C2B0001846FFF777FD10BD10B5052801D0002006
:10C2C00010BD0846FFF738FE10BD10B5052802D195
:10C2D0000846FFF753FE10BD10B5052802D10846E9
:10C2E000FFF760FE10BD70B514460D46052801D05D
:10C2F000002070BD1A4621462846FFF777FE70BD24
:10C3000010B5052801D0002010BD0846FFF760FFDA
:10C3100010BD10B50B46052801D0002010BD1146F8
:10C320001846FFF758FF10BDF0B51F480021817275
:10C33000016341633C2281638271C17141740122B6
:10C34000C2740275417581740285C17301744272B1
:10C35000164A13461478383B1C7054785C701446A7
:10C360002034657820335D701546583D2E4637469B
:10C370007C37F66F7F68AF646E64257B1D73647BCA
:10C380005C73203B146B1C63536B383A536301732B
:10C3900041738173C26A01E05162926A002AFBD143
:10C3A00041778177F0BD000094040020A41B002099
:10C3B00070B5092000F003FE0546062000F0FFFDE1
:10C3C0000404072000F0FBFD00020443082000F0F5
:10C3D000F6FD0443200A0102184A611A51438031D4
:10C3E0005043090A46180021092001F035FC3B2082
:10C3F00000F0E5FD4024204301463B2001F02CFCE9
:10C400003B2000F0DCFD8006FAD40D4800F0FAFE77
:10C410003B2000F0D4FD204301463B2001F01CFCF2
:10C420003B2000F0CCFD8006FAD42946092001F01B
:10C4300013FC304600F0E6FE70BD0000093D000030
:10C4400000A1BC330200044802D0C16B00200847A1
:10C45000C26B084610470000D04C010808B50B48D5
:10C46000C16A01221143C162C06A002110400090DC
:10C470000748416081600321C1609102016001466B
:10C4800005200007F8F7EEF908BD00000010024093
:10C490005807002008B50B48C26A01210A43C2624E
:10C4A000C06A084000900848416000218160032173
:10C4B000C160012189020160014605200007F8F7EB
:10C4C000D1F908BD001002406C070020F8B51D46E8
:10C4D00016460F460446F8F797FA31462646403688
:10C4E000009000291ED043E0681C1BD0002D05D011
:10C4F000F8F78AFA0099401AA84213D920684168CF
:10C50000E022914341602068026840218A43026032
:10C5100023E021680A6882430A6021680A680243AE
:10C520000A601FE02068816838468843DCD124E037
:10C53000681C1DD0002D06D0F8F766FA0146009859
:10C54000081AA84214D920684268E0218A43426050
:10C55000206801684022914301600120A16A4003E4
:10C560008142D6D001207074002030740320F8BDC1
:10C570002068816838468843DAD00020F8BD7047CB
:10C5800001494860704700001400002001207047F6
:10C59000014980207047000040DD4A1F10B5034864
:10C5A000406840688047801C10BD000014000020D7
:10C5B0000148007970470000A0060020F3B502464C
:10C5C00000206D498BB0002A0BD0012A7ED10024B7
:10C5D000486C2546072854D0082855D0092858D13A
:10C5E00055E06548C069F4F701FA074600910C98D8
:10C5F000F4F7FCF906900E46302000F0E0FC40070E
:10C60000800F02D000245D4D01E000242546272044
:10C6100000F0D5FC58494007400F098C401C4018D9
:10C62000F4F7E4F9544A203209929278012A21D091
:10C630000022524BF4F70CF822462B46F4F708F888
:10C640003346069AF4F704F8099A1279012A14D0AD
:10C6500000221346F3F7FCFF0322F4F78BF93A4666
:10C66000009BF4F70FF90022454BF4F7A3F807F00D
:10C670000FFB7DE000221346DCE7002201239B072D
:10C68000E8E700243F4D04E000243F4D01E03F4D2A
:10C6900000248F6C0120B840F4F794F902460B4651
:10C6A00020462946F4F7EEF802460B4600203349AF
:10C6B000F4F7E8F8304E044640360D46F089F4F7BA
:10C6C00095F90022324BF3F7C3FF00E052E0224617
:10C6D0002B46F4F76FF807910890707B001DF4F774
:10C6E00085F905910690307B002800D00220381A89
:10C6F0008000F4F77BF904900C980391C000B90016
:10C70000401AB17C09014018317C002900D0142165
:10C71000401A1C30F4F76AF9039B049AF4F7B2F854
:10C7200005F02AFC059B069AF4F744F80022074618
:10C730000E461346F4F700FA02D23846314601E0BD
:10C74000002001460022134BF3F782FF22462B46BE
:10C75000F4F730F8079B089AF3F77AFF0022084BAA
:10C76000F4F728F80C4A0D4BF3F772FF05F0DEFFE3
:10C77000F4F79CF90DB0F0BDA00600200000F03FDA
:10C7800000408F408084FE4080840E4180841E41A2
:10C7900000001140000020402B8716D9CEF7EF3F54
:10C7A00000207047F8B51E4D1E4928601E4802F053
:10C7B0004BFA1D481B49143002F046FA1A48194931
:10C7C000283002F041FA686801680120884700F0CB
:10C7D00049FCFFF7EDFD002000F08CFD68688168E2
:10C7E000284608308847114E002460002718F05D65
:10C7F00000F048FDB8198178407801F02DFA641CEA
:10C80000E4B2102CF1D3002000F03CFD06490020DA
:10C8100068390871686840688047801CF8BD00006E
:10C8200014000020B9CE000808070020F04B0108D2
:10C8300010B586B014216846F3F70AFD0E48019042
:10C840000220010302906A460C48FAF7B3F80C4C38
:10C8500001216A4689022046FAF7ACF801216A46AE
:10C86000C9022046FAF7A6F8FF216A4601312046A0
:10C87000FAF7A0F806B010BD000011100008005033
:10C880000004005010B586B014216846F3F7E0FCB0
:10C890001148FFF775FE1148019002200290032015
:10C8A000012103906A4649030D48FAF783F80D4CBD
:10C8B00001216A4689022046FAF77CF801216A467E
:10C8C000C9022046FAF776F8FF216A460131204670
:10C8D000FAF770F806B010BD6801002000001110D2
:10C8E000000800500004005070B5044601210368A0
:10C8F000002249030C48FAF793F80C4D012100225D
:10C90000890228466368FAF78BF801210022C902E0
:10C910002846A368FAF784F8FF210022013128464F
:10C92000E368FAF77DF870BD00080050000400507D
:10C93000FFB581B01D4617460E460124019800F050
:10C94000A1FC304600F05EFC052000F0D3FC012085
:10C95000F6F7BFF902F066F9064606E0019800F026
:10C960005FFBB84201DD002404E0304602F060F9CC
:10C97000A842F3D300F092FF204605B0F0BD0000BE
:10C98000F8B5002568460570A84C2079012809D023
:10C99000022857D12046683002F008FA6079012851
:10C9A0007ED123E16079002818D001284AD14021A6
:10C9B000122001F051F9122000F001FB69460870C5
:10C9C00008789A4E8006403600286ADA2021122024
:10C9D00001F042F9B07D002876D083E0934E2036F6
:10C9E0003079012835D13F2000F0E9FA6946087016
:10C9F000087880072DD40B213E2001F02DF910215D
:10CA00003F2001F029F930465C3002F0CFF9B079CF
:10CA1000002818D00D2000F0D2FA402101430D204B
:10CA200001F01AF93046703002F088F98048006849
:10CA3000002803D00069002800D080473574757441
:10CA4000A5876587F8BD7948903002F0AFF9257168
:10CA5000ECE7618F774F00290AD1A08F002807D11A
:10CA6000B078002831D0322000F0A9FA6087618FB9
:10CA7000A08F091AC9B2C01900F0CAFA608FA08746
:10CA80006A487C3002F092F9B079002823D00D205A
:10CA900000F095FA402101430D2001F0DDF801E09E
:10CAA000A8E02CE06148903002F048F96048006846
:10CAB0000028C3D08768002FC0D01222B256618FE1
:10CAC00000235C48B847B9E70BE0584801213A30E9
:10CAD00000F09EFACBE755482571903002F066F9D8
:10CAE000E4E7257151487C3002F060F95048006855
:10CAF0000028A7D000690028A4D08047F8BD1920DD
:10CB000000F05DFA40B2494F801C801060373870E9
:10CB10001A2000F054FA00217956474A00290BDA0E
:10CB2000A368934203D9091800119D3802E009183F
:10CB30000011A438081809E0A168914203D9011135
:10CB400008189D3802E001110818A43870841320D9
:10CB500000F035FA3871102000F031FA01460D204E
:10CB600001F07AF83979334800F052FAB07D0028A4
:10CB700000D125712D487C3002F018F92C4800684E
:10CB80000028BBD08468002CB8D000232222FB569A
:10CB9000B25E39792748A047284F3878002823D13A
:10CBA00027480078002808D002F03CF804462146C7
:10CBB00024A002F03DF90028F9D1244C2078002867
:10CBC00006D023A002F034F90028FAD1257004E041
:10CBD00023A002F02DF90028FAD12221715E23A0B2
:10CBE00002F026F90028F8D13D70F8BD0821122086
:10CBF00001F032F80E48257100680028F5D0006871
:10CC00000028F2D080470E480078002808D002F0B3
:10CC100009F8044621460BA002F00AF90028F9D1D0
:10CC200015A002F005F90028FAD1F8BDA0060020F1
:10CC300014000020A005002040DD4A1F97040020BA
:10CC40005C0300205B256C755D00000094040020EF
:10CC50007278446F6E652841434B290D0A0000002D
:10CC60007278446F6E650D0A00000000527373699C
:10CC70003D2025640D0A00007478446F6E650D0A2E
:10CC80000000000070B53B4C25462179E61F68790D
:10CC9000F93E2035012911D0022937D1002835D19C
:10CCA000618FA08F33460A1AE97FC0188A425CDD83
:10CCB00000F0F9FFA08FE97F401854E0002826D04B
:10CCC000012823D12B487C3002F070F880211220FB
:10CCD00000F0C2FF0020207127480068002815D00E
:10CCE000C068002812D0804724480078002808D067
:10CCF00001F098FF0446214621A002F099F800288F
:10CD0000F9D121A002F094F80028FAD170BD194899
:10CD1000903002F04BF8608F002809D1A08F0028D6
:10CD200006D1A878002813D0322000F048F9608797
:10CD3000618FA08F0A1AA97F8A420FDB491EC9B2F0
:10CD4000801900F065F9A08FA97F4018401E0AE005
:10CD5000084801213A3000F05BF9E9E7D1B28019C7
:10CD600000F056F904E0A08770BDD1B200F09BFF3F
:10CD7000608FF8E7A0060020140000205C0300206C
:10CD80005B256C755D000000727854696D654F75A8
:10CD9000740D0A0070B5294D294C294608462A7998
:10CDA00040304979C07C012A04D0022A01D10029EF
:10CDB00002D170BD002916D00129FAD10128F8D17D
:10CDC0000221122000F048FF20680028F1D04069BD
:10CDD0000028EED01C2000F0F2F821688006496996
:10CDE000800E884770BD154C012620342674607C67
:10CDF0000028F7D12046703001F0D8FF667411206A
:10CE000000F0DDF840084042A0741B2000F0D7F885
:10CE100006021C2000F0D3F80643300A0102094A3A
:10CE2000711A514380315043090A401868630C203D
:10CE300000F0C5F84009207670BD0000A006002073
:10CE400014000020093D000010B512484079002868
:10CE50001FD001281DD1122000F0B1F80E4CC007E0
:10CE60000BD00521122000F0F7FE2068002810D01A
:10CE7000816900290DD001200AE00421122000F070
:10CE8000EBFE2068002804D08169002901D0002031
:10CE9000884710BDA00600201400002005484079F6
:10CEA000002806D103482030017C002901D101214E
:10CEB00001747047A0060020F8B52E4D287901288E
:10CEC0002BD0022828D100F0CDF8FFF771FA00200E
:10CED00000F010FA284E002460002718F05D00F0E2
:10CEE000D1F9B8198178407800F0B6FE641CE4B23C
:10CEF000102CF1D3002000F0C5F91E484030007F0F
:10CF000000F026FA002028711C480068002803D091
:10CF10004068002800D08047F8BD6879002816D105
:10CF2000144E0024203634747474AC876C870B2143
:10CF30003E2000F091FE10213F2000F08DFEB079E0
:10CF400001280AD030462C71703001F02FFF0B48B9
:10CF500000680028E0D0C068DBE70D2000F02FF863
:10CF6000402101430D2000F077FE0248903001F08F
:10CF7000E5FEECE7A0060020F04B010814000020BD
:10CF800070B50025012000F07DF9FF21112000F08F
:10CF900063FE052000F0AEF900240120F5F799FEAC
:10CFA0002C2000F00CF8C007C00FA040641C054303
:10CFB000E4B2202CF1D300F071FC284670BD08B516
:10CFC0000122694600F003F86846007808BDF8B50C
:10CFD0000446012715460E46FF0305200022394668
:10CFE0000007F9F73BFD6006400EF9F7A3FF0024A8
:10CFF00005E00020F9F79EFF3055641CE4B2AC4216
:10D00000F7D30520012239460007F9F727FDF8BDBF
:10D010000A4610B501460020FFF7D9FF10BD0000F9
:10D0200010B5002804D0012808D00020C04310BD4E
:10D030001120FFF7C4FF4008404210BD07480849CF
:10D040008068884204D91B20FFF7B9FF9D3810BDC6
:10D050001B20FFF7B4FFA43810BD0000A00600207D
:10D0600040DD4A1F30B585B014216846F3F7F0F86B
:10D070000120019003200E4D0024039002946A4683
:10D0800001212846F9F796FC002201212846F9F7EC
:10D09000E5FC0120F5F71DFE6A46012128460194B2
:10D0A000F9F788FC0620F5F714FE05B030BD000046
:10D0B0000004005073B5394C064661790020002900
:10D0C00002D0012966D128E00020A0876846334DB0
:10D0D000017961872035A878002809D0322000F036
:10D0E000BBFD68460279501E3F2806D8EA770AE061
:10D0F000012101A800F0D7FDF3E73146284806F0EA
:10D1000065F82020E877E97F304600F0CCFDA08F5D
:10D11000E97F4018A087A06A3CE02048BE25403047
:10D12000407D012821D03320FFF749FF2840411CD2
:10D13000332000F091FD1D213B2000F08DFD68465D
:10D140000179164860300171222000F085FD002130
:10D150000E2000F081FD00210D2000F07DFD01205A
:10D16000FFF72DFF40070AD00EE03320FFF727FF1F
:10D1700028400146332000F06FFD1921DCE700F064
:10D18000A7FB0120F5F7A5FD68460179304600F0C0
:10D190008AFDA06D00F0AEFB7CBD0000A006002063
:10D1A000A005002010B5054B032805D00022102152
:10D1B0001846F9F753FC10BD0122F8E700040050AF
:10D1C000F0B50E4985B00A78824215D00870002566
:10D1D000012603270A4C14216846F3F739F86A46FA
:10D1E00010212046039701960295F9F7E3FB0022F0
:10D1F00010212046F9F732FC05B0F0BD6401002093
:10D200000004005070B505461048114E8560314647
:10D210002846F2F76DFF044630466043281A0002A4
:10D22000711040183146F2F763FF210244182002C2
:10D23000010E062000F010FD2004010E072000F072
:10D240000BFDE1B2082000F007FD70BDA006002034
:10D25000093D000070B50D46044600F013F8002C9F
:10D2600004D0012C0AD12946232005E00448807807
:10D27000002803D12946322000F0EEFC70BD0000EA
:10D28000C006002010B504460120FFF798FE0106F5
:10D29000174801D5012100E000214171C9B2A14226
:10D2A00024D04471012C0FD000F0F8FA0120FFF7D0
:10D2B00086FE4106490E012000F0CEFC00214020F0
:10D2C00000F0CAFC30210EE000F0E8FA0120FFF780
:10D2D00076FE80210143012000F0BEFC00214020A9
:10D2E00000F0BAFC0021412000F0B6FC10BD0000A7
:10D2F000A006002070B5154C050015D060680168C7
:10D30000012088476068016900208847606841699A
:10D31000284688470120FFF752FEC108C90029436B
:10D32000012000F099FC70BD0120FFF748FEC10804
:10D33000C900012000F090FC606801690120884765
:10D34000606801680020884770BD0000140000205C
:10D3500010B504460120FFF795FF0548002C04771F
:10D3600001D0342100E01221392000F075FC10BDFD
:10D37000E006002070B504460920FFF720FE0646AF
:10D380004D20FFF71CFE054621488068FFF700F995
:10D390007106490E084370210843C1092AD0112C97
:10D3A00002DD07210D4302E0ED08ED002D1DE943EC
:10D3B000490703D0022C0CDA02240DE0052C01DA17
:10D3C000052402E0142C00DD142401090901641F66
:10D3D00005E0112C00DD112401090901A41E20071C
:10D3E000000F0143092000F037FC29464D2000F0D2
:10D3F00033FC70BD0021C9438C4201DA0C4602E0C7
:10D400000E2C00DD0E2401090901641CE7E7000071
:10D41000A0060020F8B506460027764801F0C6FCB5
:10D42000744C683C6079002802D0012825D125E0A1
:10D43000704D4020483DAF79FFF7C1FD8107890F4E
:10D4400040200C3100F008FC4120FFF7B8FD3E21E0
:10D4500008400146C131412000F0FEFB3520FFF7B6
:10D46000AEFD8006800EA8771E210D2000F0F4FB93
:10D47000002028746874A08760877DE05D4D283D9A
:10D48000687D012825D03320FFF799FDBE21084093
:10D49000411C332000F0E0FB1D213B2000F0DCFBB1
:10D4A000606C09287ED23120FFF789FD4106490EC4
:10D4B000312000F0D1FB0021302000F0CDFB606C6A
:10D4C000030002F096F80910171E252C333D3D3D50
:10D4D00041003320FFF773FD41210143332000F069
:10D4E000BBFB1921D9E748212F2000F0B5FB4249A9
:10D4F000A06821E044212F2000F0AEFB3F49A06846
:10D500001AE044212F2000F0A7FB3D49A06813E05A
:10D5100044212F2000F0A0FB3A49A0680CE04421F0
:10D520002F2000F099FB3849A06805E044212F2006
:10D5300000F092FB3549A0684018FFF763FE03E056
:10D5400040212F2000F088FBE87CAF7D012835D0FA
:10D550001F21112000F080FB4020FFF730FD8106E5
:10D56000890E402000F078FB00210F2000F074FBB2
:10D5700000210D2000F070FBFF2101312448F2F75B
:10D5800067FE01202071002E08D01A483146143061
:10D5900001F0C2FB1748143001F0D0FB607900287D
:10D5A00016D000E003E0002F1FD005201EE0312040
:10D5B000FFF705FD802101433120C3E71D21112024
:10D5C00000F04AFB4020FFF7FAFC33210140C8E796
:10D5D0000520FFF78FFE0748E16A283001F09CFB29
:10D5E0000448283001F0AAFBF8BD0620FFF782FEB0
:10D5F000F8BD000008070020821E0000B4280000CB
:10D60000043D00005E510000127A0000C6A2000036
:10D61000A0050020FFB587B017460C460546139EAF
:10D62000FFF730FE11999848090A0691002D04D0A1
:10D63000012D7AD1022C7AD9FEE7C76105464461F3
:10D640001098A8619048203086701499C17015997F
:10D65000017118994171199981711198288438467E
:10D66000F3F7C4F907460B4601913A460020874973
:10D67000F3F708F90322F3F77DF904900591129866
:10D68000F3F7B4F9059B049AF3F794F80022804B62
:10D69000F3F790F8F3F70AFAE8623A4600207D497A
:10D6A000019BF3F7EFF8F3F701FA85B2290A02209C
:10D6B00000F0D2FAE9B2032000F0CEFA2046F6F7E5
:10D6C00029FB0146122000F0C7FA1098F6F722FB5A
:10D6D0000146132000F0C0FA2520069900F0BCFA9C
:10D6E0001198C1B2262000F0B7FA002E01D014998B
:10D6F00000E0FF21322000F0AFFA3020FFF75FFC9E
:10D700006F210840002E01D0002100E08021084355
:10D71000159909010143302000F09EFA3120FFF7EE
:10D720004EFC4021014331209FE0A0E0FFE7564836
:10D73000E41D554D8764446440350A986873119818
:10D74000E8812E74149868741598A8741698E87473
:10D7500017982875189868751998A8750C2F01D90D
:10D760000C2702E0062F00D20627072C02D0082C37
:10D7700002D003E00B2F45D00C2F43D0002028739C
:10D780001D20FFF71CFC0A99200149000843304383
:10D79000C1B21D2000F060FA1E20FFF710FC082126
:10D7A00008403901084315998900084312998905F1
:10D7B000890F0843C1B21E2000F04EFA2620FFF761
:10D7C000FEFBF7210840297BC9000843C1B226208F
:10D7D00000F042FA1298C1B21F2000F03DFA20205A
:10D7E000069900F039FA1198C1B2212000F034FAFC
:10D7F000002E03D02220149900F02EFAE87C012894
:10D8000002D00DE00120BAE74420FFF7D8FB8021C9
:10D810000143442000F020FA297D242000F01CFA66
:10D82000092C02D00321362010E017481A498068DD
:10D83000884205D90221362000F00EFA642104E066
:10D840000221362000F008FA7F213A2000F004FA85
:10D85000062F0ED03120FFF7B2FBC108C9003120DE
:10D86000C91C00F0F9F90A21372000F0F5F90BB0D6
:10D87000F0BD3120FFF7A3FBC108C9003120491DCD
:10D8800000F0EAF90C21EFE7A00600200000F03FCD
:10D8900000408F4080847E4140DD4A1F10B50A4819
:10D8A00001F084FA0848143801F080FA0020FFF7EC
:10D8B00021FD064840680168002088470249002091
:10D8C0007C39087110BD00001C07002014000020E6
:10D8D00010B5074801F06AFA0548143801F066FAF5
:10D8E0000120FFF707FD024900207C39087110BDB7
:10D8F0001C07002010B50446294801F057FA2848B3
:10D900002146143801F008FA254C7C3C6079002847
:10D9100002D001282CD119E04020FFF750FB8107ED
:10D92000890F4020103100F097F94120FFF747FBA5
:10D930003E210140412000F08FF93520FFF73FFBE9
:10D9400081061748890E5C38817711E014483C380D
:10D95000C07C012816D0F721112000F07DF940206D
:10D96000FFF72DFB8106890E4020403100F074F94D
:10D97000022020710A48143801F0E0F90320FFF773
:10D98000B9FC10BDF521112000F066F94020FFF729
:10D9900016FB33210840014640314020E6E70000F5
:10D9A0001C070020FFB581B01E460C460C9F0A9D47
:10D9B0000198FFF767FC76484068C16820468847B1
:10D9C0003A0A019973480092002908D0012973D1BD
:10D9D0002246044640342270022E57D9FEE70473D3
:10D9E00003994661C56101616A49078420310D9A36
:10D9F0008A700E9A0A71119A4A711299816203987B
:10DA0000F2F7F4FF0022644BF2F73CFFF3F74EF815
:10DA100084B2210A042000F01FF9E1B2052000F0D1
:10DA20001BF92846F2F7E2FF0B46024600205B494D
:10DA3000F2F728FFF3F73AF884B2210A022000F047
:10DA40000BF9E1B2032000F007F92520009900F05E
:10DA500003F9F9B2262000F0FFF83020FFF7AFFA03
:10DA60006F2108400D99002901D0002100E080219C
:10DA700008430E9909010143302000F0EDF83120F0
:10DA8000FFF79DFA40210143312071E0F61D466405
:10DA900085640B996173E7810D9921740F99E17485
:10DAA000109A22750E9AA274119A6275129A826562
:10DAB0000C2D02D90C2503E05CE0062D00D20625D2
:10DAC000072E02D0082E02D003E00B2D06D00C2D1D
:10DAD00004D000202073012902D00DE00120F9E7D5
:10DAE0004420FFF76CFA80210143442000F0B4F891
:10DAF000217D242000F0B0F81D20FFF760FA0B997B
:10DB00003001490008430D990843C1B21D2000F0BF
:10DB1000A3F81E20FFF753FA0B2108402901084300
:10DB20000E9989000843C1B21E2000F095F8262006
:10DB3000FFF745FAF7210840217BC9000843C1B22D
:10DB4000262000F089F82020009900F085F8F9B22D
:10DB5000212000F081F8062D0ED03120FFF72FFA9A
:10DB6000C108C9003120C91C00F076F80A2137200D
:10DB700000F072F805B0F0BD3120FFF720FAC108BF
:10DB8000C9003120491D00F067F80C21EFE70000C3
:10DB900014000020A006002080844E4080847E4136
:10DBA00030B50D467D211446C90089B04C43FFF7BE
:10DBB00029FB0020079006900390059001900490A7
:10DBC0004B200521800100230291009008941A4601
:10DBD00029461846FFF7E6FE3120FFF7F0F9BF218E
:10DBE0000140312000F038F8F021402000F034F8F6
:10DBF000A021412000F030F82146074801F08CF8C0
:10DC00000549022068390871034801F097F803209C
:10DC1000FFF770FB09B030BD080700207047000017
:10DC200010B50C4C6079002812D0012810D1FA21CF
:10DC3000112000F011F84020FFF7C1F98108890098
:10DC4000402000F009F8032020710720FFF752FB65
:10DC500010BD0000A006002013B5012201A900F0AC
:10DC600001F81CBDF8B50446012715460E46FF0312
:10DC70000520002239460007F8F7F0FE20468021F3
:10DC80000843F9F757F9002404E0305DF9F752F939
:10DC9000641CE4B2AC42F8D30520012239460007E7
:10DCA000F8F7DCFEF8BD0A4610B501460020FFF784
:10DCB000D9FF10BDF0B589B000204B4C0790A17C76
:10DCC000FF2902D0002903D003E0092009B0F0BDEC
:10DCD000A066A07FF4F766FD444DA06E01906978C0
:10DCE00068460173217F8173A17A41732F463E4EAE
:10DCF000606E38376836029003E07878687069465D
:10DD00000873394A009607AB1D3201A9207EFEF741
:10DD1000B9FA0028F1D0354E012320360122F356FE
:10DD2000AA56717B207EFDF77CFA41B23046BC30AA
:10DD300000902A7A207E6B68FDF7AFFC3746D0371B
:10DD4000009708212A7A7156207E6B68FDF7A5FCA2
:10DD5000A07A102600281BD001216956E27B607949
:10DD600001F08CFB002838D0384614382969C06887
:10DD7000081860676869F9684018A067A07A0028E9
:10DD800010D0079900292AD0206C304320641AE073
:10DD90001648A969DC30C06808186067E869F96846
:10DDA0004018A067124800780028EAD00798002899
:10DDB00015D0216C104A314321640E490988514322
:10DDC000814200D201460948A03000F0A5FF074873
:10DDD000A03000F0B3FF002078E7082076E7607FEE
:10DDE00000F036FB72E70000940400206C1B00205A
:10DDF000990100204603002060EA0000F0B58FB0D2
:10DE0000F9F74EFC01287DD108A8F4F73BFCFF4848
:10DE100000250446C16C80342E46012902D0022917
:10DE200004D00AE08667C667266005E0216981673D
:10DE30006169C167A1692160C664F5480088F54938
:10DE4000884208D8F14801214172F3A000F0F0FFA8
:10DE50000028FAD101E0ED48467200226B216820CB
:10DE6000FBF72EFCFBF71EFBF24800274665F14945
:10DE7000E64A6031081F20320191031F0090911E75
:10DE8000881EFBF7E7F9EB4A002054321346083BA3
:10DE9000111F04AE07920BC6E64C226EE16D019293
:10DEA00000910290039002460146A36DF3F73EFCF9
:10DEB00020468038416E8166616D416602460146AA
:10DEC000663A68316430F4F7A7FE21462046E63909
:10DED0005430F4F74DFC216CE06CF2F7D9FAE064B1
:10DEE000616C206DF2F7D4FA2065A16C606DF2F7D9
:10DEF000CFFA7F1C60650A2FB9DB00272646803EDB
:10DF0000CC4900E074E26031081FC04A0191203220
:10DF1000031F0090911E881EFBF79CF9C549002045
:10DF200054310A46083A0B1FC24C059306920791DA
:10DF30000490226EE16D01920091029003900246DE
:10DF40000146A36DF3F7F2FB706E2246B066E63A27
:10DF5000606D1146CE317066081FF4F75DFE2146F4
:10DF60002046E6395430F4F703FC216CE06CF2F7FC
:10DF70008FFAE0640190616C206DF2F789FA2065F8
:10DF80000090A16C606DF2F783FA60650446019918
:10DF9000B068F2F77DFAB06000997068F2F778FA2D
:10DFA00070602146F068F2F773FA7F1CF0601E2F54
:10DFB000A6DB964EA04980367068F2F7FFFA044659
:10DFC000B0629D49B068F2F7F9FA0746F0629A49E3
:10DFD000F068F2F7F3FA306306468C48007A0128BD
:10DFE00007D18A4900200872084680308763C663DB
:10DFF000446386488030416B20460091F2F799FADD
:10E000008E49884217D88E4A904214DA20460099E9
:10E01000F2F73EFA0024E4432146F2F70DFB0146F5
:10E020000098F2F735FA2146F2F706FB774980317E
:10E03000C861486303E075488030C4614463734C31
:10E0400038468034A16B0091F2F773FA7B4988421D
:10E0500015D87B49884212DA38460099F2F718FA47
:10E060000027FF433946F2F7E7FA01460098F2F736
:10E070000FFA3946F2F7E0FA2062A06301E0276266
:10E08000A763E16B30460F46F2F753FA6B498842BB
:10E0900015D86B49884212DA39463046F2F7F8F95A
:10E0A0000026F6433146F2F7C7FA01463846F2F742
:10E0B000EFF93146F2F7C0FA6062E06301E06662B0
:10E0C000E663E0692061276A504E6761B16FF2F73D
:10E0D00030FAE0613846F16FF2F72BFA20625548CA
:10E0E000616A41652168E06BF2F723FA6062002003
:10E0F0006060A060E06000F095FD524F524EE06914
:10E100003146F2F71EFAF2F77FFCF2F75BFC0022D1
:10E110003B46F2F7B7FB02460B464CA000F088FEE8
:10E120000028ECD1394848498030006AF2F709FAF2
:10E13000F2F76AFCF2F746FC00223B46F2F7A2FB3C
:10E1400002460B4645A000F073FE0028EAD1474E78
:10E15000FF21F06BC905C84210D33B49F2F7F1F932
:10E16000F2F76BFC294C606241A0616A00F060FE2E
:10E170000028F9D1606AC043401C606234464034D4
:10E18000F06BF2F7B1FC2278009202460B463CA0FD
:10E1900000F04EFE0028F3D105F0AEFB3D483E49AD
:10E1A00000780978800149010843001D174FC0B26B
:10E1B000204C786402208834607104F063FC0128EC
:10E1C0007CD004F05FFC02287AD01A482268C16B28
:10E1D000090E5155C16B226809146D1C5155818F70
:10E1E000226809126D1C51552268818F6D1C515592
:10E1F000816B2268090E6D1C5155816B22680914D0
:10E200006D1C5155018F09126D1C49E094010020CD
:10E210008C010020180B00000A0D426174746572B5
:10E220007920766F6C7461676520746F6F206C6FF6
:10E23000770D0A00940200200000F041CDCC4CBEC6
:10E24000CDCC4C3E000059400000C842526F6C6C6F
:10E250003D25302E32662020000000005069746396
:10E26000683D25302E326620200000008007002007
:10E27000416C7469747564653A25640D0A20000068
:10E28000416C7469747564653A252E316625630D99
:10E290000A20000074030020700300200EE00FE04D
:10E2A00022685155008F21686D1C485554486D1CDB
:10E2B000006801281AD0002830D089E0002000E052
:10E2C000FF202168485521686D1C485521686D1C48
:10E2D000485521686D1C485521686D1C48552168BA
:10E2E0006D1C485521686D1C4855DCE7386C0128C9
:10E2F0000B980DD0F2F788FB0012216848556D1C71
:10E300000B98F2F781FB216848556D1C786C5CE036
:10E31000F2F77AFB001240210843EEE7386C01283F
:10E320000B9867D0F2F770FB0012216848556D1CFE
:10E330000B98F2F769FB2168485521686D1C786CD1
:10E34000485531482F49C0696D1CF2F7FAF8F2F7C9
:10E350005BFB2168001248552B482A49C0696D1C97
:10E36000F2F7EFF8F2F750FB2168485526482549A7
:10E37000006A6D1CF2F7E5F8F2F746FB216800121F
:10E38000485521481F49006A6D1CF2F7DAF8F2F788
:10E390003BFB216848551B496D1CB06CF2F7D1F866
:10E3A000F2F732FB2168485516496D1CF06BF2F705
:10E3B000C8F8F2F729FB21680012485511496D1C75
:10E3C000F06BF2F7BEF8F2F71FFB216848556D1CA1
:10E3D0007F20C005B0630020387378752571FD7209
:10E3E000F8F79EFF04F030FB01460848F9F798FC67
:10E3F0000FB0F0BDF2F708FB00124021084394E78C
:10E400006C0300200000C842140200201C030020FE
:10E41000FEB5002426468F252E400B4DEF7AFF01D6
:10E420003E436F463E71009313460A4601A9FCF72E
:10E430004BF9002806D1054844710471296BC1606D
:10E44000FFF738FCFEBD0000940400209C1C002057
:10E45000F0B585B0002269460A70414E08717078A7
:10E46000487130788871306B0290706B3D4C03902E
:10E47000A08C0882F8F754FF3B480125007800285B
:10E4800009D000F0CFFB0746394638A000F0D0FC99
:10E490000028F9D10DE0A078002805D135A000F0C2
:10E4A000C7FC0028FAD1A5703DA000F0C1FC0028EF
:10E4B000FAD13CA0216B00F0BBFC42480068012867
:10E4C0001CD141480078002818D140480068002835
:10E4D00014D1F4F7B9F801221702052039460007D4
:10E4E000F6F78BFAC820F4F7F4FB05200022394632
:10E4F0000007F6F782FAC820F4F7EBFB194B6A46DF
:10E50000443301A9207EFDF7EEFE314A10465570D6
:10E51000143845707178817069460978C170616CF2
:10E52000816051607D21C900C03800F0F5FB0C48C6
:10E53000703000F003FCA07A002804D10948203094
:10E540000178491C0170A08CC1B22248026B22489C
:10E550009047206C28432064002005B0F0BD0000E7
:10E560006C1B0020940400205C0300200A0D5B2536
:10E570006C755D000A0D506C65617365207573657F
:10E580002041542B444542554720746F20736565E4
:10E5900020646562756720696E666F0D0A00000071
:10E5A0000D0A00002A2A2A2A2A2055704C696E6B0F
:10E5B000436F756E7465723D202564202A2A2A2ACD
:10E5C0002A0A0D00700300209B010020CC010020CE
:10E5D000B01C0020D04C01086C1800201FB5124C54
:10E5E0006A46617F117011494B7853700B789370B4
:10E5F0000A6B0192496B02916A4690816946207EBE
:10E60000FDF76AFE09487D21C900703000F084FBE7
:10E610000648703000F092FB206C01210843206412
:10E62000002004B010BD0000940400206C1B0020EA
:10E6300070B50D4614460A4902464B6C61B2284635
:10E6400098477D21C900074800F066FB054800F0A7
:10E6500075FB05480122016C11430164002070BD67
:10E66000D04C0108DC1B002094040020FEB50220E1
:10E67000694608706846FAF775FA002802D0ADA01E
:10E6800000F0D6FB68460079162104066846017042
:10E69000FAF768FA002802D0A6A000F0C9FB684685
:10E6A0000421AA4E41561420305609042143000289
:10E6B00037460843403F797835460143703DA87896
:10E6C000A34C8200A150401CA8700721684601702D
:10E6D000FAF748FA002802D096A000F0A9FB684695
:10E6E000397800790F04000607430021684601705D
:10E6F000FAF738FA002802D08EA000F099FB68469D
:10E700000079317B000238430143A8780A27820050
:10E71000A150401CA87068460770FAF723FA002839
:10E7200002D084A000F084FBA87801998200A15057
:10E73000401CA87068460770FAF714FA002802D047
:10E740007CA000F075FB6846017AA8788200A15091
:10E75000401CA870102168460170FAF703FA0028DF
:10E7600002D074A000F064FBA87801998200A15047
:10E77000401CA8701120694608706846FAF7F2F943
:10E78000002802D06BA000F053FBA878019982000A
:10E79000A150401CA8701220694608706846FAF71C
:10E7A000E1F9002802D063A000F042FBA8780199AB
:10E7B0008200A150401CA87013206946087068466A
:10E7C000FAF7D0F9002802D05AA000F031FBA8785F
:10E7D00001998200A150401CA8700320694608706E
:10E7E0006846FAF7BFF9002802D052A000F020FBDB
:10E7F000A87801998200A150401CC0B255498200FE
:10E800000968A1505449F27A0978401C0902C0B243
:10E8100011438200A150401CC0B24C4983004839CA
:10E820000A68E2504D4A4E4B12881B7812041B02B4
:10E830000979401C1A43C0B20A4381006250401C4F
:10E84000C1B24848484A00781278000612041043C2
:10E85000464A127812021043454A127810438A0041
:10E86000A0506A7AAB7A12061B041A43414B491C2A
:10E870001B88C9B21A438B00E250491C3E4AC9B2F8
:10E8800012688B00E250491CC9B23C4A8B001268E6
:10E89000E250491CC9B23A4A8B001268E250491C46
:10E8A000C9B2384A8B001268E250491CC9B2364AD4
:10E8B0008B001268E250491CC9B2344A8B001268BE
:10E8C000E250491CC9B2324A8B001268E250491C1E
:10E8D000C9B2304A8B001268E250491CC9B22E4AB4
:10E8E0008B001268491CE250C9B28A00491CA05032
:10E8F000CEB22A49A869F1F724FEF2F79EF8B100DA
:10E9000060502749274A09781278761C0902F0B22C
:10E9100011438200A150401C234CA8702046F4F7FC
:10E920005DFBAA780A492046F4F780FB0020A87016
:10E93000FEBD00004C4F52414D41432053544154C1
:10E940005553204552524F520A0D00001404002026
:10E9500064160020C001002064030020460300204C
:10E960009A0100205D0300205E0300205F03002069
:10E9700060030020940300206C0300206803002043
:10E980007003002074030020780300207C03002023
:10E9900080030020C4010020C80100200000C842FC
:10E9A00062030020610300200090010870B5184C3C
:10E9B0000022A11C082005F02BFC00210120E268A8
:10E9C00005F026FC214600221831102005F020FC1D
:10E9D000214600222831102005F01AFC2146002291
:10E9E0003831102005F014FC214600221031082097
:10E9F00005F00EFC074D2846F4F7F0FA303CE278BB
:10EA000005492846F4F712FB0020E07070BD0000B5
:10EA1000D403002000910108E416002010B5F6F799
:10EA200033F810BD10B594B014210EA8F1F710FC06
:10EA300038216846F1F70CFC0220009001210A9071
:10EA4000039180040C9000240001019410210D908A
:10EA50000B9404916846F6F755FB002801D0F4F7B3
:10EA600025FA1148816B0204114381630F48016844
:10EA70000322D2029143C214891801604168C9433C
:10EA8000C906FBD50F200E9003200F90109411940F
:10EA9000012112940EA8F6F725FA002801D0F4F708
:10EAA00005FA14B010BD00000010024000700040D4
:10EAB00010480168821511430160C1680E4A114077
:10EAC000C16001680D4A1140016081684908490030
:10EAD000816001680122920491430160C168FD22B6
:10EAE00012049143C160002101610549C00388609F
:10EAF00070470000001002400C40FF88F6FFF6FE51
:10EB000000ED00E010B500F001F810BD10B50248AE
:10EB1000F7F734FB10BD000068050020F0B502686F
:10EB20000124A407124D134E134FA04205D0A84252
:10EB300003D0B04201D0B84204D1134670229343AF
:10EB40004A681A43A04205D0A84203D0B04201D07F
:10EB5000B84204D103231B029A43CB681A430260D4
:10EB60008A68C2620968816201214161F0BD0000CA
:10EB700000040040000801400014014010B50123CA
:10EB8000046A8B409C430462036A8A401343036215
:10EB900010BD000070B5046A6408640004628469F2
:10EBA000056A0126B607B04208D00E4EB04205D025
:10EBB0000D4EB04202D00D4EB04202D1A408A400C6
:10EBC00002E0A408A40001221443F02294431A078F
:10EBD000120E0A2322439D43194029438261016298
:10EBE00070BD000000040040000801400014014016
:10EBF00070B5046A1025AC4304628569046A032673
:10EC00003602B54312022A430F252D031B071B0CA6
:10EC1000AA431343A0220901944311402143836175
:10EC2000016270BD10B5F8F743F8F8F773F910BD3D
:10EC300070B50546F8F73CF804462846F8F772F92F
:10EC4000201AF8F767F970BD002202604260027274
:10EC50000261C1607047000010B5054A11680029C3
:10EC600001D000230B720161106000F03FF810BD6D
:10EC70003C05002070B5F8F707F80446F8F7A2F84D
:10EC8000031B194C206800282DD00146002507E001
:10EC900016689E4202D9F61A166000E015600969EE
:10ECA0000A69002AF4D100281DD001692160C068DA
:10ECB000002800D1FEE780472068002813D0F7F72E
:10ECC000E9FF014620680268914205D90169216087
:10ECD000C0680028EFD1FEE7002804D0017A00299F
:10ECE00001D100F003F870BD3C05002070B504466A
:10ECF000F7F7C8FF054601202072F7F7CBFF216820
:10ED00004019884201D8084603E0F7F7C3FF4019CD
:10ED10002060F8F709F870BD70B505460846F8F7A9
:10ED200001F90446284600F041F8F7F7ABFF8442AA
:10ED300000D204462C606C6070BD0000F8B5040081
:10ED4000EFF3108572B62CD0174F3868014602E0F9
:10ED5000A04226D000690028FAD100266068206011
:10ED6000267200290CD0F7F795FF21680918216059
:10ED700038680268914206D22046FFF76DFF10E026
:10ED8000F8F720F8F8E70169002908D022680B6835
:10ED90009A4201D90846F6E70461216101E0046165
:10EDA000266185F31088F8BD3C05002070B5EFF3AF
:10EDB000108572B6144C21680A1E21D000281FD07D
:10EDC00081421BD1087A00260128086903D0002857
:10EDD0000AD0206014E0002804D00E722060FFF7F3
:10EDE00085FF0DE0F8F786F8266009E0814203D13F
:10EDF00008691061002803E00A4609690029F5D175
:10EE000085F3108870BD00003C05002008B5064859
:10EE100005F03EFE02200549C2010090084600238D
:10EE20002038F3F7DBFD08BDB9EE000818200020FC
:10EE30000FB4F0B5C3B0FF21002549AB013102A8E2
:10EE4000489A00F091FB82B2684602800027EFF3F7
:10EE5000108472B6012302A91548F3F7C1FC0028FB
:10EE60001BD0144E3078012802D084F3108818E0AB
:10EE700069460F48F3F72EFE0190377001212020DC
:10EE8000F9F7E2FB84F3108868460188019805F0E1
:10EE900063FE0198002804D101E084F31088002566
:10EEA000ED43284643B0F0BC08BC04B0184700004E
:10EEB000F81F00204405002038B5EFF3108472B627
:10EEC00069460D48F3F79EFD69460B48F3F702FECD
:10EED000002806D084F310886946098805F03CFEB6
:10EEE00038BD00212020F9F7AFFB0449012008704C
:10EEF00084F3108838BD0000F81F0020440500206E
:10EF000010B5818CC90707D001684A6801235B04EA
:10EF10009A43836A1A434A60818C890707D501683E
:10EF20004A6801231B049A43C36A1A434A60818CCE
:10EF3000490707D501684A6801239B049A43036B7C
:10EF40001A434A60818C090707D501684A68012382
:10EF5000DB039A43436B1A434A60818CC90607D589
:10EF60000268916801231B039943836B19439160E5
:10EF7000818C890607D501688A6801235B039A435F
:10EF8000C36B1A438A60818C490612D503685A689C
:10EF900001210905046C8A4322435A60026C8A42AB
:10EFA00007D10268516803235B059943436C1943F9
:10EFB0005160818C090607D501684A680123DB048A
:10EFC000806C9A4302434A6010BD0000F8B50026E9
:10EFD0000446C666F5F718FD054620680068124F1E
:10EFE000000709D501212B4600224905204600973C
:10EFF00000F00BFA00280DD12068006840070BD5FF
:10F0000001212B46002289052046009700F0FDF9DA
:10F01000002801D00320F8BD202060346072A07267
:10F0200026720020F8BD0000FFFFFF0110B5806AC6
:10F030000022014640314A834A82F7F7BCF910BDED
:10F0400070B5846A25466035687A0026212808D183
:10F0500020688068000604D552200653204600F040
:10F0600040F8A87A222808D120688068400604D594
:10F070005A200653204600F025F8E06E1021084380
:10F08000E0662046F7F797F970BD10B501460968AC
:10F09000806A096889060DD4002252210A5201684B
:10F0A0008A6880239A438A6000680168402211437D
:10F0B000016010BDF7F7E0FB10BD10B5806AF7F7EF
:10F0C000E3FB10BD01680A68FF2321339A430A60FD
:10F0D00001688A68520852008A602021603081727B
:10F0E000704701680A68C0239A430A602021603093
:10F0F0004172704770B50246403201466031938BD1
:10F100008D7A0C460168222D05D0886908221043AB
:10F110008861022070BD496A01268568360389B27C
:10F12000B54202D10569002D0BD01940436D5D1C1D
:10F1300045651970518B491E0904090C518307D08C
:10F1400015E0456D19402980416D891C4165F1E745
:10F1500001680A68FF2321339A430A6001688A68BC
:10F16000520852008A602021A172F7F7BBFA0020F2
:10F1700070BD0000FEB50446016880682269E3693D
:10F1800010436269102700261A4310430A68354667
:10F19000784B1A4002430A60206841680322120338
:10F1A0009143E26811434160734A2168A06991422A
:10F1B00001D0226A10438A680B231B029A43024340
:10F1C0008A606E4A20686E4990420CD1C8688007F8
:10F1D000800F06D0012843D002283FD0032826D133
:10F1E00024E0012723E0674A90420AD1C8680C2135
:10F1F000084031D0042833D008282FD00C2816D14D
:10F2000014E0614A904227D0604A904224D05A4A82
:10F2100090420CD1C9680320800201401CD0101517
:10F22000091A1DD0091A19D0814200D108270220DD
:10F23000F5F7B2FC0190504B514922684039D81380
:10F2400000929A4235D1002F0CD0022F0DD0042FFE
:10F2500012D0082F1CD113E00027E8E70227E6E7C9
:10F260000427E4E7F5F7F2FE08E00868C00601D5D8
:10F27000474805E0474803E0F5F708FF002873D04A
:10F28000626851005118814202D81103814201D2B3
:10F29000012569E0010E060250080023301859418B
:10F2A000F0F750FF032109023B4A411A914259D914
:10F2B000EEE7E26982422DD13B0000F09AF909069F
:10F2C000080B24192424241F2400019812E0F5F7C8
:10F2D000CDFE0FE008686168C00602D548082F4AD5
:10F2E00001E02F4A48088018F0F702FF86B20BE0D1
:10F2F000F5F7CCFE616840004A08F4E76168012236
:10F3000048081204EFE70125310909013007400FD1
:10F31000084327E03B0000F06CF909070A0D061DC1
:10F32000060606290600B3E7F5F790FE14E0F5F7A8
:10F330009DFE11E008686168C00602D54A081448BD
:10F3400001E014484A081018F0F7D2FE81B2009884
:10F35000C16009E0F5F79AFE61684A088018F0F785
:10F36000C7FE80B22168C8602846FEBD61684A08B1
:10F37000E9E70000F369FFEF004800400038014072
:10F380004010024000440040004C0040005000404B
:10F3900000093D000024F400FFFC0F0000127A0079
:10F3A0000048E8016921095C212901D00220704749
:10F3B00002464032518A002912D0012381681B0382
:10F3C000994202D10169002915D0C16C4B1CC3645C
:10F3D000006809788162508A401E50820020704780
:10F3E00001680A6880239A430A6000680168402225
:10F3F00011430160F2E7C16C03680988C905C90DB2
:10F400009962C16C891CC164E5E7FFB581B01746FC
:10F410000E4604460A9D1DE0681C1BD0002D05D039
:10F42000F5F7F2FA0499401AA84213D92068016846
:10F43000FF22A13291430160206881684908490098
:10F440008160202060346072A0720020207203204E
:10F4500005B0F0BD2068C1693046884304D0002063
:10F46000B842D9D00020F3E70120F9E710B50248EF
:10F4700005F0A8F910BD00005810002038B5054669
:10F480000E481446027B6846827041700D2101705F
:10F490000B48C17E002902D00E216A4611706946D0
:10F4A000007EFCF7BEFE81B22819884203D8FF28EF
:10F4B00001D8012038BD002038BD00008C1B002081
:10F4C0009404002070B505461A480C46816A284607
:10F4D000884700282AD0184818492818884201D29D
:10F4E000022021E0164817492818884201D8002038
:10F4F0001AE0154815492818884201D8012013E060
:10F50000134814492818884201D805200CE01248F5
:10F5100012492818884201D8032005E010481149F3
:10F520002818884203D804202070012070BD0020D4
:10F5300070BD0000D04C010840AA8FCC80841E0012
:10F54000C02571CCC0C62D00FF5E43CCBF2709008B
:10F55000A0B038CC20A1070040022ECC90D00300F0
:10F56000606E29CCE09304007CB51546024600206D
:10F570001C4600290BD0491E00920191044B6A469B
:10F580002146284600F092FA009A002111707CBDB5
:10F59000E50101082021020C01D010211046020AC9
:10F5A00001D010460839020901D01046091F82080F
:10F5B00001D01046891E420801D0881E7047081AE3
:10F5C0007047F8B5040C8BB2264682B25E430D0C30
:10F5D0001046370C584336048019002179411646ED
:10F5E0006E43370C36048019794126466E438919DB
:10F5F000F8BD30B47446641E2578641CAB4200D25A
:10F600001D46635D5B00E31830BC18474900CA0221
:10F610000243100000D004204A0D01D00122104303
:10F62000044A490D914201D102210843012800D129
:10F6300005207047FF0700004100080200D00420A9
:10F640000A0E01D001221043090EFF2901D1022127
:10F650000843012800D105207047FF21400009061A
:10F66000884201D101207047002070474000FF21EF
:10F670004008C905081AC00F7047000000487047CD
:10F6800048050020F8B504464F1EC8000838211868
:10F6900015461E46086849683A4606239A4310D024
:10F6A0002A463346F1F786F83A46D200083AA318BC
:10F6B0001A687F1E5B68F0F7CBFF06223B46934338
:10F6C000EED1022F23D0042F11D0062F2FD12A469E
:10F6D0003346F1F76FF8E36AA26AF0F7B9FF2A46FA
:10F6E0003346F1F767F8636A226AF0F7B1FF2A46FA
:10F6F0003346F1F75FF8E369A269F0F7A9FF2A46FC
:10F700003346F1F757F863692269F0F7A1FF2A46FB
:10F710003346F1F74FF8E368A268F0F799FF2A46FD
:10F720003346F1F747F863682268F0F791FFF8BDB8
:10F7300010B50122F1F71EF910BD10B5F0F788FFE2
:10F7400010BD002210B5134610461146F1F79AF885
:10F7500010BD0000034A10B500201107F1F70AF9A7
:10F7600010BD000001FDFFFF10B50121F0F764FF9F
:10F7700010BD10B500210846F0F720FF10BD5E2136
:10F7800010B5C9430807F0F757FF10BDF0B50E4696
:10F7900014465100FF22120687B0914203D311167E
:10F7A000316007B0F0BD01202502C0070543E00D20
:10F7B0007838C206D20E2020871A6000000E7838F2
:10F7C000401181004D4878440B189C464358002A4C
:10F7D00014D06046406893400146F84003436046B9
:10F7E000806891408646F840014303916046714627
:10F7F000C0689140F84001430F4603E0604641680D
:10F800000391876818462946FFF7DBFE02910490B2
:10F8100029460398FFF7D5FE0391069038462946FE
:10F82000FFF7CFFE0F460698029B3D18049A0399F6
:10F83000BD4201D2012700E000278818C019002F1F
:10F8400002D0884202D903E0884201D2012100E0BF
:10F85000002159180A4620329709C20C8906520322
:10F8600040033760114301900846F1F799F8029080
:10F870000198F1F7A0F81221C943F0F7DDFE0190DD
:10F880002846F1F798F82521C943F0F7D5FE0090F6
:10F8900001990298F0F7FCFD0099F0F7F9FD0121BC
:10F8A000C9024018050B2D0328460299F0F741FEC6
:10F8B0000199F0F73EFE0099F0F73FFE1049F0F78E
:10F8C00040FE00900F492846F0F73BFE0099F0F704
:10F8D000DFFD00900C492846F0F733FE0099F0F761
:10F8E000D7FD002C00DB5CE701210907C91B316053
:10F8F0000121C907484007B0F0BD0000E65F0000E5
:10F90000DB0FC92F22AAFD290000C92F02E008C879
:10F91000121F08C1002AFAD170477047002001E089
:10F9200001C1121F002AFBD1704700000149086085
:10F930007047000048050020F0B51FB486B0099854
:10F94000089A030D0021024314D05148514A181857
:10F95000504305141198012810981AD0281A401CF9
:10F9600000264D4F4D49009601910490002812DA6F
:10F97000444211E01198012449A3012801D11098B3
:10F98000C1430698119A84600360C26041600BB065
:10F99000F0BD4042E4E70446210500203F4A001C38
:10F9A00051410391029012E0E00707D032463B46F6
:10F9B00001990098F0F7FEFE0191009032463B4617
:10F9C00010461946F0F7F6FE06460F466410002C66
:10F9D000EAD10498039B0028029A0999089806DA4C
:10F9E000F0F7E8FE019B009AF0F7E4FE05E0F0F77F
:10F9F00049FF019B009AF0F745FF04460E4600229E
:10FA0000284BF1F799F803D80020C043014607E0DE
:10FA10000022254B20463146F0F71AFEF1F7D2FAC4
:10FA2000102409E0002C0ADB0A220023F0F78AFBED
:10FA3000079B30321A55641E02460A43F2D1112246
:10FA4000641C079B121B1C19119B012B03D0012363
:10FA500008430ED10AE0084304D011201090002082
:10FA6000119077E71098151A6D1E0BE010988242DE
:10FA700002DD00236D1C03E0824201DA00236D1ECB
:10FA8000002BEED0069811998260C16030C07EE7ED
:10FA900001FCFFFF104D0000000014400000F03F8B
:10FAA000300000000000F0430000E03FFFB597B0D9
:10FAB0000646002518E2252877D100242746FD496F
:10FAC000049400E00443761C32780120203A9040F0
:10FAD0000842F7D130782A280ED002223078014629
:10FAE0003039092916D804990A2359433039401866
:10FAF0001443761C0490F1E7189802C804911890FA
:10FB0000002904DA01204003044348420490022003
:10FB10000443761C30782E2814D1042004437078D6
:10FB2000761C2A2809D11898761C80C8189009E0FC
:10FB30000A214F43303FC719761C307801463039CF
:10FB40000929F5D930786C2810D006DC4C281AD059
:10FB500068280ED06A2817D104E0742813D07A28B8
:10FB600012D110E00120400504430CE001210905F9
:10FB700001E0032109050C437178814203D1012082
:10FB800000052418761C761C3078119066280BD05E
:10FB900013DC58287DD009DC00287BD04528F6D01E
:10FBA0004628F4D047281AD1A5E118E0632835D0BB
:10FBB000642870D0652812D19DE170286CD008DCD3
:10FBC0006728F1D069287BD06E280DD06F2806D128
:10FBD000BAE073282ED0752871D0782859D01A9A97
:10FBE000199990476D1C7EE16002400F022809D0F0
:10FBF00003280DD00428189801680DD00D60001D51
:10FC0000189070E11898EA1701680D604A60F6E7ED
:10FC1000189801680D80F2E70D70F0E718986A46B1
:10FC200001781172001D18900020507202A80090F7
:10FC3000012005E0189802C8189000200091C043E8
:10FC400061070DD5002101E00199491C0191B942DC
:10FC500012DA8142F8DB009A515C0029F4D10BE002
:10FC6000002101E00199491C01918142FADB019ACE
:10FC70000099895C0029F5D1019904981A9B471ACB
:10FC800021463846199A00F097FA0199401945180B
:10FC90000BE04FE02CE113E04EE000980099007873
:10FCA000491C00911A9A199990470198401E019099
:10FCB000401CF2D1214638461A9B199A10E137E0D0
:10FCC0000A200021009001916002410F022907D013
:10FCD000189A01CA1892C2179446032908D00AE05C
:10FCE0001898C01DC108C90005C91891944607E0BD
:10FCF00000B2C2179446042902D140B2C1178C4603
:10FD000000226146944506DA0A46002140429141AC
:10FD10008C462D2102E0210504D52B216A46117362
:10FD2000012103E0E10701D02021F7E7029155E02E
:10FD30000A200AE0102008E0102000900021042092
:10FD400004430191082703E008200021019100905D
:10FD50006002410F022907D0189A01CA18920022A6
:10FD60009446032908D008E01898C01DC108C900AE
:10FD700005C91891944603E080B2042900D1C0B2AD
:10FD800000210291210729D51199702906D0009AE6
:10FD90001021019B4A401A4305D00EE040216A46DB
:10FDA0001173012108E06146014306D030216A4603
:10FDB00011731199517302210291009A0821019B3C
:10FDC0004A401A430AD16146014301D1610705D572
:10FDD00030216A46117301217F1E02911199582921
:10FDE00004D035A10E910DA90D910DE037A1F9E7D1
:10FDF0006146019B009AF0F7A5F90E9B8C469B5C2F
:10FE00000D9A521E0D92137061460143F0D10D9868
:10FE100005A9081A20300190600703D501200004CD
:10FE2000844300E001270198874201DD381A00E091
:10FE30000020019900904118029809180498401A6E
:10FE40000490E00306D421461A9B199A049800F006
:10FE5000B3F94519002706E003A81A9AC05D19995D
:10FE600090476D1C7F1C02988742F5DBE0030CD5A0
:10FE700021461A9B199A049800F09EF9451904E04E
:10FE80001A9A3020199990476D1C0099481E0090CD
:10FE90000029F5DC08E00D980D990078491C0D91BA
:10FEA0001A9A199990476D1C0199481E01900029D2
:10FEB000F1DC63E109280100303132333435363763
:10FEC00038396162636465660000000030313233A6
:10FED0003435363738394142434445460000000046
:10FEE00000F05AF94519761C3078002800D0E2E578
:10FEF00028461BB0F0BD600700D406271898C01D27
:10FF0000C108C90048680A680831C30FDB071891A7
:10FF1000190001D09CA108E0210501D59BA104E0B6
:10FF2000E10701D09AA100E09AA1430011985B0873
:10FF3000109165280CD006DC452809D046281DD034
:10FF4000472841D141E0662818D067283CD13CE0E1
:10FF50000021112F01DB112000E0781C019100909D
:10FF600008A911A8FFF7E8FC139905910021119A3F
:10FF700015927F1C12980197009150E00120C00754
:10FF800003900120019008A9009711A8FFF7D4FC65
:10FF9000139A149905920022119B009212981593BE
:10FFA000059A0192002901D0104602E0791C401800
:10FFB0000190381A01D5019804E04042401E00909B
:10FFC000781C0190C01B029043E0012F00DA01274A
:10FFD0000021112F01DD112000E038460191009031
:10FFE00008A911A8FFF7A8FC13990591119A0021FF
:10FFF000129815920091019721070CD40599B942E6
:020000040801F1
:1000000001DB019900E00191012904DD159A491EE7
:10001000515C302906D0B84201DA011D05DA012110
:10002000029115E00199491EEDE7002805DC0099D1
:10003000411800910199091A03E0019A411C91426B
:1000400000DD01910099401A401C02900120C00778
:100050000390200706D402990198814202DB002018
:10006000C043029000206946C87707AF012103987A
:100070000337C907884224D0022011902B20129008
:10008000039800280CDA404203902D20129007E0DC
:100090000A210398F0F72CF830317F1E0390397055
:1000A0001199481E11900029F2DC03980028EFD125
:1000B000791E129808703078202108404530BF1E04
:1000C000387006A8C01BC01D039010980078002847
:1000D00000D00120019941180298C017091803980F
:1000E00009180498401A401E0490E00306D42146E3
:1000F0001A9B199A049800F05FF845191098007837
:10010000002803D01A9A199990476D1CE00324D552
:1001100021461A9B199A049800F04EF845191CE0E4
:100120000098002807DB00990598884203DD1598A0
:10013000405C199901E0199930201A9A904700986B
:100140006D1C401C00900298401E0290002804D1B3
:100150001A9A2E20199990476D1C0199481E0190FA
:100160000029DDDC05E038781A9A7F1C1999904740
:100170006D1C0399481E03900029F4DC21461A9B4C
:10018000199A0498ACE600002D0000002B00000036
:100190002000000000000000F8B5044600251E46BF
:1001A0001746880404D405E039462020B0476D1C6A
:1001B000641EF9D52846F8BDFFB50446002581B078
:1001C0001E46C80301D5302700E02027880404D547
:1001D00005E038460399B0476D1C641EF9D52846E2
:1001E00005B0F0BD4A68002A06D00A68531C0B60AF
:1001F00010704868401E48607047F0B50E461746BC
:100200000146E037387C85B0154600281DD02A46C7
:10021000684602F0F5F8012408E002F0F9FF210138
:100220006846491904F0A2FC641CE4B2387CA04280
:100230006846F2D803F0C4FE2001421969463046F0
:1002400002F0DEF8002005B0F0BDFF20FBE7000063
:10025000F0B51346E03389B014460D46102908D096
:10026000182D06D0202D04D000201874FF2009B0CE
:10027000F0BD224603E006781670401C521C0E4664
:10028000491EC9B2002EF6D1A8007030C0B201904C
:100290000009401E187401202E4606904FE0A71951
:1002A00038462038017F0491417F0591817F039179
:1002B000C07F029029463046EFF71AFF002904D08C
:1002C000182D27D9102918D024E01F48059A069B1D
:1002D000825C04995A400492039A825C0592029AC5
:1002E000825C0392405C0290FF225800D9091C32C4
:1002F00051434840C0B206900CE013480499415C59
:1003000004910599415C05910399415C039102991F
:10031000405C0290701BC0B2215C049A20185140CE
:10032000A1554178059A514079708178039A5140DE
:10033000B970C07802994840361DF870F6B201983D
:100340008642ACD3002092E7C0530108F0B50446C2
:100350004F008E488FB07F080D460D91874228DBF5
:100360004042381820430CD08948874203DC87423A
:1003700018D1002C16D020462946FFF7D9F90FB026
:10038000F0BD844A844B20462946F0F713FA07460D
:100390000E46824A824B20462946F0F70BFA3A462F
:1003A000334649E00120FFF7C1FAFFF7CAF90FB061
:1003B000F0BD7C48874243DAF920800587420BDA9A
:1003C00020462946FFF722F9042801D1FFF7C2F998
:1003D000204629460FB0F0BD22462B46104629463E
:1003E000F0F7E8F9064602466F480F460B4606212D
:1003F0007844FFF747F932463B46F0F7DBF90690C1
:100400006A48079132463B4604217844FFF73AF99F
:1004100032463B46F0F7CEF900225C4BF0F718F974
:1004200002460B4607990698F0F72CFA22462B460F
:10043000F0F7C0F922462B46F0F70AF90FB0F0BDED
:100440002046524C6900490800222346F0F7AAF9D9
:100450000022D243F0F78EFA0546024654480E4673
:100460000B4606217844FFF70DF92A463346F0F78C
:10047000A1F906904F4807912A4633460421784453
:10048000FFF700F92A463346F0F794F90022234695
:10049000F0F7DEF8059104902846314603F0E0FDC0
:1004A000089045480C46874219DB059B049A07993A
:1004B0000698F0F7E7F902460B4621460898F0F750
:1004C00079F92346089AF0F7C3F80122F0F752FAB7
:1004D000304A314BF0F760F9304A314B4AE000279F
:1004E0003A460B460898F0F7B3F83A4623460A9185
:1004F0000E9010461946F0F75DF92A463346F0F79C
:1005000051F90A9B0E9AF0F7BDF905460E46059B78
:10051000049A07990698F0F7B5F900910490012222
:1005200028463146F0F726FA1A4A1B4BF0F73AF9FB
:100530000E460546012221460898F0F71BFA009B5B
:10054000049AF0F737F92A463346F0F725F90546BD
:100550000E46012238462146F0F70CFA0F4C174F91
:1005600022463B46F0F71EF92A463346F0F71AF9C1
:1005700022463B46F0F716F90D9A002A00DD5DE7AA
:100580000122D20751400FB0F0BD00000000F03F43
:100590000000F07F075C143326A6913C182D4454CC
:1005A000FB21F93F0000E03FCC520000E252000086
:1005B000585200006E5200003333EF3FFB21E93FF9
:1005C00010B50348006803F0F5F8002010BD0000E6
:1005D000C401002008B56A4609A103F0A9FF01285B
:1005E00001D0022008BD0748009A0749824204D280
:1005F000086006A0FEF71CFCF3E700200A6008BDB7
:10060000256C750010270000C4010020414345748B
:10061000696D652073657474696E67206D75737498
:10062000206265206D6F7265207468616E203130C4
:10063000530A0D000EB50220694608706846F8F7A7
:1006400091FA04F0A9F8002804D16846007903F073
:10065000B1F800200EBD0EB502216A461170007877
:10066000302805D0312801D002200EBD012000E045
:10067000002010711046F8F7F1FA04F08DF80EBD65
:1006800010B502F03BF903F069F8002010BD1CB56D
:1006900004460222694603F047FD082804D00122DF
:1006A0006946204603F040FD684602F02BF9002021
:1006B0001CBD10B502F030F903F02AF8002010BD7F
:1006C0001FB504460222694603F0F4FC102804D04A
:1006D00001226946204603F0EDFC684602F020F94D
:1006E000002004B010BD10B502F030F903F010F88E
:1006F000002010BD1FB504460222694603F0DAFC53
:10070000102804D001226946204603F0D3FC684635
:1007100002F020F9002004B010BD000010B586B032
:100720006846F1F7AFFF044C04A02188FEF780FB78
:100730000028F9D106B010BD8C01002025640D0AF7
:100740000000000010B501F037FB01F065FB002050
:1007500010BD00003EB5012168460170F8F702FAAD
:10076000044668460079012805D122480078C00770
:1007700001D005203EBD20A0FEF75AFB0028FAD18B
:100780002CA0FEF755FB0028FAD12B48FEF70EFBF4
:100790002A48FEF70BFB2A48FEF708FB2948FEF71C
:1007A00005FB2948FEF702FB2848FEF7FFFA03F095
:1007B0001DF87D20C000F2F78CFA002C17D1684696
:1007C0000079012804D022480078002807D00EE0E4
:1007D00020A0FEF72DFB0028FAD11C4805E01DA043
:1007E000FEF726FB0028FAD11448FEF7A7FA0020EE
:1007F0003EBD0000D40400200A0D53746F702054D5
:1008000078206576656E74732C506C656173652015
:100810007761697420666F7220616C6C20636F6E03
:1008200066696775726174696F6E7320746F20708A
:1008300072696E740D0A0000DC1B00200C1C002085
:10084000701C0020201C0020341C0020E01200201E
:10085000A50300200A0D537461727420547820653A
:1008600076656E74730D0A0010B501F007FF02F093
:10087000A1FF002010BD000008B56A4609A103F0E1
:1008800057FE012807D108490098084A41189142AB
:1008900003D3002801D0022008BD01F0F5FE00209E
:1008A00008BD0000256C7500FF1E0AFAFEE8A4359D
:1008B00070B5054D01242C7004A0FEF7B9FA00288C
:1008C000FAD12C7070BD00005C030020456E746589
:1008D00072204465627567206D6F64650D0A0000C3
:1008E0000EB51520694608706846F8F73BF903F025
:1008F00053FF002805D169460420085602F05AFF2C
:1009000000200EBD08B56A460AA103F011FE0128B9
:1009100001D0022008BD694600200856082801DBE6
:10092000032008BD02F0A8F804A0FEF781FA002811
:10093000FAD108BD2568687500000000417474652F
:100940006E74696F6E3A54616B65206566666563A7
:10095000742061667465722041542B4144523D30CD
:100960000D0A000010B501F0FFFF002010BD38B5E2
:1009700004460222694603F015FC042804D0012233
:100980006946204603F00EFC009802F011F80020A2
:1009900038BD10B502F012F802F0E0FE002010BDE4
:1009A0001CB504460222694603F0BEFB082804D0A9
:1009B00001226946204603F0B7FB684602F002F8C0
:1009C00000201CBD0EB50020694608706846F8F787
:1009D000C9F803F0E1FE002807D16846017903A0B9
:1009E0004131FEF725FA0028F7D10EBD25630D0A27
:1009F000000000000EB500216A4611700078412801
:100A000005D0422803D0432801D002200EBD413832
:100A100010711046F8F722F903F0BEFE0028F5D158
:100A200002A0FEF705FA0028FAD10EBD41747465E4
:100A30006E74696F6E3A54616B65206566666563B6
:100A4000742061667465722041545A0D0A000000DA
:100A50000EB51920694608706846F8F783F803F068
:100A60009BFE002803D1019802F0B2FE00200EBDCB
:100A70000EB519216A46117006A101AA03F058FDAE
:100A8000012801D002200EBD6846F8F7E7F803F010
:100A900083FE0EBD256C750010B501F09DFF012889
:100AA00006D006A0FEF7C4F90028FAD1002010BD38
:100AB00003A0FEF7BDF90028FAD1F7E7300D0A00D0
:100AC000310D0A0010B50078302803D0312803D04A
:100AD000022010BD002000E0012001F083FF002073
:100AE00010BD00000648F2F779FA05488030F2F7A9
:100AF00075FA04A0FEF79CF90028FAD1F8F7BEFEBB
:100B0000808F01084F4B0A0D0000000010B5F6F76A
:100B10007BFD002010BD0EB51220694608706846A6
:100B2000F8F720F803F038FE002803D1019802F00E
:100B30004FFE00200EBD00000EB512216A46117056
:100B40000AA101AA03F0F4FC012801D002200EBD85
:100B50006846F8F783F803F01FFE0028F7D104A0D9
:100B6000FEF766F90028FAD10EBD0000256C75006D
:100B7000417474656E74696F6E3A54616B6520657B
:100B800066666563742061667465722041545A0D0F
:100B90000A0000000EB51320694608706846F7F792
:100BA000E1FF03F0F9FD002803D1019802F010FEE7
:100BB00000200EBD0EB513216A4611700AA101AACC
:100BC00003F0B6FC012801D002200EBD6846F8F7FC
:100BD00045F803F0E1FD0028F7D104A0FEF728F95D
:100BE0000028FAD10EBD0000256C750041747465B3
:100BF0006E74696F6E3A54616B65206566666563F5
:100C0000742061667465722041545A0D0A00000018
:100C100010B50348006802F0CDFD002010BD0000B3
:100C2000C801002038B56A4609A103F081FC0128FB
:100C300001D0022038BD074C0098074DA04204D2D5
:100C400006A0FEF7F5F82C60F3E72860002038BD19
:100C5000256C7500407E0500C80100204B415420E2
:100C600073657474696E67206D7573742062652096
:100C70006D6F7265207468616E20366D0A0D00001C
:100C800010B50348007802F095FD002010BD00006B
:100C9000AD03002008B56A460BA103F049FC01280A
:100CA00010D10098411E052907D80849087008A0EE
:100CB000FEF7BEF80028FAD108BD0EA0FEF7B8F87E
:100CC0000028FAD1022008BD25640000AD030020F1
:100CD000417474656E74696F6E3A54616B6520651A
:100CE00066666563742061667465722041545A0DAE
:100CF0000A0000004D6F6465206F662072616E67A8
:100D000065206973203120746F20360D0A000000C1
:100D100010B5044C04A06179FEF78AF80028F9D1D7
:100D200010BD00005C03002025640D0A00000000D7
:100D300008B56A4609A103F0FBFB012807D1084862
:100D40000078012803D168460078042801D90220E0
:100D500008BD04494871002008BD0000256400005A
:100D6000A90300205C03002010B5044C04A0A17965
:100D7000FEF75EF80028F9D110BD00005C030020EA
:100D800025640D0A0000000008B56A460FA103F0B3
:100D9000CFFB012811D10E48007801280DD800287A
:100DA00002D0012805D00AE068460078042804D85B
:100DB00005E068460078052801D9022008BD68468C
:100DC000044900788871002008BD000025640000F7
:100DD000A90300205C030020F0B585B0032069461C
:100DE000087101A8F7F7BEFE03F0D6FC00280FD16A
:100DF0000298009068460478C7788678457832462D
:100E00002B46394603A00094FEF712F80028F6D1CD
:100E100005B0F0BD253032782025303278202530DD
:100E2000327820253032780D0A0000003EB50546A4
:100E300003206946087002226C46284601A903F087
:100E4000B1F9042804D00122211D284603F0AAF993
:100E50006846F7F703FF03F09FFC3EBD10B501F0B5
:100E6000E7FD012800D0002002F0A4FC002010BD06
:100E700010B50078302803D0312803D0022010BDEF
:100E8000002000E0012001F0D9FD03A0FDF7D0FF14
:100E90000028FAD110BD0000417474656E74696F4A
:100EA0006E3A54616B6520656666656374206166A1
:100EB0007465722041545A0D0A0000000EB50120DD
:100EC000694608706846F7F74DFE002801D00120FA
:100ED0000EBD68460079002800D0012002F06AFCAF
:100EE00000200EBD10B501F095FD02F011FC0020B0
:100EF00010BD1FB504460222694603F0DBF8102836
:100F000004D001226946204603F0D4F8684601F077
:100F100085FD002004B010BD10B5064C2068EFF729
:100F2000E3FD02460B4604A0FDF782FF0028F5D141
:100F300010BD0000BC030020252E32660D0A000003
:100F40007CB501AB6A4614A103F0F2FA022803D182
:100F500068460079642801D302207CBD104E092820
:100F600004D8EFF743FD00220E4B03E0EFF73EFD00
:100F700000220D4BEFF786FC044668460D460088BC
:100F8000EFF734FD22462B46EFF762FBEFF7E8FD63
:100F9000306000207CBD000025642E256400000028
:100FA000BC03002000002440000059400EB507207B
:100FB000694608706846F7F7D5FD03F0EDFB002899
:100FC00004D16846007902F0F5FB00200EBD0EB595
:100FD00007216A4611700078302805D0312801D0E9
:100FE00002200EBD012000E0002010711046F7F72E
:100FF00035FE03F0D1FB0EBD10B50348008802F0AA
:10100000D9FB002010BD00004603002008B50021D8
:101010006A4611800AA103F08BFA012801D0022050
:1010200008BD68460088074A411E914203D8064918
:101030000880002008BD05A0FDF7FAFEEFE70000DC
:10104000256C7500FEFF00004603002054686520F3
:10105000524A5444432072616E676520697320319F
:1010600020746F2036353533350A0D0010B503482E
:10107000007802F09FFB002010BD00009A010020C4
:1010800008B500216A46117009A103F051FA012840
:1010900001D0022008BD68460078042803D805491D
:1010A0000870002008BD04A0FDF7C2FEF1E70000B3
:1010B000256400009A0100205468652072657370F1
:1010C0006F6E7365206C6576656C2072616E676506
:1010D000206973203020746F20340A0D0000000056
:1010E00010B50B4C0BA0617AFDF7A2FE0028F9D1D8
:1010F000E06A002806D0084908A0FDF799FE0028FC
:10110000F9D1E06206A0FDF793FE0028FAD110BDE8
:101110005C03002025643A00E414002025730000DD
:101120000D0A000070B50D4D0DA0697AFDF780FE27
:101130000028F9D100240B4E06E0315D0AA0FDF72E
:1011400077FE0028F9D1641CE86A8442F5D308A030
:10115000FDF76EFE0028FAD1E86270BD5C03002046
:1011600025643A00E4140020253032782000000085
:101170000D0A00000EB51020694608706846F7F7A2
:10118000F1FC03F009FB002803D1019802F020FBD9
:1011900000200EBD0EB510216A46117006A101AAED
:1011A00003F0C6F9012801D002200EBD6846F7F70A
:1011B00055FD03F0F1FA0EBD256C75000EB50A2041
:1011C000694608706846F7F7CDFC03F0E5FA002899
:1011D00004D16846007A02F0EDFA00200EBD00004E
:1011E0003EB504460A20694608706846F7F7BAFC1F
:1011F00003F0D2FA002807D107A1204602AA03F083
:1012000097F9012801D002203EBD6846F7F726FD78
:1012100003F0C2FA3EBD00002568687500000000BA
:101220000EB51120694608706846F7F79BFC03F07D
:10123000B3FA002803D1019802F0CAFA00200EBDCB
:101240000EB511216A46117006A101AA03F070F9CA
:10125000012801D002200EBD6846F7F7FFFC03F01D
:101260009BFA0EBD256C75000EB50A206946087004
:101270006846F7F777FC03F08FFA002803D101984E
:1012800002F098FA00200EBD3EB504460A206946D9
:1012900008706846F7F766FC03F07EFA002807D16D
:1012A00007A1204601AA03F043F9012801D002203A
:1012B0003EBD6846F7F7D2FC03F06EFA3EBD000073
:1012C000256C750038B50446EEF7DAFFC5B26A46FC
:1012D00016A1204603F02CF901280AD102E06D1E68
:1012E000EDB2641C207830380928F8D920783A28E3
:1012F00004D00FA0FDF79CFD022038BD6D1E611CBF
:10130000EDB2402D00D94025134C2A46206801F04B
:101310005DFF25710098607101F096FB0146204643
:10132000F6F7FEFC0028E8D0012038BD25753A000C
:1013300041542B53454E4420776974686F7574206F
:10134000746865206170706C69636174696F6E2088
:10135000706F7274000000008C030020FEB504461C
:10136000EEF78EFFC6B2002501AA21A1204603F0A8
:10137000DFF8012806D01FA0FDF75AFD29E0761EF0
:10138000F6B2641C207830380928F8D920783A2839
:10139000F1D1671C761EF4B20020694688701F4E9A
:1013A00013E068003A5C69460A70C01940784870DA
:1013B00030681BA14219684603F0BAF8012808D129
:1013C000A41E6D1CE4B2402D01D2012CE9D8002CE2
:1013D00001D00220FEBD35710198707101F034FB1F
:1013E00001460E48F6F79CFC0028F3D00120FEBD14
:1013F00025753A0041542B53454E44207769746853
:101400006F757420746865206170706C69636174B5
:10141000696F6E20706F7274000000008C030020F2
:10142000256868780000000010B50348006802F0E5
:10143000C1F9002010BD0000C001002038B56A4687
:1014400009A103F075F8012801D0022038BD074C2E
:101450000098074DA04204D206A0FDF7E9FC2C60DD
:10146000F3E72860002038BD256C75007017000078
:10147000C00100205444432073657474696E672072
:101480006D757374206265206D6F7265207468617C
:101490006E2036530A0D00000EB5162069460870FE
:1014A0006846F7F75FFB03F077F9002805D1694636
:1014B0000420085602F07EF900200EBD0EB516215C
:1014C0006A4611700AA101AA03F032F8012801D07E
:1014D00002200EBD6846F7F7C1FB03F05DF9002856
:1014E000F7D105A0FDF7A4FC0028FAD10EBD00003D
:1014F0002568687500000000417474656E74696F3A
:101500006E3A54616B65206566666563742061663A
:101510007465722041542B4144523D300D0A000045
:101520000EB51820694608706846F7F71BFB03F0F4
:1015300033F9002803D1019802F04AF900200EBDCA
:101540000EB518216A46117006A101AA02F0F0FF3B
:10155000012801D002200EBD6846F7F77FFB03F09B
:101560001BF90EBD256C750010B501F06DFA012850
:1015700000D0002002F01EF9002010BD10B5007848
:10158000302803D0312803D0022010BD002000E015
:10159000012001F05FFA002010BD10B501F0CAF97A
:1015A00002F008F9002010BD08B56A4606A102F055
:1015B000BFFF012801D0022008BD6946002008565F
:1015C00001F0BEF9002008BD256868750000000024
:1015D00010B50348C06802F0EDF8002010BD00000F
:1015E0005C03002008B56A4605A102F0A1FF0128AE
:1015F00001D0022008BD03490098C860002008BD42
:10160000256C75005C030020F8B5394C39482188F9
:101610000078014308D000280CD0012821D00228EE
:1016200036D003284BD060E033A0FDF701FC002842
:10163000FAD15AE020880A210746EEF759FD0E46F6
:101640000A21EEF755FD0D4664213846EEF750FDB0
:10165000014633462A462BA0FDF7EAFB0028E9D1D4
:1016600043E020880A210746EEF742FD0D460A2195
:10167000EEF73EFD0E4664213846EEF739FD014691
:101680002B46324624A0FDF7D3FB0028E9D12CE0FD
:1016900020880A210746EEF72BFD0E460A21EEF7B9
:1016A00027FD0D4664213846EEF722FD01463346FC
:1016B0002A461EA0FDF7BCFB0028E9D115E02088D2
:1016C0000A210746EEF714FD0E460A21EEF710FD3B
:1016D0000D4664213846EEF70BFD014633462A4697
:1016E00018A0FDF7A5FB0028E9D10020F8BD0000F7
:1016F000B4030020A90300204C37302D524C0D0AB2
:10170000000000007625642E25642E25642C4C37BD
:10171000302D524C0D0A00007625642E25642E25AE
:10172000642C4C37362D4C0D0A0000007625642EB3
:1017300025642E25642C75626C6F782D4D415837C9
:101740000D0A00007625642E25642E25642C756212
:101750006C6F782D4D4158380D0A00001CB56B4652
:1017600001AA0BA102F0E4FE022807D16846808896
:10177000962803D369460978092901D902201CBD9E
:10178000054A117005490880F1F7A8FA00201CBD30
:1017900025642C2564000000A9030020B403002068
:1017A00010B501F02BF9012800D0002002F002F85A
:1017B000002010BD10B50348806A01F0FBFF002037
:1017C00010BD00005C03002010B5064A06A102F01F
:1017D000AFFE012801D0022010BDF5F7ADFD0020BD
:1017E00010BD000084030020256C750010B503486F
:1017F000406901F0DFFF002010BD00005C03002005
:1018000010B5054A05A102F093FE012801D002207F
:1018100010BD002010BD000070030020256C750075
:1018200010B50A4CA069032807D009A0A169FDF7EB
:10183000FFFA0028F9D1002010BD07A0636A226AD0
:10184000A169FDF7F5FA0028F7D1F4E75C03002061
:1018500025640D0A0000000025642C25642C2564F5
:101860000D0A00001FB50446002103A80291039150
:10187000009002AB01AA14A1204602F059FE0328F1
:101880000FD001AA13A1204602F052FE012808D071
:101890000298FF2805D90398FF2802D9022004B036
:1018A00010BD0198002803D0F5F702FA0A49086034
:1018B0000A480199816102990162039941620121FB
:1018C000C1710020EBE7000025642C25642C256401
:1018D0000000000025640000E40100205C030020FB
:1018E00010B50348C06901F065FF002010BD00007D
:1018F0005C03002010B5054A05A102F019FE01287D
:1019000001D0022010BD002010BD0000780300208F
:10191000256C7500F7F7B2FF0120704710B501F094
:101920009FF801F047FF002010BD000010B50348EC
:10193000006901F03FFF002010BD00005C030020A3
:1019400010B504460078302802D031280CD102E0CE
:10195000F5F720FD01E0F5F717FD054A05A1204642
:1019600002F0E6FD012801D0022010BD002010BDCC
:101970006C030020256C750010B501F077F801F0BC
:1019800027FF002010BD000010B50348407801F08B
:1019900011FF002010BD00005C03002008B56A465E
:1019A00007A102F0C5FD012808D10098FF2805D83D
:1019B000044901228A704870002008BD022008BD39
:1019C000256400005C03002010B50348C07801F0D6
:1019D000F1FE002010BD00005C03002008B56A463F
:1019E00007A102F0A5FD012808D10098FF2805D81D
:1019F000044901220A71C870002008BD022008BDF8
:101A0000256400005C03002010B504A0FDF710FA67
:101A10000028FAD102F030F9002010BD76312E36C0
:101A20002E352000F0B589B004460D4648000691D9
:101A300072494008884215DB7149884203DC8842BC
:101A400007D1002C05D020462946FDF771FE09B0CC
:101A5000F0BD6C48002D02DD6B4909B0F0BD6B494B
:101A600009B0F0BD6A49884211DA6A4988420BDA46
:101A700020462946FDF7CAFD042801D1FDF76AFE7C
:101A80002046294609B0F0BD0026F6435DE06D0012
:101A900061496D08884232DA6049884219DA0026C5
:101AA000012332469B0720462946EEF7D1FD074623
:101AB0000191012220462946EEF75CFF0022584B97
:101AC000EEF76AFE3A46019BEEF7DCFE04460D4651
:101AD0003BE001260022524B20462946EEF7B8FD96
:101AE0000746009100224E4B20462946EEF754FE51
:101AF0003A46009BEEF7C6FE04460D4625E04949EE
:101B0000884219DA02260022474B20462946EEF782
:101B100051FE0022424BEEF79BFD07460291002248
:101B2000414B20462946EEF737FE3A46029BEEF738
:101B3000A9FE04460D4608E0032622462B46002057
:101B40003A49EEF79FFE04460D4622462B461046C4
:101B50001946EEF72FFE07460B4602460191EEF7B7
:101B600029FE0246029032480B4603910621784432
:101B7000FDF788FD3A46019BEEF71CFE00902D48CC
:101B8000019105217844039B029AFDF77BFD039B9D
:101B9000029AEEF70FFE02460B4601990098002EBE
:101BA0000BDAEEF755FD22462B46EEF703FE2246F2
:101BB0002B46EEF7F7FD09B0F0BDEEF749FD2246E2
:101BC0002B46EEF7F7FD1C4AF6007A4493191A6883
:101BD0005B68EEF7E1FD22462B46EEF7DDFD174A86
:101BE0007A4493191A685B68EEF7DCFD069A002ABE
:101BF000E1DA0122D207514009B0F0BD00001044E3
